:020000040000FA
:10000000008000104D020000550200005702000061
:10001000590200005B0200005D020000F671FFEF74
:100020000000000000000000000000005F0200006F
:100030006102000000000000630200006502000091
:10004000670200006702000067020000670200000C
:1000500067020000670200006702000067020000FC
:1000600067020000670200006702000067020000EC
:1000700067020000670200006702000067020000DC
:1000800067020000670200006702000067020000CC
:1000900067020000670200006702000067020000BC
:1000A00067020000670200006702000067020000AC
:1000B000670200006702000067020000670200009C
:1000C0006702000000F002F800F098F80AA090E83B
:1000D000000C82448344AAF10107DA4501D100F003
:1000E0008DF8AFF2090EBAE80F0013F0010F18BF38
:1000F000FB1A43F00103184714600100346001004B
:10010000103A24BF78C878C1FAD8520724BF30C843
:1001100030C144BF04680C60704700000023002415
:1001200000250026103A28BF78C1FBD8520728BF07
:1001300030C148BF0B6070476E2900F07D86702982
:1001400000F0A781662914F02A82652914F027821D
:10015000672914F02482612914F0238203681B0AA2
:1001600028BF41F08001692900F01881642900F05E
:100170001581752900F012816F2901F06D817829B0
:1001800000F07381E92901F00781E42901F004817D
:10019000F52901F00181EF2901F06A81F82900F0C9
:1001A00072810368DB0928BF41F08001632902F0F6
:1001B000AF84732902F0B484E32902F0BF84F329E9
:1001C00002F0C484002070471FB59DE8030000F0D2
:1001D00042FD00F0E6FB02F063FA0400002000217B
:1001E00013F072F8401C60600020002113F056F8F4
:1001F000E06002F08FF900F0F3FC1FBD0CF098F9FD
:10020000114603B40CF0A3F903BCFFF7DDFF03F0C4
:10021000D8FE0CF07BFC00000B49D1F800C04A6806
:100220005CF8043B1068184442F8040B8C4528BF66
:10023000A1F1DC0C8A4228BFA1F1DC02C1F800C0A8
:100240004A6020F000407047A01200100648804726
:1002500006480047FEE7FEE7FEE7FEE7FEE7FEE7AB
:10026000FEE7FEE7FEE7FEE7D93F0000C50000001D
:1002700070B5064600F03EF8056806F10B0020F068
:100280000704B4429CBF002070BD2B466A68BAB117
:100290001068A04210D304F1080188423CBF5068A6
:1002A000586007D35168101941601168091B01603B
:1002B00058601460101D70BD13465268002AE7D1C3
:1002C0002146284600F0B3FC0028DED170BD0000B6
:1002D0001CB50C46064B7B4469460090204600F056
:1002E000D2FF04460020694600F0E0FF20461CBD16
:1002F000D30F000000487047A8120010FFFFFFFF57
:1003000070B50446051FFFF7F5FF0068002C14BF09
:10031000446870BD002C18BFAC423CBF20466468E6
:10032000F8D301680A18AA4218BF456003D12A68A9
:1003300005461144016028684119A1421CBF6C6048
:1003400070BD6168696021680844286070BD0B4613
:100350000146184600F0B0BF0FB4044910B503AA17
:10036000029800F0A9FF10BC5DF814FB1C110010EE
:100370000FB41CB5084B06AA7B446946009005984B
:1003800000F081FF04460020694600F08FFF204600
:100390001CBC5DF814FB0000310F00002DE9F0419A
:1003A0000646002410687529314616A510D000F0C5
:1003B000AFFC002802DA404213A507E031688A0743
:1003C00001D512A502E0490704D511A5012401E0D9
:1003D00000F0A7FC00210A2206F1240709E0B0FB87
:1003E000F2FCB0FBF2F302FB1C00303078541846EC
:1003F000491C0028F3D123462A463046BDE8F04187
:1004000000F0C1BC000000002D0000002B00000027
:1004100020000000F0B40D460188090502D5214CEA
:100420007C4402E01F4C7C440E34002100F1240681
:1004300008E002F00F071209E75D42EA03721B09A8
:100440007754491C52EA0307F3D1027800231207BC
:1004500004D5702D06D009B1022311342246F0BC18
:1004600000F091BC01231034F8E770B504460D4646
:100470002146106800F055FC024629462046BDE89A
:1004800070400023C6E7D21D22F00703D3E9002302
:10049000C0E70368126843F0200303600823C361C8
:1004A0000023B7E79C4601002DE9F05F894604462A
:1004B0004FF0000ADFF874B1FB44C0F820A02046DA
:1004C000E1688847002874D0252806D0D4E90121A6
:1004D0009047206A401C2062F1E700265F462046D4
:1004E000E16888472028054607DB312D05D27819B9
:1004F00010F8200C08B10643F1E7B00701D526F04B
:100500000406C4F81CA00027C4F818A02A2D09D09E
:1005100028460CF015F838B304EB8708303DC8F8CE
:10052000185019E059F8041B204604EB870291612A
:10053000E1688847012F054618D1E069002820DAD4
:1005400026F020061DE0D8F8180000EB800005EB2F
:1005500040003038C8F818002046E1688847054652
:100560000BF0EEFF0028EED1012F0AD02E2D08D17E
:100570002046E16888477F1C0546022F46F020068A
:10058000C4DBA069002803DA404246F00106A061FE
:10059000F00701D026F010066C2D0BD0682D09D085
:1005A0004C2D39D06A2D35D0742D35D07A2D33D0DD
:1005B00016E038E0E1682F4620468847B8420546F5
:1005C00009D16C2F26D04FF48060E16806432046A5
:1005D0008847054604E06C2F1AD04FF4807006431C
:1005E0000DB3A5F14100192802D8203546F4006664
:1005F0004A462946204626604E46FFF79DFD80B1BB
:1006000001280BD0F61D26F0070000F1080956E777
:100610004020E4E78020D8E70020D6E706F104096F
:100620004DE7284652E7206ABDE8F09F2C460100BE
:1006300000B589B000926A4601F0D6FA09B000BD53
:100640000FB400B58DB010A9099000910B904FF038
:10065000FF300A9000200C90064878440690064827
:1006600078446A4607900F9909A801F08DFA0DB0F9
:100670005DF814FB4B150000631500002DE9FF5FCA
:100680001D464FF0FF3B91464FF000085F46D5E90D
:100690000146A96901987F1C8847296A82468847D4
:1006A0000028F6D1BAF1FF3F0CD0002E24F4C0642C
:1006B00019DD600614D5BAF12B0F09D0BAF12D0F50
:1006C0000ED103E0584604B0BDE8F09F44F48064C6
:1006D000A96901987F1C8847761E8246002E02DD9C
:1006E000BAF1300F03D0B9F1000F26D032E0A9697A
:1006F000761E01987F1C44F400748847002E8246C1
:1007000005DDBAF1780F06D0BAF1580F03D0B9F170
:10071000000F10D01EE0B9F1000F02D0B9F1100F98
:1007200018D1A969761E01987F1C24F400748847AB
:100730008246102002E0082000E00A20814609E0FD
:10074000A96908FB0908761E01987F1C44F400740F
:1007500088478246002E05DD4946504600F092FE4D
:100760000028EDDAE96901988847A00502D46FF006
:100770000100A8E7E00725D1600613D5600502D582
:10078000C8F1000000E0404629680A1D2A60096897
:10079000220501D5087015E0220701D5088011E077
:1007A00008600FE02868011D29600068210502D556
:1007B00080F8008006E0210702D5A0F8008001E063
:1007C000C0F8008038467EE770B50446C0688107EF
:1007D00013D0800601D5A56A04E0A16960680844C9
:1007E0002169451A204601F051FE0022064629469D
:1007F000204601F077FD304670BD002070BD70B519
:1008000010B1BDE87040DFE70025074C6E1E07E021
:100810002046FFF7D9FF00B13546206D20F00104D6
:10082000002CF5D1284670BDC81000102DE9F0410C
:100830000C4607461646104600F078F82078611CF2
:1008400061280AD0722802D077283CD102E0012525
:10085000002405E00225042402E0082448F20205F1
:1008600011F8010B2B2806D0622809D011F8010CD1
:1008700074280AD00BE045F0030544F00204EFE7CA
:1008800045F0040544F00104EAE744F0100438465A
:1008900021460BF09FFE411C15D000213161716093
:1008A0004FF40071F560F1617061200704D53046A6
:1008B0000222002101F016FD306D40F0010030658C
:1008C0003046BDE8F0810020FBE72DE9F0410D4600
:1008D0000646104C206DC10704D0410804D020F01A
:1008E0000104F7E722460EE05420FFF7C1FC0700A1
:1008F0000ED0206D47F00101084354212065384691
:1009000000F006F93A4629463046BDE8F0418DE749
:100910000020D6E7C810001011B14FF4807201E03A
:100920004FF480624FF4007301F058BD2DE9F04799
:1009300004464FF000094FF0FF37C568D4E904863C
:10094000A80707D0204601F0A1FD30460BF004FEB9
:10095000002802DA3846BDE8F087280502D540466F
:10096000FFF7CEFC4C21204600F0D2F8206D20F09D
:10097000010020654846EEE70B4910B5A1F17C0265
:100980000A4CC2E93712372106E000EB104342F867
:100990002130074B00FB03400B1EA1F10101F4DCE9
:1009A00010BD0120E8E7000040120010E119D666F2
:1009B000CD0D0100014A01F051BE0000AC01001054
:1009C00010B5431C02E010F8011B71B18107FAD188
:1009D0004FF0013202C88C1A8C4314EAC211F9D0CC
:1009E000C01A0A0603D0C01E10BDC01A10BD0A04EA
:1009F00001D0801E10BD0902FCD0401E10BD40EA8F
:100A0000010370B59B072ED14FF00136042A2AD37B
:100A100008C810C99D1B9D43121F15EAC61517D0A3
:100A2000D8B2E1B2401A50EA056110D198B2A1B231
:100A3000401A50EA05410AD123F07F4024F07F415B
:100A4000401A50EA052102D1180EA0EB146070BDC7
:100A5000A342DBD018BA21BA884201D9012070BD67
:100A60004FF0FF3070BD0AB9002070BD10F8013B97
:100A700011F8014B63B1A3420AD1521E08D010F8FD
:100A8000013B11F8014B1BB1A34201D1521EEDD124
:100A9000181B70BD421E12F8013F002BFBD111F84C
:100AA000013B002B02F8013BF9D1704710B5203A09
:100AB000C0F00B80B1E81850203AA0E81850B1E817
:100AC0001850A0E81850BFF4F5AF5FEA027C24BFCD
:100AD000B1E81850A0E8185044BF18C918C0BDE8C4
:100AE00010405FEA827C24BF51F8043B40F8043B8D
:100AF00008BF7047D20728BF31F8023B48BF11F842
:100B0000012B28BF20F8023B48BF00F8012B70479B
:100B10004FF0000200B5134694469646203922BF96
:100B2000A0E80C50A0E80C50B1F12001BFF4F7AFE1
:100B3000090728BFA0E80C5048BF0CC05DF804EBC3
:100B4000890028BF40F8042B08BF704748BF20F831
:100B5000022B11F0804F18BF00F8012B70470000E6
:100B60004FF0013C50F8042B51F8043B9A4221D13C
:100B7000A2EB0C03934313EACC1317D150F8042BC8
:100B800051F8043B9A4215D1A2EB0C03934313EAAC
:100B9000CC130BD150F8042B51F8043B9A4209D1E5
:100BA000A2EB0C03934313EACC13DBD04FF000000D
:100BB000704700BFD01A01BAB1FA81F101F01801F3
:100BC00022FA01F0CB40C1F12001DBB2C0B2C01A61
:100BD0002CFA01F3D11A914311EAC311E6D17047FF
:100BE00070B5064C7C44064D7D4403E020682044EB
:100BF0008047241DAC42F9D170BD00007856010039
:100C0000785601002DE9F04117460E46054633B1EE
:100C100007FB0354E41B2046B047A542FAD1A5F1D7
:100C20000800BDE8F081704770477047704738B5DD
:100C300004460A460020694602F0B9FA002808BFB7
:100C400038BD02460099204601F032FD012038BD32
:100C5000012002F063BAF8B502F09EFA05460020C2
:100C60000C46102000BF0646A819A0420DD93246F6
:100C70006946002002F09BFA070008BF02F04EFA16
:100C80000098A04218BF0546C419FFF733FB056062
:100C90000746F01D20F007004619284600F00AF824
:100CA000B44208BFF8BDA21B31463868BDE8F84021
:100CB00001F0FEBC00210160C0E901107047102066
:100CC000704770B5044685690068C10601D53026B5
:100CD00000E02026C00707D070BDD4E901213046CE
:100CE0009047206A401C20626D1EF6D570BD70B51D
:100CF000044685690078C00707D170BDD4E9012199
:100D000020209047206A401C20626D1EF6D570BDE1
:100D100009684A0501D540B27047C905FCD500B243
:100D2000704709684A0501D5C0B27047C905FCD5AE
:100D300080B2704770B50C460546012A05D0287868
:100D4000800600D5EA69002302E0012305E05B1C70
:100D5000934202D2E05C0028F9D1A869E618C01AD3
:100D6000A861286A184428622846FFF7AAFF04E011
:100D7000D5E9012114F8010B9047B442F8D3284675
:100D8000FFF7B5FF70BD2DE9F0470D469946924635
:100D9000044600F124080168880604D5E06921F0C2
:100DA0001001216000E00120A84201DD471B00E0A6
:100DB0000027A1697A1902EB0900081AA0612078BE
:100DC000C00602D42046FFF77CFF002608E0D4E9E5
:100DD00001211AF806009047206A401C761C206208
:100DE0004E45F4DB2078C0060AD52046FFF769FFA0
:100DF00006E0D4E9012130209047206A401C20629F
:100E0000381EA7F10107F4DC07E0D4E9012118F846
:100E100005009047206A401C2062281EA5F10105AC
:100E2000F3DC2046FFF763FF2078000602D502209E
:100E3000BDE8F0870120FBE711680268006A5305EE
:100E400001D508700AE0D30501D5088006E0130635
:100E500003D5C217C1E9000200E008600120704715
:100E600070472DE9FF4F0C461E464FF0FF378BB001
:100E7000D2E90001DDF860800A908A46C1F30A5584
:100E800005B93D46002108464FF00000BAF1000FB9
:100E900000F4400005DA00EB80004FF4400101EA65
:100EA00050004FEA9059B9F1010F00DDB9460A9898
:100EB00050EA4A000ED044F61050A5F2FF354543E3
:100EC0002F14B8F1000F1ED07542291E1EDDC9F186
:100ED00000021CE0B8F1010F4FF0000001D03021FA
:100EE00003E0F24305E02154401CB042FBDB3046F6
:100EF0000022002121540B99C1F80880C1E900208B
:100F00000FB0BDE8F08FBD1B6D1CDEE74A4600DA6E
:100F1000694206A801F0E8FF06AB93E8070003ABBF
:100F200083E8070050460A9902F03DFC8DE807006F
:100F3000A0F500501F3800900398002D09DD42F203
:100F40001F014A46084403A90390684602F0C7FE01
:100F500008E0A0F500504A461F3803A903906846F0
:100F600002F0E5FE8DE807000004000C03D04FF00E
:100F7000FF30410800E01046B8F1000F03D0002216
:100F8000009215461EE0751E05D401F0ABFB303211
:100F900062556D1EF9D5B3460122084302D00022E6
:100FA0007F1C04E02078302801D100227F1E002A17
:100FB000099786D01DE0112D07DA01F093FB30323E
:100FC00062556D1C50EA0102F5D1084302D0009829
:100FD000C8B10EE00021681E05E0235C625C63542A
:100FE0002254401E491C8142F7DBAB46A81B401E21
:100FF0000990002004F80B000B98099AC0F80880AB
:10100000C0E9002B7CE711264FF0000859E72DE9D5
:10101000F04F88460446D21D22F0070191B0D1E975
:101020000001CDE90A010BF001F802460B98C00F50
:1010300001D02D2007E02068810701D52B2002E098
:10104000202101EAC000032A099001D0072A05DB0C
:1010500003464146204601F011FD0BE12078800651
:1010600001D5E06900E00620B8F1650F814606D0A1
:10107000B8F1660F18D0B8F1670F70D131E00020D9
:10108000B9F1110F009001DB112301E009F1010317
:101090000AAA01A90CA8FFF7E4FEDDE90C700026FE
:1010A00009F10105834647E001204B4600904FF0CF
:1010B00000470AAA01A90CA8FFF7D3FEDDE90DB08D
:1010C0000C995D46002610B909F101000D18B9EB25
:1010D000050003D4C0F1FF3609F10105A5EB0900B5
:1010E0002BE0B9F1010F01DA4FF001090020B9F14D
:1010F000110F0090484601DD112300E003460AAAC3
:1011000001A90CA8FFF7ADFEDDE90C704D460026E5
:101110008346207800070AD4AB4500DA5D4601A873
:10112000012D04DD411911F8011C302907D04F456C
:1011300002DA17F1040F04DA012082460FE06D1E77
:10114000EEE7002F02DCED1B3E4403E0781CA842D2
:1011500000DD7D1CB81B00F1010A4FF0004720782C
:10116000000703D4AA4501DB4FF0FF3A0021B7F195
:10117000004F0DF143088DF8431024D002202B239B
:10118000002F01DA7F422D230A21021EA0F1010067
:1011900000DC5FB197FBF1FC97FBF1F201FB1C7CDB
:1011A00017460CF1300C08F801CDEEE7A8F101006C
:1011B00003702188090501D5452100E06521A0F1D2
:1011C000010800F8011C09980FA9A1EB0807FF1DF1
:1011D00000B10120411901EBEA70A1693844081AF5
:1011E000401EA0612078C00602D42046FFF769FDAA
:1011F000099828B1D4E901219047206A401C206257
:101200002078C00622D52046FFF75BFD1EE0002EA9
:1012100004DBB34502DD01A8805D00E03020D4E9A5
:1012200001219047206A401C2062761CAAF101002F
:101230005FEA000A0AD101F033FAC0680168405C35
:10124000D4E901219047206A401C2062281EA5F1A4
:101250000105DCDC07E0D4E9012118F8010B904717
:10126000206A401C2062381EA7F10107F3DC2046EB
:10127000FFF73DFD032011B043E6000001694A1C61
:1012800002610878704700B58FB0CDE901310021C7
:10129000059105497944CDE9031011466846FFF7E9
:1012A00003F90FB000BD0000E5FFFFFF0A6802F878
:1012B000010B0A6070470000074B70B50D467B4478
:1012C000FFF7E1FF0446284600F000FE10B14FF0A2
:1012D000FF3070BD204670BD6BB900002DE9FF5F87
:1012E00015468A460446DFF8AC80F8440027D8E962
:1012F00000103E46CDE9001010E03AF816106A469C
:1013000002A801F0DFFE411C07D02178890603D531
:10131000E269391891420DD80744761C207880067E
:1013200002D5E069B84205DDAE42E6DB3AF81600C8
:101330000028E2D1A069C01BA0612046FFF7C1FCD4
:10134000D8E90010CDE90010002017E03AF8181095
:101350006A4602A801F0B6FEB0F1FF3F81460BD00D
:1013600000250DF1080B05E0D4E901211BF805006B
:1013700090476D1C4D45F7D308F10100B0428046FF
:10138000E4DB206A384420622046FFF7B0FCBDE869
:10139000FF9F00000E3801002DE9F0418046D21D6C
:1013A00022F007020025D2E90002F52915A614D083
:1013B000011E72F1000106DA0023D0EB030063EB9B
:1013C000020211A608E0D8F800108B0701D50FA67D
:1013D00002E0490701D50EA601251146002408F1B7
:1013E000240704E001F07EF930323A55641C50EADB
:1013F0000102F7D12B46324621464046BDE8F04176
:10140000FFF7C1BC000000002D0000002B00000011
:101410002000000030B4002100F1240408E002F0B4
:101420000705D208303542EA4372DB086554491C8F
:1014300052EA0305F3D10468002310A2250708D55A
:1014400004F020040C4304D0C46901230CA2641EE0
:10145000C46130BCFFF797BC10B504462146106844
:10146000FFF75FFC02462046BDE810400023D1E7AD
:10147000D21D22F00701D1E90023CBE700000000D4
:10148000300000003A2800D2303820F02002412AF3
:1014900001D3A2F13700884201D34FF0FF307047EB
:1014A0002DE9FF4F1C4691464FF0FF3581B00021DA
:1014B0008A468846D4E90167A16902986D1C88476D
:1014C000216A834688470028F6D1BBF1FF3F0CD044
:1014D000002F26F4C0661ADD700615D5BBF12B0F60
:1014E0000AD0BBF12D0F0FD104E04FF0FF3005B053
:1014F000BDE8F08F46F48066A16902986D1C8847AC
:101500007F1E8346002F02DDBBF1300F03D0B9F1FF
:10151000000F2AD025E0A1696D1C02987F1E46F4B9
:1015200000768847002F834605DDBBF1780F06D093
:10153000BBF1580F03D0B9F1000F10D011E0B9F191
:10154000000F02D0B9F1100F0BD1A1696D1C0298E8
:101550007F1E26F4007688478346102000E008208E
:1015600081464FEAE970009017E00A20F8E7434609
:10157000AAFB0928DDF800C07F1E03FB098046F4A2
:10158000007605F101050AFB0C0112EB0B0A02982B
:1015900041EBEB78A16988478346002F06DD494679
:1015A0005846FFF76FFF5FEA000BE0D5E16902984C
:1015B0008847B00502D46FF0010098E7F00718D112
:1015C000700610D55146700505D50023D1EB0301F7
:1015D00063EB080200E042462068031D23600068B8
:1015E000C0E9001205E02068011D21600068C0E923
:1015F00000A828467BE72DE9FF5F4FF000089946D9
:10160000144646469169D2E901A7DDF838B0019841
:101610008847054659EA0B0005D009E0A169019801
:10162000761C88470546216A284688470028F5D158
:10163000681C03D05FEACA7005D015E04FF0FF3098
:1016400004B0BDE8F09F2068011D2160D0F8008043
:101650000AE05FEACA7001D108F8015BA169761C53
:1016600001987F1E88470546002F1ADD681C18D098
:10167000B9F1000F0DD0E81705EBD060421120F052
:101680001F0059F822102A1A012090400142E0D18F
:1016900007E0BBF1000FDCD12846216A884700280B
:1016A000D7D0E16901988847BBF1000F07D1002E20
:1016B00005DD5FEACA7002D1002188F80010A06839
:1016C000B84203DDBBF1000F03D017B16FF001008A
:1016D000B6E73046B4E700002DE9FF4F064689B073
:1016E0000878FF2806D0491C2D2805D000244FF08B
:1016F000000908E000200CE00124F8E709EB890369
:10170000491C00EB43090878FF28F7D114B1C9F14F
:1017100000008146107800252C46AA4629462D282F
:1017200001D02B2804D1521C2D2813D00020824632
:101730008B461078FF280FD04FF0000C0A21521C66
:10174000A5FB017804FB018105FB0C11C5194BEBCE
:101750000104EEE70120EAE7002108464FF000000F
:10176000BAF1000F02D000EB80004008C0F38158AE
:10177000B8F1010F01DD4FF0FF380C9809EB0007BD
:1017800055EA040009D04FF0020917F5FA7F0BDA89
:101790004FEACA70C6E900B012E04FEACA70C6E963
:1017A00000B00DB0BDE8F08FB7F5FA7F0DDDF04861
:1017B0007844D0E90010C6E9001040EACA707060B1
:1017C00000F072FFC0F80090EBE7391E02DAC8F1B2
:1017D000000200E0424600DA794206A801F084FBEC
:1017E00006AB93E8070003AB83E8070044F23E0032
:1017F0005BEA04010090584604D144F21E012C46D5
:101800005D460091210C0904014306D1009924048E
:1018100044EA15442D041039009104F07F4101433E
:1018200006D10099240244EA15642D02083900917A
:1018300004F07041014306D10099240144EA157473
:101840002D01091F009104F04041014306D1009988
:10185000A40044EA9574AD00891E009104F0004193
:10186000084304D100986D196441401E009042461F
:101870006846002FCDE9014503A902DD02F06BFAAD
:1018800001E002F040FABAF1000F04460D4601D023
:1018900084F0004440F2FF7724F00040284303D056
:1018A000C4F30A50B84212D100F0FEFEC0F8009016
:1018B000C4F30A50B8420AD1AE487844D0E90010C7
:1018C000C6E9001004F000410843706069E7C6E90A
:1018D000005466E72DE9FF4F1F464FF0000A4FF016
:1018E000FF38454691B0D7E90146CDF83CA000F05D
:1018F000D7FEC0680168405C1090B96912986D1CF1
:101900008847396A814688470028F6D1B9F1FF3FF8
:101910000AD0002E24F4D06411DDB9F12B0F08D0C9
:10192000B9F12D0F0BD102E0404615B03AE744F46F
:101930008064B96912986D1C8847761E81466005DF
:1019400004A901D52D2000E02B20002E01F1010B70
:101950000DF130088DF810003FDDB9F1690F08D0A6
:10196000B9F1490F05D0B9F16E0F02D0B9F14E0FA0
:101970001CD13B4601A8009580E85002DDE9121217
:101980006FF0020012F099FEC11CCED10EE0B969D1
:1019900012986D1C884781461398761E44F4007493
:1019A00005600F98401C002E0F9016DDB9F1300F26
:1019B000EDD0B9F1780F02D0B9F1580F0DD10F98D1
:1019C00001280AD13B46CDE90054DDE91212001F7F
:1019D000029612F070FEC11CA7D1109989453ED124
:1019E00044F0800406E01399681CAAF1010A44F44B
:1019F00000740860B9696D1C1298761E88473028FB
:101A00008146F0D02BE01099894505D1200603D4FA
:101A1000761E44F0800418E048460AF091FD08B3B1
:101A2000761E0DF123018B4544F4007408D2A9F110
:101A300030000BF8010B200607D5AAF1010003E0E6
:101A4000200602D40AF101008246A00502D51399AE
:101A5000681C0860B96912986D1C88478146002E81
:101A6000D1DC53E0002E51DDB9F1650F02D0B9F1A0
:101A7000450F4BD1A00549D5B9696D1C1298761E4A
:101A800024F440748847002E81460CDD2B2804D0B6
:101A9000B9F12D0F07D144F48074B96912986D1C07
:101AA0008847761E8146E00501D52D2100E02B21D7
:101AB00008F8011BCDF8008021E0761E0DF13901F8
:101AC000884544F400740CD2A9F1300010F0FF00F6
:101AD00088F8000002D10099884509D908F1010869
:101AE00006E0E00501D5244801E042F20F7082468D
:101AF000B96912986D1C8847814613980560002EBD
:101B000004DD48460AF01CFD0028D6D1F969129878
:101B10008847FF2053468BF8000088F8000000201B
:101B20000A900B9004AA0CA90AA8FFF7D5FDA005FE
:101B300002D46FF00100F8E614F0240F0AD0E00799
:101B400014D13868DDE90A12031D3B600068C0E962
:101B500000120BE00AA968460AF0BCFAE00705D1BA
:101B60003868009A011D3960006802602846DCE68A
:101B7000784901006E480100F1D8FFFF0268114466
:101B80001378016018467047D16005497944516166
:101B900004497944116200211161114600F0DABF55
:101BA000EDFFFFFFD90B0000426842B1016811F858
:101BB000013B23B1521EC0E90012184670470121B3
:101BC000C160881E704742685AB1C368016843B952
:101BD00083688B4205D0491E521CC0E900120020C8
:101BE00070474FF0FF307047034B7B449361034BCA
:101BF0007B44D361FFF7C8BF4BAF0000D313000095
:101C00002DE9FF4F4FF000089A461446C14646465C
:101C100083B0D2E901B7CDF80080CDF80480916996
:101C200004988847109905465AEA010005D009E052
:101C3000A1690498761C88470546216A284688478A
:101C40000028F5D1681C03D05FEACB7005D02AE0EC
:101C50004FF0FF3007B0BDE8F08F2068011D216014
:101C6000D0F800801FE002A86A46E9B201F00CFA41
:101C7000411C07D0801C09D04FF000095FEACB70EF
:101C800007D00AE0E169049888473EE04FF0010977
:101C900004E0BDF8081028F8021B7F1EA169049813
:101CA000761C88470546002F1ADD681C18D0BAF14B
:101CB000000F0DD0E81705EBD060421120F01F0097
:101CC0005AF822102A1A012090400142CBD107E095
:101CD00010980028C7D12846216A88470028C2D01A
:101CE000E16904988847B9F1000F0ED1109830B916
:101CF000002E04DD5FEACB7001D1A8F80000A068D7
:101D0000B84202DD109818B117B16FF00100A1E7D9
:101D100030469FE72DE9FF4F4FF000089B461446E1
:101D2000454683B0D2E90196CDF80080CDF8048015
:101D30009169DDF848A00498884707465BEA0A00E5
:101D400005D009E0A16904986D1C88470746216AFF
:101D5000384688470028F5D1781C03D05FEAC9705F
:101D600005D01BE04FF0FF3007B0BDE8F08F2068D2
:101D7000011D2160D0F8008010E05FEAC97007D132
:101D80006A464046B9B201F09DF9411C31D0804409
:101D9000A1696D1C0498761E88470746002E14DD45
:101DA000781C12D0BBF1000007D03B46DDE91012D1
:101DB00001F08AF80028E0D107E0BAF1000FDCD189
:101DC0003846216A88470028D7D0E16904988847B7
:101DD000BAF1000F06D1002D04DD5FEAC97001D110
:101DE00088F80000A068B04203DDBAF1000F03D00C
:101DF00016B16FF00100B7E72846B5E72DE9FF5FA0
:101E00009B46144600273D469169D2E90196DDF8CC
:101E100040A00198884780465BEA0A0005D009E0A7
:101E2000A16901986D1C88478046216A4046884711
:101E30000028F5D1B8F1FF3F03D05FEAC97005D0A3
:101E400014E04FF0FF3004B0BDE8F09F2068011DA2
:101E5000216007680AE05FEAC97001D127F8028BA8
:101E6000A1696D1C0198761E88478046002E15DDFD
:101E7000B8F1FF3F12D0BBF1000007D04346DDE9C7
:101E80000E1201F021F80028E5D107E0BAF1000FA9
:101E9000E1D14046216A88470028DCD0E1690198F9
:101EA0008847BAF1000F05D1002D03DD5FEAC97044
:101EB00000D13880A068B04203DDBAF1000F03D032
:101EC00016B16FF00100BEE72846BCE7007B00F0CA
:101ED0008000704770B50D4601461446D3685069BE
:101EE0002A460AF069FC002807DA411C07D0E1689D
:101EF00020F0004041F48041E160281A70BD204686
:101F000000F090FA4FF0FF3070BDC168002202600F
:101F100021F4805141F0400111F4C06FC16001D043
:101F20008260704702694168891AC269891A8160B2
:101F300070472DE9F0470446C06840F48000E06037
:101F4000010312D520F40020E060810606D4E26A85
:101F500061688A4200D80A46511A216040F4001094
:101F6000E06094F82500BDE8F08720F40010E06000
:101F7000800602D5204600F0ACFAE06842F281010A
:101F80004FF0FF390140012903D0204600F04AFA02
:101F9000B6E02168002600290ADAC94340F48050DF
:101FA0002160C4E902606068411C61600078DAE782
:101FB00044F2400108420CD020F4A04040F0400020
:101FC0002660E06021696068401AE169401AA060FB
:101FD00096E0216991B9C00310D4E069FEF748F991
:101FE0002061B0B1E06840F4006010F4407FE06030
:101FF00002D140F48070E06020696060E068D4F84D
:1020000014A0C1061AD5C0030ED5204600F03EFA32
:1020100014E004F1240020610120E061E06820F474
:10202000407040F48060E6E721696068401AA16969
:10203000014450460AF0F0FB0028A6DBE068C0032C
:102040002AD56168E06A884200D808462169451AA5
:10205000E069471B1BD02046D4F8188000F016FA20
:1020600008EB05015046C4F818800AF0D5FB00289B
:102070008BDBE06840F40030E060000202D5A0692C
:102080002844A061E1692069C91B45180DE020467C
:1020900000F0FCF9E769F5E725696168D4E906070E
:1020A000491BE56208446560A061E06820F010000B
:1020B00010F4C06FE06002D0204600F0C9FFE06875
:1020C00040F48050C4E90260000205D52069E06256
:1020D00060606FF0010046E7224639462846FFF768
:1020E000F9FE411C0CD02918E16258B1401E206055
:1020F000681C6060E06840F40030E060287832E7F7
:10210000484630E765602046FFF7FFFEF8E72DE917
:10211000F04705460C46C86820F4201040F48000C3
:10212000C860800602D5084600F0D3F9E06841F2A5
:1021300082014FF0FF390140022903D0204600F010
:1021400071F9B5E000F42041B1F5004F0FD1C003A3
:1021500006D56168E06A884200D80846606006E0FB
:102160002069E062606060690AF00CFAA061A06812
:102170000022EEB200280DDAE1688B050AD4C043D4
:10218000A06041F490302260E0606068411C6160B2
:102190000670A5E0E0689046226040F40050E060E0
:1021A000206968BB60690AF001FA012704F124057F
:1021B000A0B1A08910F4407F08D0E069FEF758F87C
:1021C000206118B1E06840F4006016E0E761256125
:1021D000E06820F4407040F480600EE0E069FEF7B3
:1021E00047F800282061F1D0E06840F4006010F466
:1021F000407FE06002D140F48070E0602069606060
:10220000E06825696FF0010AC1051FD56168E06AC1
:10221000884200D80846411B04D02246284600F0D8
:102220000BF9F0BBE068010203D5E562C4E901588F
:1022300054E0691CE1626160E16940F48030491E4C
:10224000C4E9021030462E70BDE8F087010202D5C5
:1022500000F480320AE06068411C61600670E0684A
:102260000A2E40F48030E06006D00022E16A606807
:10227000814203D90B4602E00122F7E70346A78912
:102280005B1B7F0503D4E7699F4200DDE2B1814219
:1022900000D80146E5620F1AC4E90158002B09DD98
:1022A00000E005E022461946284600F0C5F808B1CE
:1022B0004846C9E747B1A069E5626560C01BA061F7
:1022C000E06840F01000E060E068000208D5616856
:1022D000A069E562491B08446560A0615046B3E708
:1022E0003046B1E72DE9F041044616460D464769F0
:1022F000007B80072ED038460AF058F950BB3EB319
:10230000012E02D0022E25D104E0204600F07EFEF0
:1023100005441DE038460AF035F9E168002841F02F
:102320001001E16005DA204600F07CF80120BDE8EC
:10233000F081C9030BD56268E16A914200D8114669
:10234000A26911442269891A814200DD08460544C8
:10235000002D01DA0220EAE7E16A6068E268814262
:1023600006D29103E06203D522F4003141F010025D
:10237000A6690027AE4213DCE16A814201D90B460F
:1023800000E0034603EB060C2369ACEB030CAC4501
:1023900006DD814201D98C4600E084469C4505D18A
:1023A000A760276042F02000A5620DE0AD1BE66942
:1023B000AE1B8142A66000D90846C01A281A2060C8
:1023C0005819606022F0200003490840E0600020B6
:1023D00084F84870ABE70000BFCFD7FF70B5C46882
:1023E000A50713D0650211D4B2F5807F09D0B2F5EC
:1023F000007F06D0B2F5806F08D1012300F12401DF
:1024000006E05D1E6FF07F46B54201D3012070BD2E
:102410000161C361416024F470611143C160002017
:1024200070BD0000C16821F4001141F08001C1605D
:1024300000218160016070472DE9F0478146144614
:102440000E464FF0FF383248D5685769054209D02B
:102450003846A1690AF0E0F9002811DB2C48C04396
:102460000540E5602B463246494638460AF0E8F911
:10247000A16920F00042B21A11440028A16103D0E2
:102480002046FFF7CFFF4046BDE8F08770B5044611
:102490000569C06A6168884200D80846E16821F48D
:1024A0002011E160C90312D5A84208D02246411B81
:1024B0002846FFF7C1FF10B14FF0FF3070BD00207C
:1024C000E562C4E90150E06820F48030E06000205B
:1024D00070BD10B50446C06820F02000E060A16A1D
:1024E000A06988420DD02046FFF7D0FFE06820F4B5
:1024F000405040F01000E060A06AA0612069E062F6
:10250000606044F24001E0688843E06010BD000074
:102510001000020010B542485421FEF7F9FA414874
:102520005421FEF7F5FA40485421FEF7F1FA3F49ED
:102530003B483C4A3F4B08603D490A603A491960B4
:10254000531C0365481C1065012008653B48344A4C
:1025500039A17844FEF76AF920B9384878440A3836
:1025600000F0D5FD37482F4A35A17844FEF75EF9D3
:1025700020B9344878440A3800F0C9FD32482A4A64
:102580002FA17844FEF752F920B92F4878440A3831
:1025900000F0BDFD40232248DC0000212246FFF769
:1025A0001DFF20B125487844543800F0B0FD1D4887
:1025B000224640230021FFF711FF20B12148784433
:1025C000543800F0A4FD1848224610230021FFF7DC
:1025D00005FF002806D01C487844BDE81040563856
:1025E00000F095BD10BD104870B5006D20F00104DD
:1025F0000B48FEF79BF90B48FEF798F90A48FEF7DF
:1026000095F909E0206D20F001052046FEF78EF9CE
:102610002046FDF775FE2C46002CF3D170BD00005E
:10262000C81000101C11001070110010A001001043
:10263000A4010010A8010010720000002623010070
:1026400077000000152301000523010010B500F0FC
:102650006DFDBDE8104000F055BD00002DE9F041D2
:1026600015460E46040002D12C6804B90BA420467E
:1026700000F084FD0444207870B127463146384686
:1026800000F06CFD0444207810B1002004F8010B28
:1026900038462C60BDE8F0810027F9E70000000013
:1026A00000487047AC12001000487047C01200107C
:1026B000034640688C46002818BF88423CBF03464A
:1026C0004068F8D318681844884207D00CF103001A
:1026D00020F00700001D411A521A0146081D0A6029
:1026E000FDF70EBE30B5B0F10A024FEA900E71F15F
:1026F00000034EEA817EB0EB0E0061EB91014FEAE0
:10270000101E4EEA017E10EB0E0041EB11114FEA54
:10271000102E4EEA016E10EB0E0041EB11214FEA34
:10272000104E4EEA014E10EB0E0041EB11414018E5
:1027300041F100014FEAD00040EA41704FEAD10177
:1027400010EB80054FEA810444EA907444EB0104E5
:102750006D1944EB0404521BA3414FF0000348BF22
:102760000A3200D530BD401C41F1000130BD10B52A
:10277000044600F03FFD0068005D00F0010010BD60
:102780002DE9F04F04460D46D21D22F0070089B016
:10279000D0E900974846394609F048FC0246F80F50
:1027A00001D02D2307E02068810701D52B2302E00B
:1027B000202101EAC0038DF820300BB1012000E098
:1027C0000020032A824601D0072A04DB294620463E
:1027D00000F054F93FE12078800601D40D2500E097
:1027E000E569C7F30A560D2D49DA00214FEA175B58
:1027F00008464FF00000002F00F4400007DA00EB1D
:1028000080004FF4400100EBD07001EA60008115B8
:10281000012901DD4FF0FF3100224FEA850CBCF1A8
:10282000180F06D31346ACF118004FF08052C24087
:1028300003E04FF4801323FA0CF30CF10C0CBCF101
:10284000200F04D3ACF1200C09FA0CF001E007FAD8
:102850000CF000294FF0004801DD18B90FE00ED14F
:1028600040450CD319EB02095F4121B9404502D123
:102870009F4329EA0209BBEB175F00D0761C208832
:10288000000502D57B48784402E07A48784419383C
:1028900008AA302302F80A30037C0AF10101002E55
:1028A0000AF1020A53546A4602DC4FF0300101E09B
:1028B0004FF031014FF001088DF8001002D0A6F260
:1028C000FF3603E059EA470100D06B4E002D02DCD1
:1028D0002178090704D54FF002082E218DF8011048
:1028E000C44600210BE0C7F303433F01C35C491C0E
:1028F0006D1E02F80830052908F1010801DA002DE3
:10290000F1DC00210CE000EB1973491C1B786D1EF3
:10291000082902F808304FEA091908F1010801DA1C
:10292000002DF0DC21688B0602D516E0A8F1010825
:10293000E04505DD02EB080313F8013C302BF5D030
:10294000B8F1000F09DD02EB080313F8013C2E2B50
:1029500003D1090701D4A8F10108002D05DD3E21AE
:1029600002F808106D1E08F10108407C002E02F8E4
:10297000080008F1010804DA2D20764202F8080068
:1029800002E02B2002F808000A214FF47A708642F8
:1029900008F101080BDB96FBF0F3303302F8083046
:1029A00096FBF0F308F1010800FB136601E0642ECA
:1029B0000CDB642096FBF0F3303302F8083096FB12
:1029C000F0F308F1010800FB136601E00A2E06DBB4
:1029D00096FBF1F0303002F8080008F1010896FB90
:1029E000F1F001FB1060303002F80800A16908F135
:1029F000010808EB050202EB0A00081AA061207822
:102A0000C00602D42046FEF75CF9216A08AE01EB4D
:102A10000A00206204E0D4E9012116F8010B904776
:102A2000BAF1010AF7D22078C00602D52046FEF797
:102A300048F96E4609E016F8010B3E280FD0D4E99C
:102A400001219047206A401C2062B8F10108F2D2AF
:102A50002046FEF74CF909B00320BDE8F08F206A4C
:102A60002844206203E0D4E90121302090476D1E04
:102A7000EBD3F8E78D22010002FCFFFF2DE9F041C6
:102A80001F46044603260168072A01F4006004DBA0
:102A900008B116A505E016A503E008B115A500E0EC
:102AA00015A521F010002060A069C01EA0610FB123
:102AB000401EA0612046FEF704F94FB1D4E9012180
:102AC00038469047206A401C2062C01C206206E005
:102AD000206AFAE7D4E9012115F8010B9047761E28
:102AE000F8D22046FEF703F9BDE8F0814E414E00D2
:102AF0006E616E00494E4600696E660010B543690E
:102B000013B1AFF3008001E0FEF714F9012010BD0E
:102B1000127800F124010A7000224A700122EDE7C8
:102B200011684FF0FF32E9E710B5436913B1AFF315
:102B3000008001E0FEF7D2FB012010BD128800F1F9
:102B4000240182840022C2840122EDE711684FF043
:102B5000FF32E9E72DE9F34F4FF0000A0C465646E5
:102B60008DB001200C9001F10C000B9062690B9864
:102B700001219047051E2DD0252D2CD0216A884794
:102B8000C0B162690B9801219047216A88470028EB
:102B9000F7D16269411E0B98904700E0761CA1694D
:102BA0000D988847216A88470028F7D1E1690D9878
:102BB0008847DBE7A1690D988847A842074601D1FD
:102BC000761CD3E7E1690D9888477F1C02D1BAF1E2
:102BD000000F6FD06BE162690B9800273D463946C4
:102BE00090472A2804D162690B980121904701255A
:102BF000DFF8D08262690B9801219047A0F1300183
:102C00000A290AD24745E5DC07EB870100EB4107BB
:102C1000303FDFD445F01005ECE7E90601D46FF052
:102C200000476C280AD04C2814D0682815D06A2890
:102C30000DD074281CD07A281AD01DE062690B9838
:102C4000012190476C2802D045F0040514E045F0BE
:102C500002050DE045F020050AE062690B980121AC
:102C60009047682802D045F0080505E045F4006566
:102C700062690B9801219047C4E9015765283DD04E
:102C800019DC58287AD00CDC452837D004DC2528FC
:102C900026D041289ED131E046282FD0472899D10F
:102CA0002CE05B2877D0612828D063287CD064286A
:102CB00023D15AE0F6E06F2848D008DC66281DD002
:102CC00067281BD0692821D06E2816D127E07028EC
:102CD00045D0732868D0752847D078280DD14DE0AD
:102CE000A1690D988847252805463FF469AFE16939
:102CF0000D9888476D1C3FF46AAFD8E00D992346C4
:102D00006A466FF0010011F0D4FCC5E045F04000C8
:102D100023464FF000026060A80736D43EE0E80783
:102D20007FF447AF2068011D21600068290501D5A7
:102D300006701BE7290701D5068017E7A90703D509
:102D4000F117C0E9006111E706600FE745F04000A8
:102D500023464FF008026060A80716D41EE040F634
:102D60000E0125EA0100606016E045F040002346B0
:102D70004FF00A026060A80707D40FE045F040005A
:102D80006060A80708D5234610220D996FF0010056
:102D9000FEF786FB80E007E0102223460D996FF0D6
:102DA0000100FDF76BFC77E04FF0000963284F4608
:102DB000C8464B46CB4602D05B2806D038E0E80632
:102DC00001D40120A060012732E06269D4F80CB080
:102DD0000B98012190475E2807D14FF00109494621
:102DE0006269D4F80CB00B989047216939B9002179
:102DF0000A4603AB43F82120491C0829FADBD8B363
:102E0000216949B308F1010862690B9801219047D3
:102E10005D28F4D1B9F1000F09D0002003A951F8C1
:102E20002020D24341F82020401C0828F7DB03ABC8
:102E30002069002820794FEA40701ED05B46224668
:102E4000CDF80080CDE901970D9900286FF00100C1
:102E500020DAFEF7D3FF1FE0C11703AA00EBD16110
:102E60004B1121F01F0102EB8302411A136801206C
:102E7000884003431360C7E719E00D9922460028F4
:102E80006FF00100009702DAFEF7BAFE04E0FEF7E9
:102E9000B2FB01E0FEF73EFF00280ADA401C06D133
:102EA0000C9820B14FF0FF300FB0BDE8F08F5046C6
:102EB000FAE7E90701D10AF1010A064400200C9063
:102EC00054E60000CCCCCC0C10B508E030F8024B36
:102ED0009C4204D10AB1002010BD012010BD491E42
:102EE000F4D2104610BD00002DE9F0478146164689
:102EF0008AB0334878440DC88DE80D0030487844D6
:102F0000801C03AC0DC884E80D0041F69B300844DA
:102F1000372190FBF1F290FBF1F5A5F1800501FB63
:102F200012041B3C02D56442012000E00020DFF8BF
:102F300090A080460027FA44AAF1BE0A0DE0E007FF
:102F400009D03246684607EB47010AEB810100F0E1
:102F5000EEFE8DE8070064107F1C002CEFD1184FA7
:102F60007F44AC3F18E0E80714D007EB04100DF1E4
:102F7000180A90E80E008AE80E00C068F04201D1FD
:102F800098190890324606A903A800F0D0FE03ABBA
:102F900083E807006D10641C002DE4D132466946B9
:102FA000B8F1000F03A802D000F099FE01E000F094
:102FB000BEFEC9E90001C9F808200AB0BDE8F087E3
:102FC000B01C0100704710B54FF0FF34C1688A0291
:102FD0000FD5036B42689A420BD1014690F8252029
:102FE000104600F045FB401C01D1204610BD0020DA
:102FF00010BD11F0C00FF8D1026941689142F4D9B7
:103000000268491E521CC0E90021F0E710B50146D4
:10301000C268900703D0900607D5886A0AE0FFF7D8
:1030200043FB01210160881E10BD8B69486818446C
:103030000B69C01A91F848301BB191F84910401A39
:1030400010BD1103FCD50028FADD401E10BD0000A4
:1030500070B5054640F202260A4C0FE094F8500085
:10306000C00708D0AC4206D0E06836EA000002D1C2
:103070002046FDF7A9FB206D20F00104002CEDD1C6
:1030800070BD0000C810001070B516460C4605460D
:1030900000F0B0F8036893F80101012804D0185D2E
:1030A00068B101202C8070BDD3F80301324621465F
:1030B00003F2031303442846BDE8704018474FF05D
:1030C000FF3070BD70B516460C46054600F092F80C
:1030D000036893F80101012806D0FF2C0FD8185D72
:1030E00068B101202C7070BDD3F80701324621462B
:1030F00003F2071303442846BDE8704018474FF019
:10310000FF3070BD002801D000F06EB8704710B5D8
:1031100000F0ECFABDE81040FFF7F4BF10B500F086
:10312000FFFABDE81040FFF7EDBF000010B5002129
:1031300002A000F0C1FA012010BD00005349475021
:1031400056464E3A205075726520766972747561E4
:103150006C20666E2063616C6C65640030B503465C
:103160001D781DB10A4603E0AC4201D1181A30BDEA
:1031700012F8014B002CF7D15B1CF1E730B5034688
:103180001D783DB10A4612F8014B1CB1AC42FAD190
:103190005B1CF5E7181A30BD124B694600F58052EA
:1031A0008A421A6001D8114670471960704730B5DD
:1031B0000C4D6B46A3F580532C6822449A420FD8DD
:1031C0009B1A02F5805003EBD37302EB6303984222
:1031D00000D91846C01D20F007020C60101B2A60A1
:1031E00030BD0000B001001001491820ABBEFEE761
:1031F0002600020010B5FFF753FA001D10BD00BFF6
:10320000C900010010B5FFF74FFA006810BD10B5F6
:103210000446FFF749FA046010BD00002DE9FF4F96
:103220001F464FF03C0987B04FF00042DDE9141013
:1032300001F10108DDF858A002EA40500390002097
:1032400005908346054604460490B969461E0898D1
:103250008847AAF1010A0290BAF1000F3BDD0298FB
:103260002E2815D01021FEF70DF900282EDB4FF087
:10327000010B0599014317D0B9F1000F0BDB4A464A
:10328000C11700F07DFA05430C43A9F1040905E0DC
:10329000012004900BE008B145F0010501200590E4
:1032A000049820B9361D02E0049800B1361FB969B0
:1032B000089808F101088847BBF1000FAAF1010A3C
:1032C0000290C9D00999C1F80080C5E7029870281A
:1032D00008D0502806D0F96908988847BBF1000F3C
:1032E00014D04FE0002002900120BBF1000F0490A9
:1032F00009D0B969089808F101088847AAF10109BD
:10330000B9F1000F07DCF969089888476FF00100F0
:103310000BB0BDE8F08F2B2804D02D280CD14FF036
:10332000FF300490B969089808F101088847A9F1AD
:103330000109B9F1000FE6DD411CE4D00A21FEF7D6
:10334000A1F80028DFDB029908F1010801EB8101F7
:1033500000EB41000290B969089888470A21FEF7FE
:1033600091F8099AA9F10109B9F1000FC2F800809A
:1033700001DD0028E7DAF96908988847049902987E
:1033800000FB016655EA040004D004F04041090046
:1033900002D006E0039898E0A40044EA9574AD00DA
:1033A000B61E04F00041080002D16D196441761E7A
:1033B000159810F0240F03D04FF00B095C4803E080
:1033C0004FF028096FF07D008246564507DAAAEBD8
:1033D00006018944B9F1410F01DD4FF04109012097
:1033E0000021A9F1010200F0CBF9024628400B466A
:1033F0002140084301D0012100E00021501E02912C
:1034000043F1FF3128402140084301D0012000E072
:1034100000200299834651EA0B014FD00021084653
:103420004FF00000039900F4400039B100EB800038
:103430004FF4400100EBD07001EA600080150128D4
:1034400002DD4FF0FF3000E013D0401C36D0029870
:1034500060B3BBF1000F0CD14A460120002100F0FF
:103460008FF928402140084301D0012000E00020CE
:10347000E0B101204A46002100F082F903464019DC
:103480000A4661412D1A8C4111D3B9F1400F09DD73
:10349000159810F0240F02D0AAF1340603E0AAF127
:1034A000170600E0761C00254FF0004406E05B1E86
:1034B00042F1FF3220EA030521EA0204CAF10100C9
:1034C000B04206DA1B49039808430190002000909F
:1034D0000EE0039AC4F3D321E80A0A43164940EAEE
:1034E00044500A433146CDE90002684609F014F819
:1034F000159810F0240F0BD01598C00715D1386817
:10350000DDE90012031D3B600068C0E900120CE019
:1035100002A8694608F0DEFD1598C00705D1386895
:10352000029A011D3960006802604046F0E6000022
:1035300002FCFFFF0000F07F0000F03F2DE9FF4F8D
:1035400092461D4685B04FF00041DDE9124BDDE9A2
:1035500014727F1E01EA4B50414940F0FF4940EA96
:103560000108002122F020004928049102D04E28B1
:1035700028D04CE03BA0012607C88DE80700A969C8
:103580000698641C88477F1E014606D41DF8060075
:1035900018B121F0200181420BD0E96906988847D3
:1035A000032E34D0082E32D06FF0010009B0BDE8F0
:1035B000F08F761C032E01D0082EE0D1601CCAF8D3
:1035C0000000DCE7A9690698641C88477F1E2AD49E
:1035D00020F02000412826D1A9690698641C88475C
:1035E0007F1E20D420F020004E281CD1A969069807
:1035F000641C88477F1E48F4002849F48009CAF8F3
:10360000004001D4282806D0E969069888475FEA77
:10361000CB7012D022E0A9690698641C88477F1EEF
:1036200001D4002803DAE96906988847BCE729280D
:10363000F1D1641CCAF80040E9E71BF0240F07D061
:1036400028680499031D2B600068C0E9001805E094
:103650002868021D2A600068C0F800902046A5E78F
:103660000000F07F494E46494E4954590000000081
:10367000CA68431C0FD00D4B1A420CD1D3070AD095
:1036800081F825004B680B6300238B6012F0C06F3C
:103690000B6003D004E04FF0FF30704742F000723F
:1036A000034B1A40034B1A43CA607047802008003E
:1036B000BFFFDFFF0010480070B505460C460A202A
:1036C00000E06D1C00F054F835B128780028F8D1DE
:1036D00002E0641C00F04CF814B120780028F8D106
:1036E000BDE870400A2000F043B8000010B5014664
:1036F00002A0FFF7E1FF012010BD0000534947522F
:10370000545245443A2052656469726563743A20A4
:1037100063616E2774206F70656E3A2000000000B0
:1037200010B5012805D0002103A0FFF7C5FF012037
:1037300010BD09A1F8E7000053494752544D454DCB
:103740003A204F7574206F662068656170206D6542
:103750006D6F7279000000003A2048656170206D3D
:10376000656D6F727920636F727275707465640035
:1037700008B569468DF800000320ABBE08BD704750
:10378000B2F120030AD5C2F1200301FA02F120FAB6
:1037900003F300FA02F041EA0301704700FA03F173
:1037A0004FF0000070475FEA400C08BF91F0000F37
:1037B0004FEA8C234FEAC12243EA51514FEA1C5091
:1037C00018BF00F5F0404FEA300018BF41F000414B
:1037D0005FEA6C5C00F02980BCF1FF3F08BF40F05D
:1037E00080407047130C06BF12044FF0100C4FF0CE
:1037F000000C130E04BF12020CF1080C130F04BFCF
:1038000012010CF1040C930F04BF92000CF1020C96
:10381000D30F04BF52000CF1010C11464FF000020F
:10382000A0F11F00A0EB0C00704711F0004F08BF83
:10383000704731F000413FF4D5AF0B0C06BF0904CF
:103840004FF0100C4FF0000C0B0E04BF09020CF1EE
:10385000080C0B0F04BF09010CF1040C8B0F04BF03
:1038600089000CF1020CCB0F04BF49000CF1010CD4
:10387000CCF12003A0EB0C0022FA03F302FA0CF2C5
:1038800041EA030100F10100704720F07F4C80EA1B
:10389000030023F07F47ACEB070303F57C5300F0F4
:1038A000004003F1FF032DE980494FEA154B09B4AD
:1038B0004FEA144325EA0B4E24EA03480FF204268C
:1038C00006EB132749083E785FEA320203FB0667DE
:1038D000C7F5000707FB06F64FEA54374FEAD6460E
:1038E00006F1020607FB066CCCF1005C4FEA1C47B0
:1038F0002CEA074C07FB06F40CFB06F504EB154617
:103900004FEA961634BF00204FF000404FEAD137FF
:1039100006FB07FC4FEA1C4C0CFB0BF7D21B03FB0E
:103920000CF761EB07010CFB0EF7B0EB074072EBF5
:1039300017420CFB08F734BFA2EB0742B2EB074279
:1039400061EB17414FEA0C444FEA910706FB07FC75
:103950004FEA1C4C0CFB0BF7B0EBC74072EB573235
:1039600003FB0CF734BFA2EBC742B2EBC74261EBDB
:1039700057310CFB0EF7B0EBC70072EB57720CFB24
:1039800008F734BFA2EBC702B2EBC70261EB577175
:10399000039F4FEA816141EA921104EBCC044FEAA4
:1039A000D1374FEA826206FB07FC42EA90124FEAE7
:1039B00080604FEA1C4C0CFB0BF7D21B03FB0CF78F
:1039C00061EB07010CFB0EF7B0EB074072EB1742FF
:1039D0000CFB08F734BFA2EB0742B2EB074261EBE6
:1039E00017414FEA8C554FEA910704EB9C2406FBE4
:1039F00007FC4FEA1C4C0CFB0BF7B0EBC74072EB1B
:103A0000573203FB0CF734BFA2EBC742B2EBC742FD
:103A100061EB57310CFB0EF7B0EBC70072EB57723E
:103A20000CFB08F734BFA2EBC702B2EBC70261EB95
:103A3000577115EB4C254FEA816141EA92114FEA2B
:103A400082624FEAD13742EA901206FB07FC44F14A
:103A500000044FEA80604FEA1C4C0CFB0BF7D21BB2
:103A600003FB0CF761EB07010CFB0EF7B0EB074013
:103A700072EB17420CFB08F734BFA2EB0742B2EB24
:103A8000074261EB174115EB1C154FEA813141EA02
:103A900092414FEA823242EA90424FEA80304FEA46
:103AA0000C7644F1000448EA03434EEA0B484FF019
:103AB000000EB2EB080C71EB030724BF62463946D7
:103AC0004EEB0E0E4FF0000B0018524149414BEBEC
:103AD0000B0BB2EB080C71EB03077BF1000B24BF5F
:103AE000624639464EEB0E0E4FF0000B0018524165
:103AF00049414BEB0B0BB2EB080C71EB03077BF16D
:103B0000000B24BF624639464EEB0E0E51EA020707
:103B100018BF46F0010616EB0E7655F1000254F17F
:103B2000000103D5BDE88901BDE80088BDE8890131
:103B3000BDE80048B619524141EB0101A3F1010370
:103B4000704780807F7E7D7C7B7A7978777676750A
:103B50007473727171706F6E6E6D6C6C6B6A6A6982
:103B60006868676666656464636362616160605F1C
:103B70005F5E5E5D5D5C5C5B5B5A5A595958585795
:103B800057565655555554545353525252515150FD
:103B900050504F4F4F4E4E4D4D4D4C4C4C4B4B4B50
:103BA0004A4A4A4949494848484747474746464696
:103BB00045454544444444434343434242424241D1
:103BC0004141000046EA0646A3F570534FEA164607
:103BD00046EA42564FEAD22242EA415210B54FEA33
:103BE000D121A3F1010300F017F820F0004000F10B
:103BF000010C00F0004701EB00501146BCF5006FCE
:103C000040EA070000D210BD02484FF0000140EA30
:103C1000070010BD0000F07F002B26D4770021D0D4
:103C20001CB54FEA370703B44FF010004FF01001F6
:103C30004FF000000FBCBDE810400BF1010BBBF1D1
:103C4000010F08BF5FEA170722BF12F1010211F14D
:103C500001014FF0004143F1000300F0004043EA4E
:103C600000007047F9D35708DAE746EA064613F131
:103C7000400F4FEA16461FDD13F1200FDFBF16433A
:103C80000A46002120335B42C8D0C3F1200746EA30
:103C9000064602FA07F74FEA164646EA0706C3F158
:103CA000200722FA03F201FA07F721FA03F14FF095
:103CB000000342EA0702B1E746EA020646EA064680
:103CC0004FEA164646EA0106BCBF46EA0646360CEF
:103CD0004FF000034FF000024FF000019EE72DE986
:103CE000C048934630B491E8380007C831EA400C28
:103CF00048BF34EA430C03D5FFF7C7FDFFF78CFF3D
:103D0000F0BCBDE800882DE9C048934630B491E886
:103D1000380007C831EA400C48BF34EA430C03D5E9
:103D2000FFF7B3FDFFF74EFFF0BCBDE800882DE9BB
:103D3000C048934630B491E8380007C810F0804F6F
:103D400008BF13F0804F03D100F019F8FFF764FFAC
:103D5000F0BCBDE800882DE9C048934630B491E836
:103D6000380007C810F0804F08BF13F0804F03D110
:103D700000F005F8FFF726FFF0BCBDE8008820F052
:103D80007F4780EA030023F07F4C07EB0C03A3F589
:103D90007C5300F00040A3F1FE0392F0000F00F00E
:103DA000B38095F0000F00F077802DE901494FEACC
:103DB00011404FEA144621EA004800FB06FC24EAC1
:103DC000064708FB06F607FB08F800FB07F718EBA9
:103DD00006484CEB164C4FEA124B18EB07484FEADB
:103DE00015464CEB174022EA0B4E0BFB06FC25EA6E
:103DF00006470EFB06F607FB0EFE0BFB07F71EEB56
:103E0000064E4CEB164C4FF000061EEB074E4CEBEB
:103E1000174B18EB0B0840F1000018EB0E0B58EB9A
:103E2000000840F100008F1A4FF000013CBFC94369
:103E3000661B14BFB5EB040C00213CBFC943F61B45
:103E40004FEA17444EEA8E0E27EA04454FEA1C4714
:103E500004FB07622CEA074C05FB07F70CFB05F691
:103E600004FB0CFC16EB074642EB174216EB0C4624
:103E700042EB1C421BEB060658EB0202414146EAAC
:103E80009E0601D5BDE80189B619524141EB0101F9
:103E9000A3F10103BDE801894FEA14454FEA114738
:103EA00024EA054621EA074C05FB07F406FB07F761
:103EB0000CFB06F105FB0CFC11EB074144EB17442E
:103EC0004FEA124711EB0C4144EB1C4422EA074C29
:103ED00005FB07F206FB07F70CFB06F605FB0CFCDF
:103EE00016EB074642EB174216EB0C4642EB1C451D
:103EF0006A1854F1000148BF7047B619524141EBAE
:103F00000101A3F10103704795F0000F37D04FEA8C
:103F100011424FEA144721EA024624EA074C02FB09
:103F200007F106FB07F70CFB06F402FB0CFC14EB95
:103F3000074441EB17414FEA154714EB0C4441EBA2
:103F40001C4125EA074C02FB07F506FB07F70CFBB3
:103F500006F602FB0CFC16EB074645EB174516EB85
:103F60000C4645EB1C42121951F1000148BF704745
:103F7000B619524141EB0101A3F1010370474FEA29
:103F800014454FEA114724EA054621EA074C05FB90
:103F900007F106FB07F70CFB06F24FF0000605FBE6
:103FA0000CFC12EB074241EB174112EB0C4251EBB8
:103FB0001C4148BF7047921841EB0101A3F1010376
:103FC000704710B50EF0B8F9BDE8104009F092B88E
:103FD0000021C1607047000025482021C0F8A011D1
:103FE000D0F8A01111F0200F05D000BFD0F8A0111B
:103FF00011F0400FFAD00221C0F804110022C0F8DD
:10400000A821C0F8AC210121C0F80C110B23C0F885
:104010008430AA23C0F88C304FF0550CC0F88CC007
:10402000C0F88010C0F88C30C0F88CC0D0F8881070
:1040300011F0806FFAD00321C0F88010C0F88C30E6
:10404000C0F88CC0D0F8881011F0407FFAD005215C
:10405000C0F808110749C0F8C410C0F8C8210168A9
:1040600043F23A0221F470411143016070470000AD
:1040700000C00F40DE8728042DE9F04F95B0FD48C1
:1040800006F0ECF8FC4806F0E9F8FC4806F0E6F823
:10409000FB4806F0E3F8FB4806F0E0F8FA4806F0C3
:1040A000DDF803F001FE032005F074F8F74CF34E41
:1040B000626BA6F5CF65012A40F02383606A20B1C8
:1040C000F3A105F1300006F0D8FF642004F014FAE3
:1040D000A06A0FF0B7F83C2004F00EFAA06A0FF0C7
:1040E000B1F8606A002845D0E54DD5F880000FF0A2
:1040F000DBFECDE90801A5F5B870D0F880000FF01F
:10410000D3FE8346A5F5B870079105F083FF0FF045
:10411000CBFE814605F5B8708A46006A0FF0C4FEF2
:1041200007468846286A0FF0BFFE0546D3480E466C
:10413000006A0FF0B9FE0246DDE90803CDE90C0381
:10414000079BCDE90AB32069CDF81890CDE907A007
:10415000606B04908DE8E001DA4D0B46D84905F11B
:10416000300006F08AFF00F037FDD7A105F13000DE
:1041700006F083FF606B012804BF2069002804D18A
:10418000BE48016AD1488142A5D3C048406A002890
:104190005FD0BC4CD4F880000FF086FE8246A4F5B8
:1041A000B8708B46D0F880000FF07EFE8046A4F5F4
:1041B00038708946D0F880000FF076FE06460F462C
:1041C000204605F027FF0FF06FFE0A900D46A4F57C
:1041D000B87005F01FFF0FF067FECDE90710A4F5DA
:1041E000387005F017FF0FF05FFE06910490206A0B
:1041F0000FF05AFECDE90201A4F5B870006A0FF085
:1042000053FE04469D480191006A0FF04DFE0B4697
:104210000EA9DFF878C281E8C00FDCF81010CDE9F4
:104220000B5107990991069A0499CDE90612DCF819
:1042300034100094A34C02460491A54904F13000C7
:1042400006F01BFF00F0C8FC9FA104F1300006F04F
:1042500014FF8E4C606B002804BF2169002905D132
:10426000864D9A492A6A8A42C0F03F82216909B183
:1042700001280DD0814D95492A6A8A4240F2F18188
:10428000012808BFDFF83CA240F0EB8100F0B6B98E
:10429000606A18B18FA19E4806F0EFFEC82004F0B6
:1042A000D1F99C480EF0CEFF02F02AFE03F01CFA72
:1042B0004FF07C500EF0C6FF032004F06BFF04208B
:1042C00004F068FF052004F065FF03F0EDFC606A70
:1042D00098B17C4D90A105F1300006F0CEFE00F0C3
:1042E0007BFC9BA105F1300006F0C7FE01F0DEFE6D
:1042F00075A105F1300006F0C0FE604EA6F5CF6551
:10430000782004F09FF9A06A0EF09CFF606A28B341
:10431000D6F880000FF0C8FD81468A46574805F060
:1043200079FE0FF0C1FD07468846306A0FF0BCFDEC
:10433000CDE9069A024620690B460297CDE9038033
:10434000606B0090864905F1300006F096FE00F0A3
:1043500043FC5DA105F1300006F08FFE20690028C6
:1043600004BF606B0128CBD0606A30B3D6F8800000
:104370000FF09AFD81468A46404805F04BFE0FF04B
:1043800093FD80460F46306A0FF08EFDCDE9069A08
:1043900002462069CDF80880CDE90370606B0B46BA
:1043A00000906F4905F1300006F067FE00F014FC44
:1043B00045A105F1300006F060FE2069B0B1606AE9
:1043C000002854D067A105F1300006F056FE00F039
:1043D00003FC6FA105F1300006F04FFE01F066FE10
:1043E00039A105F1300006F048FEFEE0606B0028C0
:1043F0003FD13C2004F026F9A06A0EF023FF606A4A
:1044000028B3D6F880000FF04FFD81468A461B483E
:1044100005F000FE0FF048FD07468846306A0FF0B1
:1044200043FDCDE9069A024620690B460297CDE985
:104430000380606B00904A4905F1300006F01DFED4
:1044400000F0CAFB20A105F1300006F016FE20693D
:10445000616B0843CDD0606A50B1D6F880000FF090
:1044600023FD81468A46054805F0D4FD96E0BCE070
:10447000B3E0BFE0AC0500101C0700108C08001072
:10448000FC0900106C0B0010DC0C0010C8000010C0
:104490000D0A0D0A4C696D69742033203D20256496
:1044A0002C206D6F766520656C626F7720616E647D
:1044B0002077726973742075700D0A0D0A00000070
:1044C000845C0100140200100D0A000000D004C634
:1044D000E45C0100436F6C6C6973696F6E20446526
:1044E000746563746564206F6E20456C626F77201D
:1044F000686F6D652E20204D6F76696E6720646F42
:10450000776E2032303020737465707300000000C5
:10451000440200108FC2F53C436F6C6C6973696F85
:104520006E2073746F707065642074686520757098
:1045300077617264206D6F76656D656E742E204DA7
:104540006F766520646F776E2E202020200000009B
:104550000D0A20204D41582049203D200000000038
:10456000405C01000D0A436F6C6C6973696F6E20CB
:1045700064657465637465642C2072657475726E0D
:10458000696E67206572726F72202D3120200000E5
:104590000D0A2020204D4158203D20000FF084FCC2
:1045A00080460F46306A0FF07FFCCDE9069A02463E
:1045B0002069CDF80880CDE90370606B0B46009050
:1045C0009C4905F1300006F058FD00F005FBAFF204
:1045D000081105F1300006F050FD2069002800F0B8
:1045E0001C81606A00287FF4EDAE15B04FF0FF30FB
:1045F000BDE8F08F15B00020BDE8F08F782004F002
:1046000021F8A06A0EF01EFE606A20B3D5F8800083
:104610000FF04AFC80468946874805F0FBFC0FF006
:1046200043FC06460F46286A0FF03EFCCDE906899A
:1046300022690296CDE90372626B009202460B4634
:104640007C490AF1300006F018FDAFF284110AF13E
:10465000300006F012FD2069002804BF606B0128BD
:10466000CCD0606B002808BF744E08D074A17D4880
:1046700006F003FD15B06FF00100BDE8F08F3220A9
:1046800003F0E0FFA06A0EF0DDFD606A18B3D5F814
:1046900080000FF009FC81468A46674805F0BAFCA5
:1046A0000FF002FC07468846286A0FF0FDFBCDE9B3
:1046B000069A024620690B460297CDE90380606B9B
:1046C00000905C4906F1300006F0D7FC64A106F1C9
:1046D000300006F0D2FC2169606B0843CFD0606BDC
:1046E000012804BF2069002884D1032004F052FD72
:1046F000042004F04FFD052004F04CFD0020E8628A
:1047000078E70A2003F09EFFA06A0EF09BFD606A26
:1047100028B3D6F880000FF0C7FB81468A4646488A
:1047200005F078FC0FF0C0FB07468846306A0FF0B2
:10473000BBFBCDE9069A22690297CDE90382626B41
:10474000009202460B463B4905F1300006F095FC0D
:1047500000F042FA42A105F1300006F08EFC20691B
:10476000616B0843CDD02069B8B33FA105F130009B
:1047700006F083FCD6F880000FF096FB07468946CA
:104780002D4805F047FC0FF08FFB80468A46306AC3
:104790000FF08AFBCDE90679024620690B46CDF879
:1047A0000880CDE903A0606B0090224905F130003C
:1047B00006F063FC032004F0EDFC042004F0EAFCA6
:1047C000052004F0E7FC2EA105F1300006F055FCB1
:1047D00015B06FF00200BDE8F08FFFE701291CD093
:1047E00000297FF407AF2FA105F1300006F045FC4A
:1047F000032004F0CFFC042004F0CCFC052004F0DE
:10480000C9FC0020F0620EA105F1300006F035FC75
:1048100015B06FF00300BDE8F08F032004F0BAFC80
:10482000042004F0B7FC052004F0B4FC0020F06282
:10483000E0E60000405C01008C080010140200104B
:1048400050726F626C656D207769746820686F6D57
:10485000652121210D0A2072657475726E202D323A
:104860000D0A000044020010436F6C6C6973696F9D
:104870006E20646574656374656421210D0A00000F
:1048800050726F626C656D207769746820686F6D17
:10489000652121210D0A2072657475726E202D33F9
:1048A0000D0A000057544621210D0A0010B584B0AE
:1048B00005200EF0D9FC184C2068B0F1FF3F04D160
:1048C0002C22164916A00DF027FC6069006861686B
:1048D000084018BF01201849184A0028C8626946D4
:1048E000AFF2370000901648039208D006F044F962
:1048F00003996846002904BF04B010BD07E006F024
:1049000073F903996846002904BF04B010BD896893
:10491000884704B010BD00001C030010645D010056
:104920006F626A2D3E70696E20213D202850696EAD
:104930004E616D65294E4300C8000010CC4F010048
:10494000AC03001010B584B005200EF08DFC184C9F
:104950002068B0F1FF3F04D12C22164916480DF013
:10496000DBFB606900686168084018BF01201349DB
:10497000134A002808636946AFF2370000901148D7
:10498000039208D006F0F8F803996846002904BF9E
:1049900004B010BD07E006F027F903996846002926
:1049A00004BF04B010BD8968884704B010BD000082
:1049B00034030010645D010020490000C8000010AD
:1049C000CC4F0100F403001010B584B005200EF0A8
:1049D0004BFC184C2068B0F1FF3F04D12C22164943
:1049E00016480DF099FB606900686168084018BFBF
:1049F00001201349134A002848636946AFF2370083
:104A000000901148039208D006F0B6F80399684662
:104A1000002904BF04B010BD07E006F0E5F80399D3
:104A20006846002904BF04B010BD8968884704B0F7
:104A300010BD00004C030010645D0100204900001F
:104A4000C8000010CC4F01003C04001010B584B029
:104A500005200EF009FC184C2068B0F1FF3F04D18E
:104A60002C22164916480DF057FB606900686168F2
:104A7000084018BF01201349134A0028886369467B
:104A8000AFF2370000901148039208D006F074F896
:104A900003996846002904BF04B010BD07E006F082
:104AA000A3F803996846002904BF04B010BD8968C3
:104AB000884704B010BD000064030010645D01006D
:104AC00020490000C8000010CC4F010084040010F1
:104AD00010B584B005200EF0C7FB184C2068B0F16B
:104AE000FF3F04D12C22164916480DF015FB6069D2
:104AF00000686168084018BF01201349134A002864
:104B0000C8636946AFF2370000901148039208D09D
:104B100006F032F803996846002904BF04B010BDBE
:104B200007E006F061F803996846002904BF04B065
:104B300010BD8968884704B010BD00007C030010D8
:104B4000645D010020490000C8000010CC4F010046
:104B5000CC04001010B584B005200EF085FB184C75
:104B60002068B0F1FF3F04D12C22164916480DF001
:104B7000D3FA606900686168084018BF01201349D2
:104B8000134A002808646946AFF2370000901148C4
:104B9000039208D005F0F0FF03996846002904BF8E
:104BA00004B010BD07E006F01FF80399684600291D
:104BB00004BF04B010BD8968884704B010BD000070
:104BC00094030010645D010020490000C80000103B
:104BD000CC4F0100140500102DE9F04F19488BB09F
:104BE000406F0FF061F9834617480191406F0FF055
:104BF0005BF9814615488A46406F0FF055F9074624
:104C000013488846406F0FF04FF9054611480E468D
:104C1000406F0FF049F900900F480C46406F0FF0BD
:104C200043F90B4601990246CDE908B10DF1040B99
:104C30000AA18BE8F007184806F01FFA0BB0BDE890
:104C4000F08F0000DC0C00106C0B0010FC09001051
:104C50008C0800101C070010AC0500104D6F74206C
:104C600049206D313D25372E3366206D323D253785
:104C70002E3366206D333D25372E3366206D343D4F
:104C800025372E3366206D353D25372E3366206D52
:104C9000363D25372E336600440200102DE9F04FD3
:104CA00085B003F001F8E24CE24D606A20B1E2A168
:104CB00005F1300006F0E1F9E24F0126304604F03C
:104CC00069FA38460EF0BEFA761C062EF6DDDE488E
:104CD00005F0C4FADD4805F0C1FADD4805F0BEFA7A
:104CE000DC4805F0BBFADC4805F0B8FADB4805F013
:104CF000B5FADA4EDFF868B3606A002824D0D6F837
:104D000080000FF0D1F881468A46D44805F082F938
:104D10000FF0CAF807468846306A0FF0C5F80B4610
:104D20002169CDF80890CDE903A1CDE900780246CC
:104D3000CCA105F1300006F0A0F9FFF74DFFD6A198
:104D400005F1300006F099F95846B1690FF0A7FB5C
:104D5000B061A06A0EF076FA706FB0F17F5FCBDDC4
:104D600002F0A2FF606A002824D0D6F880000FF07D
:104D70009BF881468A46B94805F04CF90FF094F843
:104D800007468846306A0FF08FF82269CDF8089000
:104D9000CDE903A2CDE9007802460B46B1A105F1A9
:104DA000300006F06AF9FFF717FFBBA105F13000EC
:104DB00006F063F95846B1690FF0A2F8B061A06A35
:104DC0000EF040FAB548716F8142CBDA062004F04C
:104DD000E1F902F069FF606A20B1B1A105F130008C
:104DE00006F04BF900F0B8FF0700DFF86092606A48
:104DF0004FF001080ED028B13A46ADA105F13000C0
:104E000006F03BF9C9F82C8001F050F905B038469E
:104E1000BDE8F08F20B1ADA105F1300006F02DF90D
:104E20000027C9F82C70606A20B1AEA105F13000EE
:104E300006F023F9FFF720F95FEA000ADFF8109285
:104E4000606A0AD0002800F092805246A9A105F1BC
:104E5000300006F012F900F08AB820B1ABA105F1DC
:104E6000300006F00AF9C9F82C7002F01DFF606AE4
:104E700020B1ACA105F1300006F0FFF802F040F8D7
:104E80005FEA000BDFF8CC91606A09F5B87A08D0C8
:104E9000002842D05A46A8A105F1300006F0EDF8EE
:104EA0003BE020B1AAA105F1300006F0E6F8C9F810
:104EB0002C70CAF82C7002F0F7FE606A20B1ABA12A
:104EC00005F1300006F0D9F802F00EFC5FEA000BA5
:104ED000606A07D008B35A46AAA105F1300006F06F
:104EE000CCF81AE020B1AFA105F1300006F0C5F80A
:104EF000C9F82C70CAF82C7002F0D6FE606A20B196
:104F000088A105F1300006F0B8F801F0F9FF5FEA7A
:104F1000000B606A0BD00028BCD1C9F82C80CAF8FD
:104F20002C8001F0C3F805B05846BDE8F08F20B1E1
:104F300087A105F1300006F0A0F8C9F82C70CAF876
:104F40002C70606A20B19FA105F1300006F095F841
:104F500003F034FD5FEA000ADFF8EC90606A0ED0DF
:104F600028B152469DA105F1300006F086F8C9F837
:104F70002C8001F09BF805B05046BDE8F08F20B1C1
:104F80009CA105F1300006F078F8012004F002F948
:104F9000C9F82C70606A20B19BA105F1300006F0C1
:104FA0006CF800F06FFA5FEA0009606A11D028B16E
:104FB0004A4699A105F1300006F05FF8274805F050
:104FC000EDFAC6F82C8001F071F805B04846BDE84E
:104FD000F08F20B196A105F1300006F04EF80620C2
:104FE00004F0D8F8F762606A20B197A105F13000AB
:104FF00006F043F829480EF025F9A0690FF0B6F83D
:105000000146124805F0A1F8E0690FF0AFF801463B
:105010000F4805F09AF840F6AD110E4805F095F8E6
:105020008F490D4805F091F805B00020BDE8F08FDC
:10503000C800001014020010486F6D696E670D0AF9
:10504000000000000AD7A33BAC0500101C070010AD
:105050008C080010FC0900106C0B0010DC0C001018
:105060000000C84261786973363D252E31662020E4
:1050700049363D252E346620644964743D252E341E
:1050800066207374616C6C5F73746174653D307815
:1050900025303258202000000D0A0000CDCC4C3EB7
:1050A000486F6D652053686F756C6465720D0A00FA
:1050B000486F6D652053686F756C6465722066611A
:1050C000696C2C2025640D0A00000000486F6D6596
:1050D0002053686F756C64657220737563636573C4
:1050E000730D0A00486F6D6520456C626F770D0A7D
:1050F00000000000486F6D6520456C626F77206688
:1051000061696C2C2025640D0A000000486F6D65F4
:1051100020456C626F7720737563636573730D0A46
:1051200000000000486F6D6520577269737420504D
:10513000697463680D0A0000486F6D6520577269D5
:105140007374206661696C2C2025640D0A000000D0
:10515000486F6D6520577269737420506974636875
:1051600020737563636573730D0A0000486F6D6586
:1051700020577269737420526F746174696F6E0D79
:105180000A000000486F6D652057726973742052E1
:105190006F746174696F6E206661696C2C20256480
:1051A0000D0A0000486F6D652057726973742052B4
:1051B0006F746174696F6E20737563636573730DCB
:1051C0000A000000486F6D65204261736520526FD0
:1051D000746174696F6E0D0A00000000486F6D65A0
:1051E0002062617365206661696C2C2025640D0A5C
:1051F00000000000486F6D65206261736520737563
:1052000063636573730D0A00486F6D6520477269AB
:10521000707065720D0A0000486F6D6520677269D5
:1052200070706572206661696C2C2025640D0A001F
:10523000486F6D6520677269707065722073756361
:10524000636573730D0A00000D0A456E64206F6676
:10525000204D617374657220486F6D650D0A000002
:1052600053F6FFFF2DE9F34F91B0044604F0F6FF2B
:10527000D4F884000EF018FECDE90B10606F0EF02C
:1052800013FECDE90910A06A0EF00EFE82468B4691
:10529000606A0EF009FE80468946206A0EF004FE20
:1052A00006460F4660680EF0FFFD02900D46A069AD
:1052B0000EF0FAFD10900091654805F001FE0EF029
:1052C000F3FD0B9B099A0B9203AA0D9382E8E00F62
:1052D000009B109ACDE9002302460B465D495E48CB
:1052E00005F0CBFE1298A061594805F020FE53E06E
:1052F000204604F08FFED4F884000EF0D5FDCDE9F1
:105300000B10606F0EF0D0FD0A908B46A06A0EF075
:10531000CBFD82460791606A0EF0C6FD8046894645
:10532000206A0EF0C1FD06460F4660680EF0BCFD17
:1053300002900D46A0690EF0B7FD10900091444810
:1053400005F0BEFD0EF0B0FD8C460B990D9107994E
:10535000CDF82CB0CDE908A103A9024681E8E0030D
:10536000009B1099CDE9001363463A493A4805F08D
:1053700084FE3A480DF066FF354805F0A1FD384936
:10538000884204DD37A1344805F077FE15E03B483C
:1053900003F082FF002851D0394DA06929460EF054
:1053A000AFFD216A0EF04AFFA2D32946A0690FF093
:1053B00081F8216A0FF042F89AD3D4F884000EF0F5
:1053C00073FD81468A46606F0EF06EFDCDE90910CF
:1053D000A06A0EF069FD08911090606A0EF064FDFD
:1053E00080460791206A0EF05FFD06460F46606812
:1053F0000EF05AFD05460391A0690EF055FD0446D6
:105400008B46134805F05CFD0EF04EFD0B460999E6
:105410000B91CDE90C9A109A0899CDF81880CDE936
:105420000821CDE9004B024602950A490A48CDE918
:10543000046705F022FE13B0BDE8F08F01210F488C
:1054400003F0C8FFC0B2712818BF5128A4D1B4E737
:105450005C0500102458010044020010BC74133C89
:105460000000204153657420706F696E7420746968
:105470006D656F7574210D0A0000000014020010A4
:10548000000070412DE9F04F87B0D34804F0E6FEEC
:10549000D24804F0E3FED24804F0E0FED14804F024
:1054A000DDFED14804F0DAFED04804F0D7FE02F069
:1054B000FBFBCE4CCE4E3046A1690EF021FDCD4D0A
:1054C000A061A86A0EF0F0FCDFF82C83DFF82C93C3
:1054D00042464B460EF0BEFA0DF0B8FF0DF0B2FE9C
:1054E0003046A1690EF00CFDA061A86A0EF0DCFC4C
:1054F00042464B460EF0AEFA0DF0A8FF0DF0A2FEAC
:10550000686A00281AD0D4F880000EF0CDFC8346DB
:105510000391606F0EF0C8FC07468A46206A0EF0C1
:10552000C3FC0B460399CDE9027ACDE904B12969A0
:1055300002460091B2A1C14805F09FFD606FB0F135
:105540007F5FCDDDBE480DF07DFEBE48A1690EF047
:10555000A6FFA061BC480DF075FE02F0A5FBBB4F95
:10556000A16938460EF09BFFA061A86A0DF06AFEA3
:10557000686A002819D0D4F880000EF095FCCDE9B7
:105580000310606F0EF090FC82468B46206A0EF08E
:105590008BFC0B46039902460591CDE902AB2869C5
:1055A000009097A1A54805F068FDDFF8A4A2606F00
:1055B0005045D5DCA7480DF045FE8E48406A0028CE
:1055C0001FD08A48D0F880000EF06EFC83468748D2
:1055D0000391406F0EF068FC009084480D46006A0D
:1055E0000EF062FC039B0246CDE904B30098CDE9BE
:1055F0000205804800690B46009081A18F4805F0A4
:105600003CFD062003F0C6FD02F04EFB794D30460E
:10561000A1690EF044FFA061A86A0DF013FE686A4C
:10562000D0B1D4F880000EF03FFCCDE90310606FDC
:105630000EF03AFC83460091206A0EF035FC039B85
:105640000593009B0246CDE902B328690B46009002
:105650006BA17A4805F011FD7F48216A8142D6D9B5
:1056600002F022FB6248A1690EF019FFA061A86A4E
:105670000EF01AFC604A614B0EF0ECF90DF0E6FEFC
:105680000DF0E0FD686AC0B1D4F880000EF00CFCAB
:1056900081468B46606F0EF007FC06468846206AFE
:1056A0000EF002FC0B4602A981E8400B2969024674
:1056B000009153A1614805F0E0FC606FB0F17F5F9D
:1056C000D0DD5F480DF0BEFD02F0EEFA3846A1696C
:1056D0000EF016FCA061A86A0DF0B4FD686AC0B1B6
:1056E000D4F880000EF0E0FB81468B46606F0EF030
:1056F000DBFB06468846206A0EF0D6FB02AA82E84B
:10570000400B2A69009202460B463DA14B4805F02A
:10571000B4FC606F5045D9DC3846A1690EF0F0FB4F
:10572000A06147480DF08EFD02F0BEFA206A4B4A98
:1057300020F000418A4213DD062003F02BFD45488E
:105740000DF080FD686A18B145A13C4805F095FC54
:10575000264804F023FF07B04FF0FF30BDE8F08F7C
:1057600020F00046686A40B130460EF09DFB0246CC
:105770000B4645A1314805F080FC206A0EF0F6FC8E
:10578000002818BF454F11D0686A20B144A107F125
:10579000300005F072FC062003F0FCFC50460DF0D2
:1057A00051FD206A0EF0E2FC0028EDD102F07CFAF7
:1057B0000027C4E91767696A304639B10EF074FBF7
:1057C00002460B463BA11D4805F057FCE76207B0B7
:1057D0000020BDE8F08F0000AC0500101C07001091
:1057E0008C080010FC0900106C0B0010DC0C001081
:1057F0000000C842C8000010CDCCCCCCCCCCE43FDB
:10580000706F736974696F6E203D20252E3166209C
:10581000207374616C6C5F73746174653D307825BE
:10582000303258202020493D25372E3266206449E9
:1058300064543D252E34660D0A0000004402001019
:10584000CDCC4C3D000048439A99193E0000484297
:105850000AD7A33CCDCCCC3D000048C500A08C4568
:105860000D0A46756C6C207468726F77206E6F74C9
:1058700020726561636865642C2072657475726E50
:10588000202D310D0A000000706F736974696F6E0E
:10589000203D20252E31660D0A0000001402001064
:1058A0005A65726F696E67206178697320360D0AD8
:1058B0000000000047726970706572206D61782089
:1058C0007468726F7720697320252E31660D0A0087
:1058D0002DE9FF4F9146A54A8A4691B0D2E907517A
:1058E000D2E905761E980A91A149546ADFF884B27C
:1058F000C96A984671B9A049C96A59B99F49C96A24
:1059000041B99F49C96A29B99E49C96A11B99E49D5
:10591000C96A89B19F4C9DA104F1300005F0ADFB2F
:10592000DBF8240020B19CA104F1300005F0A5FBB8
:1059300015B00120BDE8F08F80F000401E908D482A
:105940000078722833D150460EF0AEFADFF86CB210
:105950009B4B5A460EF07EF80DF078FD8246484685
:105960000EF0A2FA5A46964B0EF074F80DF06EFD4A
:10597000814640460EF098FA5A46914B0EF06AF86E
:105980000DF064FD80461E980EF08EFA5A468C4B40
:105990000EF060F80DF05AFD1E901F980EF084FA7C
:1059A0005A46874B0EF056F80DF050FD1F903846C2
:1059B00051460EF077FC074648460EF075FA814ACC
:1059C000814B0EF07BF98246894630460EF06CFA28
:1059D00052464B460EF03EF80DF038FD06460EF0EE
:1059E00063FACDE9020181468A4640460EF05CFA30
:1059F000DFF8D881DFF8D8B142465B460DF058FD9C
:105A000042465B460EF05AF98346884628460EF019
:105A10004BFA5A4643460EF01DF853464A460EF0DE
:105A200059F90DF013FD054620461F990EF03AFC7A
:105A30000EF03AFACDE900010446884628460EF0F9
:105A400033FA644A644B0EF005F882468B461E9882
:105A50000EF02AFA614A624B0EF03CF90690894634
:105A60000A980EF021FA4B46069A0DF0F3FF5246C3
:105A70005B460DF01DFD434622460DF019FD0DF06D
:105A8000E5FC04460EF010FA81468846DDE9000187
:105A900001220EF0BAFD4A4643460EF01BF90DF006
:105AA000D5FC80463348406AF8B140460EF0FCF918
:105AB000CDE9060120460EF0F7F9CDE904012846AC
:105AC0000EF0F2F98B46DDE902318246894638460E
:105AD00000930EF0E9F9CDF80CB0CDE9019A024639
:105AE0000B4640A14C4805F0C8FA39462048119AA7
:105AF00004F0CAFA31462048119A04F0C5FA294642
:105B00001E48119A04F0C0FA21461D48119A04F06B
:105B1000BBFA41461B48119A04F0B6FA20980EF0E1
:105B2000C3F90C46054600223C4B0DF093FF064698
:105B30000F4628462146294A394B0DF08BFF2A464D
:105B400023460DF087FF32463B460DF0B1FC0022A4
:105B5000344B0DF0ADFC0DF079FC01460A48119A6A
:105B600004F092FA15B00020BDE8F08FF046010075
:105B7000AC050010C80000101C0700108C080010B5
:105B8000FC0900106C0B0010DC0C00104E414B0D9A
:105B90000A000000140200100D0A53636F72626F56
:105BA00074206D75737420626520486F6D65642084
:105BB000666972737421210D0A000000E8C35CB0AD
:105BC000DDA54C4052B81E85EB115E40E17A14AE63
:105BD00047C157404818062CB98ACD3FA4703D0AEA
:105BE000D73356400D0A71303D25352E326620716F
:105BF000313D25352E32662071323D25352E3266F7
:105C00002071333D25352E32662071343D25352EE9
:105C10003266200D0A0000004402001000804B4054
:105C2000D7A3C03F004052402DE9F04F8BB004464F
:105C3000DFF8F0B0DFF8F0A002A805F096F93B48D5
:105C400005F0AEFA204604F009FB02A805F07DF944
:105C50005146A0690EF054F9354FDFF8D880DFF8CF
:105C6000D890A06119E0204604F0D4F9796A89B18E
:105C70000EF01AF905460E4602A805F021F90EF0BD
:105C800013F9CDE9005602460B462CA108F130006D
:105C900005F0F3F948460DF0D5FA02A805F010F921
:105CA00059460EF0CBFADED35146A0690EF002FC45
:105CB000A06102A805F03BF91BE0204604F0AAF918
:105CC0000146786A90B108460EF0EEF805460E4699
:105CD00002A805F0F5F80EF0E7F8CDE90056024607
:105CE0000B4616A108F1300005F0C7F948460DF043
:105CF000A9FA02A805F0E4F859460EF09FFADCD3A1
:105D0000124806901248099006A9124A074805F061
:105D100013FA099906A800291CBF896888470BB0A7
:105D2000BDE8F08F0AD7A33C00007A44C00E0010F3
:105D3000C8000010140200106F12833A743D252E23
:105D4000336620252E3466200D0A00008161000094
:105D5000CC4F0100CDCC4C3D2DE9F04F89B09A4895
:105D600004F07CFA994804F079FA994804F076FA3C
:105D7000984804F073FA984804F070FA974804F0D1
:105D80006DFA01F091FF964C924E206BA6F5387596
:105D900001287DD1606A20B192A1A5F59B6005F034
:105DA0006CF9DFF82CB29A4FA96938460EF0A8F8C2
:105DB000A8613846DBF818100EF071FBCBF818001C
:105DC000B0690EF071F8DFF84C82DFF84C92424671
:105DD0004B460DF07FFF0DF039FB7F4FB061B86986
:105DE0000EF062F842464B460DF062FB0DF02EFBC2
:105DF000B861A06A0DF026FA606AF0B1D5F88000AB
:105E00000EF052F881468A46A7F58A6004F002F93E
:105E10000EF04AF807468846286A0EF045F8CDE9A4
:105E2000069A024620690297CDE90380206B0B4653
:105E300000907A497A4805F020F9206910B9206B62
:105E40000028B0D1606A2746F0B1D5F880000EF086
:105E50002BF8804689465D4804F0DCF80EF024F803
:105E600082468B46286A0EF01FF80246CDE9068965
:105E700038690B46CDF808A0CDE903B0386B009027
:105E80006649674805F0F9F8386B68B9022000E008
:105E900018E003F07FF9032003F07CF9042003F0FD
:105EA00079F9052003F076F9386958B1786A20B19C
:105EB0003A695C495A4805F0E0F809B06FF0020011
:105EC000BDE8F08F58480DF0BDF9606A18B157A1D0
:105ED000534805F0D2F8DFF8F8B0634FA9693846A7
:105EE0000EF0DDFAA8613846DBF818100EF008F85D
:105EF000CBF81800B0690DF0D7FFDFF87081DFF83C
:105F0000709142464B460DF0D3FA0DF09FFA324F96
:105F1000B061B8690DF0C8FF42464B460DF0DAFE9D
:105F20000DF094FAB861A06A0DF08CF9606AF0B1D6
:105F3000D5F880000DF0B8FF81468A46A7F58A6043
:105F400004F068F80DF0B0FF07468846286A0DF0A7
:105F5000ABFFCDE9069A22690297CDE90382226B55
:105F6000009202460B462D492D4805F086F820691F
:105F7000216B0843B1D0606AA8B1144804F04AF814
:105F80000DF092FF06460F46286A0DF08DFF02467F
:105F900020690B460296CDE90370206B009035A175
:105FA0001F4805F06AF8022003F0F4F8032003F01C
:105FB000F1F8042003F0EEF8052003F0EBF80020E0
:105FC000E86209B0BDE8F08FAC0500101C070010B6
:105FD0008C080010FC0900106C0B0010DC0C001089
:105FE000C80000100D0A4D6F76652053686F756C00
:105FF00064657220757020756E74696C20737769A2
:1060000074636820636C6F736573200D0A00000071
:106010000000C842E00B93A982B13840E05701006C
:1060200044020010D8530100CDCCCC3D0D0A4D6F79
:1060300076652053686F756C646572206261636B6E
:1060400020646F776E20756E74696C207377697445
:106050006368206F70656E7320616761696E2028C8
:10606000736C6F77290D0A00000020411AA3755444
:1060700035C103400D0A61786973323D252E3166C2
:1060800020202073773D25316420202049323D2592
:106090002E3466207374616C6C5F73746174653D3B
:1060A0003078253032580D0A000000002DE9F04FFD
:1060B0001C488BB0D0F884000DF0F6FE83461A48D9
:1060C0000191D0F884000DF0EFFE814617488A4612
:1060D000D0F884000DF0E8FE074615488846D0F851
:1060E00084000DF0E1FE054612480E46D0F884000B
:1060F0000DF0DAFE009010480C46D0F884000DF048
:10610000D3FE0B4601990246CDE908B10DF1040B0F
:106110000AA18BE8F007194804F0AFFF0BB0BDE807
:10612000F08F0000DC0C00106C0B0010FC0900105C
:106130008C0800101C070010AC0500104D61782081
:1061400049206D313D25372E3366206D323D253790
:106150002E3366206D333D25372E3366206D343D5A
:1061600025372E3366206D353D25372E3366206D5D
:10617000363D25372E33660D0A000000440200101C
:1061800070B54E4803F046FF4D4C60644D4803F037
:1061900041FFA0644C4803F03DFFE0644B4803F02E
:1061A00039FF20654A4803F035FF6065494803F030
:1061B00031FFA0654148484D406FA84210DD474E71
:1061C0003068B0F1FF3F04D12422454945480BF027
:1061D000A3FF316970680860206940F00100206108
:1061E0003848406FA84210DD3C4E3068B0F1FF3FA8
:1061F00004D124223A493B480BF08EFF3169706884
:106200000860206940F0020020612F48406FA842DA
:1062100010DD324D2868B0F1FF3F04D1242230490F
:1062200030480BF079FF296968680860206940F000
:106230000400206125482C49406F884210DD274D1D
:106240002868B0F1FF3F04D12422254925480BF0EE
:1062500063FF296968680860206940F008002061D0
:106260001B48406FB0F17E5F10DD1C4D2868B0F117
:10627000FF3F04D124221A491A480BF04DFF296927
:1062800068680860206940F0100020611148406F84
:10629000B0F17F5FD8BF70BD104D2868B0F1FF3FEF
:1062A00004D124220E490F480BF036FF2969686893
:1062B0000860206940F02000206170BDAC0500102E
:1062C000C80000101C0700108C080010FC0900100A
:1062D0006C0B0010DC0C00106666663FE4010010D9
:1062E000645D010020490000CDCC4C3F2DE9F04712
:1062F0008AB0824602A804F038FE02A804F025FE07
:10630000484D0020A96E002918BF0120464EB16EED
:10631000002918BF40F00200444FB96E002918BF91
:1063200040F00400DFF80881D8F86810002918BF91
:1063300040F00800DFF8FC90D9F86810002918BF79
:1063400040F010003C4CA16E002918BF40F0200026
:10635000A0B102A804F0B4FD51460EF06FF814D2BB
:10636000384C36A104F1300004F087FE3648406A0C
:1063700020B136A104F1300004F07FFE02A804F041
:10638000BDFD0AB00020BDE8F0872E4802F084FF72
:1063900058B901212B4803F01DF8C0B2202802D0C3
:1063A000712825D001E001F049FEA86E00220028E6
:1063B00018BF0122B06E002818BF42F00202B86E6A
:1063C000002818BF42F00402D8F86800002818BF5F
:1063D00042F00802D9F86800002818BF42F0100205
:1063E000A06E002818BF42F02002002AB1D1C5E7F4
:1063F00009A8009008AB07AA06A901A802F000FAB4
:106400001E4805F031FD05460998DDE906120090A9
:10641000089B019802F046FDA5610AB00120BDE885
:10642000F0870000AC0500101C0700108C0800105D
:10643000FC0900106C0B0010DC0C00104E414B0DE1
:106440000A00000014020010C800001054696D65B5
:106450006F7574206F636375726564206265666F23
:1064600072652066696E697368696E672070726F05
:1064700066696C65206D6F76650D0A00C9000010B5
:106480002DE9F04F0024F44EF44F91B00125284639
:1064900002F080FE38460CF0D5FE6D1C062DF6DDB0
:1064A000EF4803F0DBFEEF4803F0D8FEEE4803F0C0
:1064B000D5FEEE4803F0D2FEED4803F0CFFEED48E6
:1064C00003F0CCFEE648866100F5B870866100F501
:1064D000B87000F5B878866100F53870C8F81860B3
:1064E00000F5B87986613046C9F818600DF0DCFC1B
:1064F000CDE90B0102460B46A8F5FD65DEA105F1CD
:10650000300004F0BAFDE2480CF09CFED9F82000FF
:106510000DF0CAFC824605F658108B46006A0DF055
:10652000C3FCCDE90601D8F820000DF0BDFC814682
:1065300005F5CF600591006A0DF0B6FC029005F5F7
:10654000A1608846006A0DF0AFFCCDE9000105F5B9
:106550006670006A0DF0A8FC02460B46CDE903897F
:10656000CCA105F13000CDE908AB04F086FD05F6BD
:10657000C82003F04FFD0DF097FC834605F6581038
:10658000079103F047FD0DF08FFCCDE9051005F5EF
:10659000FD6003F03FFD0DF087FCCDE9031005F52C
:1065A000CF6003F037FD0DF07FFC824605F5A1605A
:1065B000019103F02FFD0DF077FC8046894605F52B
:1065C000667003F027FD0DF06FFC0B46079902463D
:1065D000CDE908B10599079103990591019905F154
:1065E0003000CDE902A1BBA1CDE9008904F045FD51
:1065F00005F5667003F0D2FF05F5A16003F0CEFF4C
:1066000005F5CF6003F0CAFF05F5FD6003F0C6FF96
:1066100005F6581003F0C2FF05F6C82003F0BEFFD0
:1066200005F56670DFF8E082006A804506DDB7A1F7
:1066300005F1300004F021FD44F00104DFF824B23C
:10664000DBF82000404506DAC0A105F1300004F077
:1066500014FD44F00204DFF810A2DAF820004045EF
:1066600006DACAA105F1300004F007FD44F0040485
:10667000DFF8F891D9F82000404506DAD3A105F1FA
:10668000300004F0FAFC44F008047948006A404500
:1066900006DADEA105F1300004F0EFFC44F010044E
:1066A0007448006A404506DAE8A105F1300004F0BC
:1066B000E4FC44F02004F5480CF0C4FD4FF0010860
:1066C000404602F067FD38460CF0BCFD08F10108B9
:1066D000B8F1060FF4DD624803F0C0FD614803F035
:1066E000BDFD614803F0BAFD604803F0B7FD6048A6
:1066F00003F0B4FD5F4803F0B1FD594986F0004056
:10670000886101F5B87101F5B876886101F53871D5
:10671000B06101F5B878886101F53879C8F81800DA
:10672000C9F81800DDE90B210B46D9A105F13000AD
:1067300004F0A3FC56480CF085FDD9F820000DF0BC
:10674000B3FB08908B46D8F820000DF0ADFB069007
:1067500006F5B8708A46006A0DF0A6FB04908946DB
:10676000306A0DF0A1FB0290A6F5B8708846006A69
:106770000DF09AFB0E903A480E46006A0DF094FB1D
:106780000246CDF824B0CDF814900E98CDE900065D
:106790000B46CDF81CA0CDF80C803EA105F13000D1
:1067A00004F06BFC334803F035FC0DF07DFB8346B1
:1067B0002F48079103F02EFC0DF076FB04908A46DB
:1067C0002A4803F027FC0DF06FFBCDE902012648B3
:1067D00003F020FC0DF068FB80468946214803F059
:1067E00019FC0DF061FB06461D48009103F012FCF8
:1067F0000DF05AFB0B460799CDE908B1049ACDE993
:10680000062ADDE90212CDE9041200990246CDE91B
:106810000061CDE902892FA105F1300004F02DFCC3
:106820000F4803F0BBFE0F4803F0B8FE0E4803F01C
:10683000B5FE0E4803F0B2FE0D4803F0AFFE0D4862
:1068400003F0ACFE0648984EDFF86082006AB04262
:1068500000D22DE13DE100000000C8430AD7A33B70
:10686000AC0500101C0700108C080010FC0900107B
:106870006C0B0010DC0C0010616C6C20617865738F
:10688000202B252E336620636F756E74730D0A00FE
:106890009A99993E706F73313D252E336620706F43
:1068A00073323D252E336620706F73333D252E33B2
:1068B0006620706F73343D252E336620706F7335FC
:1068C0003D252E336620706F73363D252E336620AE
:1068D000200D0A0049313D252E33662049313D25E2
:1068E0002E33662049313D252E33662049313D2522
:1068F0002E33662049313D252E33662049313D2512
:106900002E33660D0A0000000000C8424661696C23
:106910006564204D6F74203120706F7369746976DF
:106920006520636C6F736564206C6F6F7020746595
:1069300073742E204973206D6F746F722031206242
:1069400061636B77617264733F0D0A004661696C25
:106950006564204D6F74203220706F73697469769E
:106960006520636C6F736564206C6F6F7020746555
:1069700073742E204973206D6F746F722032206201
:1069800061636B77617264733F0D0A004661696CE5
:106990006564204D6F74203320706F73697469765D
:1069A0006520636C6F736564206C6F6F7020746515
:1069B00073742E204973206D6F746F7220332062C0
:1069C00061636B77617264733F0D0A004661696CA5
:1069D0006564204D6F74203420706F73697469761C
:1069E0006520636C6F736564206C6F6F70207465D5
:1069F00073742E204973206D6F746F72203420627F
:106A000061636B77617264733F0D0A004661696C64
:106A10006564204D6F74203520706F7369746976DA
:106A20006520636C6F736564206C6F6F7020746594
:106A300073742E204973206D6F746F72203520623D
:106A400061636B77617264733F0D0A004661696C24
:106A50006564204D6F74203620706F736974697699
:106A60006520636C6F736564206C6F6F7020746554
:106A700073742E204973206D6F746F7220362062FC
:106A800061636B77617264733F0D0A00CDCC4C3E3D
:106A9000616C6C2061786573202D252E3366206330
:106AA0006F756E74730D0A000000C8C20000A0402C
:106AB0006BA105F1300004F0E0FA14F0010F10D0E2
:106AC00077A105F1300004F0D8FA40460CF0BAFB8B
:106AD00007E014F0010F04D0794905F1300004F00B
:106AE000CCFA7848006AB04210D277A105F13000A4
:106AF00004F0C3FA0020022810D183A105F1300070
:106B000004F0BBFA40460CF09DFB07E00020022891
:106B100004D1854905F1300004F0AFFA8348006ADA
:106B2000B04210D282A105F1300004F0A6FA002094
:106B3000042810D18EA105F1300004F09EFA4046E1
:106B40000CF080FB07E00020042804D1904905F1F7
:106B5000300004F092FA8F48006AB04210D28EA141
:106B600005F1300004F089FA0020082810D19AA11C
:106B700005F1300004F081FA40460CF063FB07E0B9
:106B80000020082804D19C4905F1300004F075FA72
:106B90009A48006AB04210D299A105F1300004F081
:106BA0006CFA0020102810D1A5A105F1300004F0E6
:106BB00064FA40460CF046FB07E00020102804D1A0
:106BC000A74905F1300004F058FAA648006AB0421F
:106BD00010D2A5A105F1300004F04FFA0026202EB6
:106BE00011D1B1A105F1300004F047FA40460CF094
:106BF00029FB08E00026202E05D10026B24905F128
:106C0000300004F03AFAB14803F0C8FC2D4803F014
:106C1000C5FC464803F0C2FC5E4803F0BFFC774861
:106C200003F0BCFC8F4803F0B9FC0124204602F0BD
:106C3000B1FA38460CF006FB641C062CF6DDA448BD
:106C40000CF000FB002E04BF11B0BDE8F08F3246FF
:106C500011B005F13000BDE8F04F9EA104F00DBA6F
:106C60004661696C6564204D6F742031206E6567E4
:106C7000617469766520636C6F736564206C6F6FF7
:106C80007020746573742E204973206D6F746F7259
:106C90002031206261636B77617264733F0D0A007B
:106CA0004D6F74203120686173206661696C656482
:106CB00020626F746820636865636B73210D0A003E
:106CC000785401001C0700104661696C6564204D12
:106CD0006F742032206E6567617469766520636C1D
:106CE0006F736564206C6F6F7020746573742E20F1
:106CF0004973206D6F746F722032206261636B770D
:106D0000617264733F0D0A004D6F74203220686118
:106D100073206661696C656420626F7468206368C3
:106D200065636B73210D0A00D05401008C080010BC
:106D30004661696C6564204D6F742033206E656711
:106D4000617469766520636C6F736564206C6F6F26
:106D50007020746573742E204973206D6F746F7288
:106D60002033206261636B77617264733F0D0A00A8
:106D70004D6F74203320686173206661696C6564AF
:106D800020626F746820636865636B73210D0A006D
:106D900028550100FC0900104661696C6564204DAE
:106DA0006F742034206E6567617469766520636C4A
:106DB0006F736564206C6F6F7020746573742E2020
:106DC0004973206D6F746F722034206261636B773A
:106DD000617264733F0D0A004D6F74203420686146
:106DE00073206661696C656420626F7468206368F3
:106DF00065636B73210D0A00805501006C0B001058
:106E00004661696C6564204D6F742035206E65673E
:106E1000617469766520636C6F736564206C6F6F55
:106E20007020746573742E204973206D6F746F72B7
:106E30002035206261636B77617264733F0D0A00D5
:106E40004D6F74203520686173206661696C6564DC
:106E500020626F746820636865636B73210D0A009C
:106E6000D8550100DC0C00104661696C6564204D4A
:106E70006F742036206E6567617469766520636C77
:106E80006F736564206C6F6F7020746573742E204F
:106E90004973206D6F746F722036206261636B7767
:106EA000617264733F0D0A004D6F74203620686173
:106EB00073206661696C656420626F746820636822
:106EC00065636B73210D0A0030560100AC0500109C
:106ED000CDCC4C3E4572726F725F737461746520E5
:106EE0003D203078253034582C2065786974696EDF
:106EF000672070726F6772616D210D0A00000000DB
:106F00002DE9F04F91B0FC4803F0A8F9FB4803F0DD
:106F1000A5F9FB4803F0A2F9FA4803F09FF9FA48F3
:106F200003F09CF9F94803F099F900F0BDFE042044
:106F300002F030F9052002F02DF9F548806B0128A8
:106F400066D000F0B1FEF24CEE4DF24F3846A96922
:106F50000CF0D6FF05F5B876A8613846B1690DF09A
:106F60009EFAB061A06A0CF06DF9606A002837D013
:106F700005F5B870D0F880000CF096FF82462846E0
:106F80008B46D0F880000CF08FFF8046894605F5CF
:106F9000B87003F03FF80CF087FF06900F462846C4
:106FA00003F038F80CF080FF0546D7480E46006A1B
:106FB0000CF07AFFCDE90001D248006A0CF074FFB2
:106FC00002460AA80B4680E8000F2069D249CDE9A5
:106FD0000770CDE90456A06B0290D04804F04DF83C
:106FE0002169A06B0843AFD02069002800F06882B7
:106FF000DA4CCBA104F1300004F03FF8D8A104F141
:10700000300004F03AF811B06FF00400BDE8F08FE2
:10701000BF4E706A18B1D549C04804F02EF800F090
:1070200043FEB84D05F5B874D14FA96938460DF047
:1070300036FAA8613846A1690CF062FFA061B06A17
:107040000CF000F9706A00283AD0D4F880000CF0F7
:107050002BFFCDE90801D5F880000CF025FF824612
:107060008B46A94802F0D6FF0CF01EFF8146A548CA
:10707000059102F0CFFF0CF017FF02908846206ABE
:107080000CF012FF07460091286A0CF00DFFDDE9B5
:107090000823CDE90C23CDE90AAB32690892059AA1
:1070A0000B46CDE90692029ACDE90428B26B029212
:1070B000009A9949CDE900720246984803F0DDFF35
:1070C0003069002804BFB06B012807D1A948296A9C
:1070D000814203D2A848216A8142A5DB8C48406ADC
:1070E00000283DD02646D4F880000CF0DDFE824614
:1070F00084488B46D0F880000CF0D6FE8046894646
:10710000814802F087FF0CF0CFFECDE905107D48E5
:1071100002F080FF0CF0C8FE04910290306A0CF07F
:10712000C3FE064677480F46006A0CF0BDFE0B46CC
:107130000AA9DFF8DCC181E8000FDCF81010089123
:1071400005990791049A0299CDE90412DCF83810E8
:107150000096CDE9017102466F49704803F08DFF3A
:107160006B4E3069C0B1706A20B1326983A16B483F
:1071700003F083FF7E4FA8463846A9690CF0C0FE95
:10718000C8F81800A0463846A1690DF088F9C8F87B
:107190001800B06A0CF056F8042001F0FBFF05203F
:1071A00001F0F8FF00F080FD706A18B17AA15B4829
:1071B00003F063FF844FA96938460CF0A1FEA86173
:1071C0003846A1690DF06BF9A061B06A0CF03AF88D
:1071D000706AA8B3D4F880000CF066FE0A908B4663
:1071E000D5F880000CF060FECDE90710464802F0AB
:1071F00011FF0CF059FE06908A46424802F00AFF41
:107200000CF052FE80468946206A0CF04DFECDE916
:107210000001286A0CF048FE02460A98CDE90C0BE2
:10722000DDE90730CDE90A0330690B46CDE907A057
:10723000CDE90489B06B02903749384803F01DFF4F
:107240003069002804BFB06B0128B4D03048406AD0
:10725000E0B3A246D4F880000CF026FE814629480F
:107260008B46D0F880000CF01FFE06468846264864
:1072700002F0D0FE0CF018FECDE90510214802F016
:10728000C9FE0CF011FE02910490DAF820000CF017
:107290000BFE82461B480191006A0CF005FE0B466E
:1072A0000AA9DFF86CC081E8400BDCF810100891E7
:1072B0000599079102990591DCF838100246029170
:1072C000CDF800A01449154803F0D7FE104E3069E0
:1072D0000028706A7DD020B132693C490F4803F024
:1072E000CCFE084803F05AF9074803F057F911B0EB
:1072F0004FF0FF30BDE8F08FAC0500101C07001008
:107300008C080010FC0900106C0B0010DC0C001045
:10731000C80000100000F04180520100440200103B
:107320007374616C6C206465746563746564207744
:1073300068696C652073776974636820776173206E
:10734000737570706F73656420746F20626520635D
:107350006C6F73656421210D0A0000001402001097
:1073600072657475726E202D350D0A00805701000C
:107370000000484200803BC500803B450D0A6D611E
:107380007820777269737420757020726561636804
:1073900065640D0A000000004D6F76696E67205726
:1073A0007269737420646F776E20756E74696C20D7
:1073B0006C696D69742073776974636820636C6F9E
:1073C0007365730D0A00000000002042885601001A
:1073D000FFE718B18CA1994803F04FFE994D984FE3
:1073E0003846A9690CF08CFD05F5B874A8613846DB
:1073F000A1690DF054F8A061B06A0BF023FF706A28
:10740000E8B3D4F880000CF04FFDCDE90910A4F5E5
:10741000B870D0F880000CF047FD08908B462046ED
:1074200002F0F8FD0CF040FD81468A46A4F5B870E4
:1074300002F0F0FD0CF038FD07468846206A0CF09B
:1074400033FD04467F480D46006A0CF02DFD0B46C7
:10745000DDE90921CDE90C12089ACDE90A2B316941
:10746000CDF81890CDE907A1CDE90478B16B00946F
:10747000CDE9015102467449704803F0FEFD3069C0
:10748000B16B0843AAD0306988B1706A20B1326903
:107490006E496A4803F0F1FD6A4803F07FF86C48D2
:1074A00003F07CF811B06FF00100BDE8F08F012906
:1074B0007CD1706A68B167A1604803F0DEFD08E026
:1074C000A06B012872D1606A18B16DA15B4803F00E
:1074D000D4FD042001F05EFE052001F05BFE594D55
:1074E000724E3046A9690CF00BFD05F5B874A86121
:1074F0003046A1690CF0D3FFA0616D480BF0A2FEED
:1075000000F0D2FB6B4C4F4E6B4F3846B1690CF01C
:10751000C6FF06F5B875B0613846A9690CF0F0FCF5
:10752000A861A06A0BF08EFE606AE0B3D5F8800017
:107530000CF0BAFC8346A5F5B8700991D0F880002C
:107540000CF0B2FC82462846079102F063FD0CF075
:10755000ABFC8146A5F5B870059102F05BFD0CF01F
:10756000A3FC07468846286A0CF09EFC0546354871
:107570000E46006A0CF098FC0B4609990246CDE9CC
:107580000CB10799CDE90AA120690599CDE90478E4
:10759000CDE906910890A06B0095CDE901602A49DC
:1075A000264803F06AFD2069002800E017E004BFC8
:1075B000A06B0128A7D0206978B1414C3F4904F164
:1075C000300003F05AFD3FA104F1300003F055FDF7
:1075D00011B06FF00500BDE8F08FA06B20B111B0C5
:1075E0004FF0FF30BDE8F08F606A18B138A1134842
:1075F00003F043FD042001F0CDFD052001F0CAFD9C
:1076000011B00020BDE8F08F4D6F76696E6720578E
:107610007269737420646F776E20756E74696C2064
:107620006C696D697420737769746368206F706525
:107630006E7320616761696E0D0A000044020010DC
:1076400000002042FC09001080520100E0560100B9
:107650006C0B001057726973742070697463682032
:10766000686F6D65642120466972737420496620D5
:10767000636F6E646974696F6E210D0A0D0A0000F4
:10768000577269737420706974636820686F6D65E0
:107690006421205365636F6E6420494620636F6EDA
:1076A000646974696F6E0D0A0D0A00000000E14301
:1076B000CDCC4C3EC800001000002041E05201003B
:1076C0001402001072657475726E202D360D0A005A
:1076D000577269737420706974636820686F6D6590
:1076E00064210D0A0D0A00002DE9F04F8FB004202F
:1076F00001F050FD052001F04DFDFD4802F0AEFD0A
:10770000FC4802F0ABFDFC4802F0A8FDFB4802F08B
:10771000A5FDFB4802F0A2FDFA4802F09FFD00F033
:10772000C3FAF94CF54EE06B06F5B875A5F6581797
:10773000012840F08181606A20B1F4A107F1300096
:1077400003F09BFCFE4FB16938460CF0D9FBB061E9
:107750003846A9690CF0D4FBA861A06A0BF072FD51
:10776000606A00283AD0D5F880000CF09DFBCDE986
:107770000201D6F880000CF097FB04908B46E0489D
:1077800002F048FC0CF090FBCDE90001DB4802F070
:1077900041FC0CF089FB81468A46286A0CF084FB88
:1077A00007468846306A0CF07FFB0246DDE902039B
:1077B000CDE90C030498CDE90A0B20690890DDE9B6
:1077C0000003CDE90603CDE9049AE06B0097CDE90B
:1077D00001800B46DB49DC4803F04FFC20690028A0
:1077E00004BFE06B0128ADD0C748406A00283DD0F7
:1077F000AA46D5F880000CF057FB0446BF4801911B
:10780000D0F880000CF050FB04908B46BC4802F08E
:1078100001FC0CF049FB80468946B84802F0FAFBAF
:107820000CF042FB02900F46DAF820000CF03CFB13
:107830000090B2488A46006A0CF036FB0246019876
:10784000B14BCDE90C400498CDE90A0B1869CDF88D
:107850001880CDE907900298CDE90407D86B0B4654
:10786000CDE901A0B749B84803F007FCA64C206950
:1078700058B1606A20B12269B449B34803F0FDFBF6
:107880000FB04FF0FF30BDE8F08FE06B002840F004
:10789000D5819A4EAE4F3846B1690CF031FB06F5F2
:1078A000B875B0613846A9690CF02AFBA861A06AD6
:1078B0000BF0C8FC606A00283CD0D5F880000CF0C2
:1078C000F3FA0290A5F5B8708B46D0F880000CF062
:1078D000EBFA81468A46284602F09CFB0CF0E4FA5B
:1078E00007468846A5F5B87002F094FB0CF0DCFA68
:1078F00006460191286A0CF0D7FA00907F480D46A1
:10790000006A0CF0D1FA02460298CDF834B0CDF8F6
:107910002890CDE90BA020690697CDE90780019B4F
:10792000CDE90463E06B0B46CDE9015085498648FB
:1079300003F0A3FB2069E16B0843AAD0206900286B
:107940004FD07148406A002800F06E816C4ED6F826
:1079500080000CF0A9FACDE90001A6F5B870D0F8C6
:1079600080000CF0A1FA05468846304602F052FB32
:107970000CF09AFA04468B46A6F5B87002F04AFB62
:107980000CF092FA81468A46306A0CF08DFA06466F
:107990005A480F46006A0CF087FA02460B46DDE9AA
:1079A0000001DFF864C1CDE90A58CDE90C01DCF82B
:1079B0001000CDF81090CDE907B0CDE905A4DCF8B2
:1079C0003C000096CDE90170624C5E4904F1300044
:1079D00003F053FB60A104F1300003F04EFB00F014
:1079E00023B92069002808BF012940F02781606A77
:1079F00018B163A1544803F040FB206A0CF0B6FBB9
:107A00000CF0F0FB3D4C0546A1690CF079FAA06141
:107A100004F5B8742846A1690CF072FAA0616048B8
:107A20000BF010FC042001F0B5FB052001F0B2FBC7
:107A30000FB00020BDE8F08F304E5A4F3846B16984
:107A40000CF05EFA06F5B875B0613846A9690CF01D
:107A500057FAA861A06A0BF0F5FB606AE0B3D5F8AD
:107A600080000CF021FACDE90001A5F5B870D0F83E
:107A700080000CF019FA82468B46284602F0CAFABA
:107A80000CF012FA8146A5F5B870029102F0C2FA24
:107A90000CF00AFA07468846286A0CF005FA0546F3
:107AA00016480E46006A0CF0FFF902460B46DDE967
:107AB0000001CDE90C01CDE90AAB20690299CDE9BD
:107AC0000478CDE906910890E06B0095CDE901605E
:107AD0001C491D4803F0D1FA2069E16B0843ABD083
:107AE000206918B10848406A08B15DE0A1E09BE058
:107AF000AC0500101C0700108C080010FC090010D9
:107B00006C0B0010DC0C0010C8000010526F746188
:107B100074652043435720286C6F6F6B696E672034
:107B200061742920756E74696C206C696D697420AC
:107B3000697320707265737365640D0A000000003C
:107B40000000C842D451010044020010385701001F
:107B500000002042140200105374616C6C20737496
:107B600061746520726561636865642C206578695D
:107B700074696E672077697468202D320D0A0000E1
:107B8000577269737420526F7461746520486F6D09
:107B90006520737563636573732121200D0A0000EE
:107BA000CDCC8C3F00002041394CD4F880000CF043
:107BB0007BF98246A4F5B8708B46D0F880000CF0B3
:107BC00073F980468946204602F024FA0CF06CF9DD
:107BD0000746A4F5B870019102F01CFA0CF064F9A4
:107BE00005460E46206A0CF05FF9044629480091CC
:107BF000006A0CF059F902460AA8DFF89CC080E838
:107C0000000FDCF810000B460199CDE90456CDE9D0
:107C100006710890DCF83C0000990290CDE9004123
:107C20001E491F4803F029FA0FB06FF00100BDE8AC
:107C3000F08F2069002808BF012903D00FB0002071
:107C4000BDE8F08F606A20B1AFF2CC01144803F0B8
:107C500014FA206A0CF08AFA0CF0C4FA0D4C0546AE
:107C6000A1690CF04DF9A06104F5B8742846A1692A
:107C70000CF046F9A0610B480BF0E4FA042001F087
:107C800089FA052001F086FA0FB00020BDE8F08FD8
:107C90006C0B0010FC090010C8000010D45101004A
:107CA000440200109A99993F10B5084C2068B0F131
:107CB000FF3F04D12422064906480AF02DFAE16864
:107CC0006068086004490020086110BDE4010010EC
:107CD000645D010020490000C800001070B5744CBC
:107CE00084B02068B0F1FF3F04D12C227149724862
:107CF0000AF012FA606900686168084018BF012044
:107D00006E4D00286E4CE8626E4800906E486946E1
:107D1000039405D002F030FF0399684639B104E0BE
:107D200002F062FF0399684609B189688847674E87
:107D30003068B0F1FF3F04D12C225E495E480AF062
:107D4000EBF9706900687168084018BF012028636A
:107D500000285F4800905F486946039405D002F010
:107D60000BFF0399684639B104E002F03DFF039927
:107D7000684609B189688847574E3068B0F1FF3FBF
:107D800004D12C224B494C480AF0C6F970690068AE
:107D90007168084018BF0120686300284F480090B0
:107DA0004F486946039405D002F0E6FE0399684601
:107DB00039B104E002F018FF0399684609B18968F7
:107DC0008847484E3068B0F1FF3F04D12C22394932
:107DD00039480AF0A1F9706900687168084018BF55
:107DE0000120A86300284048009040486946039459
:107DF00005D002F0C1FE0399684639B104E002F0F3
:107E0000F3FE0399684609B189688847384E30689F
:107E1000B0F1FF3F04D12C22264927480AF07CF913
:107E2000706900687168084018BF0120E863002885
:107E30003048009030486946039405D002F09CFE1B
:107E40000399684639B104E002F0CEFE0399684612
:107E500009B189688847294E3068B0F1FF3F04D1E5
:107E60002C22144914480AF057F9706900687168A7
:107E7000084018BF012028640028214800902148AC
:107E80006946039408D002F077FE039968460029FA
:107E900004BF04B070BD07E002F0A6FE0399684677
:107EA000002904BF04B070BD8968884704B070BD64
:107EB0001C030010645D010020490000C800001090
:107EC000CC4F0100AD480000AC030010340300109B
:107ED00045490000F40300104C030010C94900009C
:107EE0003C040010640300104D4A0000840400109C
:107EF0007C030010D14A0000CC0400109403001051
:107F0000554B00001405001070B5454C2068B0F1C9
:107F1000FF3F04D12422434943480AF0FDF8E168B9
:107F200060680860414C2068B0F1FF3F04D1242212
:107F30003C493D480AF0F0F8E168606808603C4C54
:107F40002068B0F1FF3F04D12422364936480AF0B8
:107F5000E3F8E16860680860314C2068B0F1FF3FE9
:107F600004D124222F4930480AF0D6F821696068EC
:107F70000860304E30460BF065F9294C2068B0F1AE
:107F8000FF3F04D12422274927480AF0C5F8E168B9
:107F900060680860284D28460BF054F9234C20688F
:107FA000B0F1FF3F04D124221E491F480AF0B4F863
:107FB00021696068086030460BF044F91B4C20686A
:107FC000B0F1FF3F04D12422164917480AF0A4F863
:107FD000E1686068086028460BF034F9144C2068AA
:107FE000B0F1FF3F04D124220E490F480AF094F863
:107FF00021696068086030460BF024F90C4C206859
:10800000B0F1FF3F04D12422064907480AF084F862
:10801000E168606808602846BDE870400BF012B95E
:10802000B4010010645D010020490000CC01001083
:10803000E4010010CDCCCC3DCDCC4C3E2DE9F04F31
:10804000F34DF448F44E2978A0F55674F34F806A46
:1080500095B0632900F0A2800DF13408642900F086
:108060003F8172291CBF15B0BDE8F08F0BF01CFFDB
:1080700032463B460BF0EEFC02460B46E8A1EA48CE
:1080800002F0FBFF13AB0FAA12A90EA8CDF80080D7
:1080900000F0B6FBE54803F0E7FE0BF005FFCDE985
:1080A00006010D980BF000FF82468B4613980BF0EB
:1080B000FBFE804689460F980BF0F6FE02900F46B5
:1080C00012980BF0F1FE04460E460E980BF0ECFEF3
:1080D0000B460246DDE90601CDE90046CDE908017F
:1080E00003ACD3A184E8800FCF4802F0C6FFD84C80
:1080F00004F5B87794F82C0097F82C1004F538762E
:1081000004F58A68084396F82C1098F82C2004F59A
:10811000B8691143084399F82C1004F5E66A08433E
:108120009AF82C10084300F03F02CAA1A4F55A7037
:1081300002F0A3FFA06E0022002818BF0122B86E33
:10814000002818BF42F00202B06E002818BF42F0AB
:108150000402D8F86800002818BF42F00802D9F8D5
:108160006800002818BF42F01002DAF86800002802
:1081700018BF42F02002B9A1BA4C04F1300002F05D
:108180007CFFB9A104F1300002F077FF6868002895
:1081900004BF15B0BDE8F08F00F09AB80BF084FE74
:1081A00032463B460BF056FC02460B469CA104F1BE
:1081B000300002F062FFAD48006A0BF075FE0490DB
:1081C000AB488B46006A0BF06FFE8246A9480791C8
:1081D000006A0BF069FECDE91001A748006A0BF0B8
:1081E00063FE8046A5488946006A0BF05DFE0646A0
:1081F00097480F46006A0BF057FE02460498CDE9F7
:10820000080BCDF818A0DDE91003CDE904038DE8D3
:10821000C0030B469AA104F1300002F02EFF9348F0
:10822000406A0BF041FE069091488B46406A0BF085
:108230003BFE02908F488A46406A0BF035FE049060
:108240008D488946406A0BF02FFE80468B4801918D
:10825000406A0BF029FE06467D480F46406A0BF047
:1082600023FE02460698CDE9080B0298CDF81CA023
:10827000CDE90590019B04F13000CDE902830B4666
:1082800087A1CDE9006702F0F8FE79497748A1F5AA
:10829000B873CA6AC06AA1F53871DB6AC96ACDE9E8
:1082A00002207648CDE90013C36AA0F5B87084A116
:1082B000C26A04F1300002F0E0FE6BA104F130006C
:1082C00002F0DBFE6868002804BF15B0BDE8F08F3F
:1082D00080A104F1300002F0D0FE15B0BDE8F08FAF
:1082E0000BF0E2FD32463B460BF0B4FB02460B4678
:1082F0004BA14D4802F0C1FE13AB0FAA12A90EA864
:10830000CDF8008000F07CFA484803F0ADFD0BF09A
:10831000CBFD82468B460D980BF0C6FD8146119130
:1083200013980BF0C1FD804605910F980BF0BCFD32
:1083300006460F4612980BF0B7FD044601910E98C1
:108340000BF0B2FD0B461199CDE908ABCDE90691D2
:108350000246CDF8108000945FA13348CDE9026752
:1083600002F08BFE3A4E06F5B87896F82C0098F895
:108370002C1006F5387906F58A64084399F82C1014
:1083800094F82C2004F5B87A114308439AF82C107D
:1083900004F53877084397F82C10084300F03F02A3
:1083A0002CA1A4F5F76002F068FEB06E0022002850
:1083B00018BF0122D8F86800002818BF42F0020256
:1083C000D9F86800002818BF42F00402A06E002807
:1083D00018BF42F00802DAF86800002818BF42F01F
:1083E0001002B86E002818BF42F020021BA11D4CDD
:1083F00004F1300002F041FE1BA104F1300002F054
:108400003CFE686800287FF463AF15B0BDE8F08FCC
:10841000C80000106C050010FCA9F1D24D62503F5D
:1084200054252E326600000044020010C9000010DE
:108430005052252E34662C252E34662C252E34667B
:108440002C252E34662C252E34662C252E336600E2
:10845000AC05001053253032580000004D25303255
:1084600058000000140200100D000000DC0C001089
:108470006C0B0010FC0900108C0800101C07001089
:108480005043252E31662C252E31662C252E316643
:108490002C252E31662C252E31662C252E3166009A
:1084A00056252E32662C252E32662C252E32662C31
:1084B000252E32662C252E32662C252E32660000A3
:1084C0005325642C25642C25642C25642C25642CD0
:1084D000256400000A0000005044252E32662C2539
:1084E0002E32662C252E32662C252E32662C252E19
:1084F00032662C252E32660070B505460BF072FEF2
:10850000134CA1690BF0CBFFA06128460BF04FFA8A
:10851000104A114B0BF09EFA104E04460D46B069FE
:108520000BF0C2FC2B4622460BF0D4FB0AF08EFF68
:10853000B0612E4625460A4CA0690BF0B5FC2A46D0
:1085400033460AF0B5FF0AF081FFA06170BD00005C
:108550008C080010909E2287889BCF3FFC0900105A
:108560006C0B001070B52D4C84B026463068B0F10D
:10857000FF3F04D12C222A492A4809F0CDFD706919
:1085800000687168084214BF002501252068B0F119
:10859000FF3F04D124222249224809F0BDFD606832
:1085A000002D14BFE168216908603068B0F1FF3F19
:1085B00004D12C221A491B4809F0AEFD70690068ED
:1085C0007168084218486946AFF26702009203904A
:1085D00007D0164A164802F0AFFD0399684649B124
:1085E00006E0144A124802F0A7FD0399684609B153
:1085F00089688847104890F855001B281CBF04B0B4
:1086000070BDBFF34F8F0D4801680D4A01F4E06162
:1086100011430160BFF34F8F00BFFDE7B4010010AD
:10862000645D010020490000CC4F01006666A63F52
:10863000700E0010CDCC4C3E140200100CED00E08A
:108640000400FA0570B505460BF0CCFD134CA1698A
:108650000BF056FCA06128460BF0A9F9104A114B0B
:108660000BF0F8F9104E04460D46B0690BF01CFCF7
:108670002B4622460AF01CFF0AF0E8FEB0612E46A7
:1086800025460A4CA0690BF00FFC2A4633460BF036
:1086900021FB0AF0DBFEA06170BD00008C08001019
:1086A000909E2287889BCF3FFC0900106C0B001026
:1086B0002DE9F04784B0064690460D46684602F024
:1086C00054FC0024A2462746684602F03EFC1CE00B
:1086D000DFF81C91D9F80000B0F1FF3F04D124224B
:1086E0004449454809F018FDD9F80C00D9F80410A0
:1086F0000160BAF1000F0ED0BAF1010F2BD0BAF120
:10870000020F18BF4FF0000A3BD0AC42E0DB04B0D0
:108710002046BDE8F087394800F0BEFD60B9012170
:10872000364800F057FE3055641CAC4204D0334844
:1087300000F0B2FD0028F2D0DFF8B4904FF0010A4B
:10874000D9F80000B0F1FF3F15D1242229492A4869
:1087500009F0E2FC0FE0684602F0B2FB41460BF084
:10876000CFFBDFF88C9007464FF0020AD9F80000E3
:10877000B0F1FF3FE9D0D9F81010D9F80400086033
:10878000C3E71E4800F088FDC8B1684602F098FBB8
:1087900039460BF053FE98BF4FF0030ADFF85090B4
:1087A000D9F80000B0F1FF3F1CD000BFD9F810107D
:1087B000D9F804000860BAF1030FA6D1A7E7012198
:1087C0000E4800F007FE3055641CAC4214BF4FF059
:1087D000000A4FF0030ADFF81890D9F80000B0F152
:1087E000FF3FE3D124220349034809F095FCDDE76C
:1087F000CC010010645D010020490000140200104B
:108800002DE9FF4F604883B0614AD0E90A17D0E9EB
:108810000D45066B5D48D2F820B002F5B872006ACB
:10882000126A01925B4AD2F8209002F5B872D2F82F
:1088300020A00BF0D9FB0090394658460BF0D4FB32
:1088400080F000400BF030FB534A544B0AF030FEEE
:108850000AF0FCFD8046584601990BF051FB80F070
:10886000004031460BF0C0FB074628460BF01CFBCE
:1088700001220BF0CAFE83460E46494650460BF0D5
:108880003FFB0BF011FB5A4633460AF0CDFE0AF0CF
:10889000DDFD0646214648460BF0A6FB0BF004FB27
:1088A00081460291284631460BF0FCFC21460BF034
:1088B0009BFB0BF0F9FA05468A4620460BF0F4FACA
:1088C00083460C4601980BF0EFFA354A354B0BF016
:1088D000C1F85A4623460AF0A7FE334A334B0AF042
:1088E000E7FD2A4653460AF0E3FD4A46029B0BF099
:1088F000F1F90AF0ABFD04462D480078722834D116
:1089000000980BF0D1FA2B4DDFF8AC902A464B467D
:108910000BF0A0F80AF09AFD009040460BF0C4FA64
:108920002A464B460BF096F80AF090FD80463846F2
:108930000BF0BAFA2A464B460BF08CF80AF086FD8B
:10894000074620460BF0B0FA2A464B460BF082F859
:108950000AF07CFD044630460BF0A6FA2A464B4648
:108960000BF078F80AF072FD06460399009808604B
:108970000498C0F800800598076006980460109875
:10898000066007B0BDE8F08FF0460100AC050010AE
:108990001C070010FC09001052B81E85EB115E4048
:1089A0004818062CB98ACD3FA4703D0AD73356C06B
:1089B000C800001070E20DA545DF913F2DE9F04F92
:1089C00089B0E44801F04AFCE34801F047FCE34881
:1089D00001F044FCE24801F041FCE24801F03EFCB9
:1089E000E14801F03BFCFFF75FF9E04CE04E606AC4
:1089F00020B1E0A106F1300002F03FFBE06AD54D66
:108A0000002800F02E81012000F0C4FB606A0028DD
:108A100027D0DCA106F13000E26A02F02EFB606A8A
:108A200000281ED0D5F880000BF03EFA81468A4619
:108A3000C84801F0EFFA0BF037FA07468846286A73
:108A40000BF032FACDE9069A024620690B460297EE
:108A5000CDE90380E06A0090D1A106F1300002F078
:108A60000CFBDFF874B3A86959460BF049FAA8610A
:108A7000A06A0AF0E7FBE06A28B1206918B9D74973
:108A8000286A8842CBDB606A002848D0D5F880008D
:108A90000BF00AFA81468A46AE4801F0BBFA0BF0A9
:108AA00003FA07468846286A0BF0FEF9CDE9069AD4
:108AB000024620690297CDE90380E06A0B460090E8
:108AC000B7A106F1300002F0D8FA606A002826D07B
:108AD000C3A106F13000E26A02F0CFFA606AF0B199
:108AE000D5F880000BF0E0F981468A46994801F0FC
:108AF00091FA0BF0D9F907468846286A0BF0D4F9A9
:108B0000CDE9069A0B4621690297CDE90381E16A16
:108B100002460091A2A106F1300002F0AEFA5946D9
:108B2000A8690BF0C7FCA861A06A0AF08BFBE06A99
:108B300010B120690028D1D0606AF0B1D5F880006A
:108B40000BF0B2F981468A46824801F063FA0BF0D5
:108B5000ABF907468846286A0BF0A6F9CDE9069AD4
:108B6000024620690297CDE90380E06A0B46009037
:108B70008BA106F1300002F080FA2069002870D045
:108B8000012000F007FBFFF78FF8606A30B39B49C4
:108B900006F13000E26A02F070FA606AF0B1D5F8CE
:108BA00080000BF081F981468A466A4801F032FA6A
:108BB0000BF07AF907468846286A0BF075F9CDE97B
:108BC000069A024620690297CDE90380E06A0B46C7
:108BD000009073A106F1300002F04FFA5946A869DF
:108BE0000BF08EF9A861A06A0AF02CFBE06A10B1C4
:108BF00020690028D1D0606AF0B1D5F880000BF070
:108C000053F981468A46534801F004FA0BF04CF9B7
:108C100007468846286A0BF047F9CDE9069A0246CE
:108C200020690B460297CDE90380E06A00905CA1C1
:108C300006F1300002F021FA206900281CBF606AAA
:108C4000002804D06EA106F1300002F016FAE06AA6
:108C500038B97649A8690BF053F9A86174480AF04D
:108C6000F1FA012000F096FAFFF71EF8606A00287A
:108C700026D070A106F13000E26A02F0FEF9606AC7
:108C8000F0B1D5F880000BF00FF981468A463148E3
:108C900001F0C0F90BF008F907468846286A0BF086
:108CA00003F9CDE9069A024620690B460297CDE901
:108CB0000380E06A00903AA106F1300002F0DDF98D
:108CC0005A49A8690BF01CF9A861A06A0AF0BAFA1F
:108CD000E06A012802D020690028D0D0206900284D
:108CE000606A0DD020B162A106F1300002F0C5F932
:108CF000184801F053FC09B06FF00100BDE8F08F97
:108D0000F8B1D5F880000BF0CFF8804689461148BD
:108D100001F080F90BF0C8F882460F46286A0BF084
:108D2000C3F80B46CDE906892169CDF808A0CDE945
:108D30000371E16A0246009119A106F1300002F0C8
:108D40009CF9012000F026FA0020E86209B0BDE895
:108D5000F08F0000AC0500101C0700108C080010FC
:108D6000FC0900106C0B0010DC0C0010C800001097
:108D700014020010486F6D696E6720426173650DC3
:108D80000A0000004D6F76696E672043572C204C17
:108D9000696D69742031203D2025640D0A000000B2
:108DA00061786973313D252E3166207377313D2519
:108DB00031642049313D252E3366207374616C6C1B
:108DC0005F73746174653D30782530325820617866
:108DD00031644964540D0A000000C8420000FA449E
:108DE0004D6F76696E67204343572C204C696D693F
:108DF000742031203D2025640D0A00003852010006
:108E0000436F6C6C6973696F6E206465746563741D
:108E100065642C2052657475726E696E6720657288
:108E2000726F72202D310D0A0000000000002041F9
:108E30000AD7A33C4D6F76696E6720636C6F636BD6
:108E40007769736520286C6F6F6B696E6720646F3C
:108E5000776E2920756E74696C2073776974636806
:108E60002069732072656C6561736564200D0A006A
:108E7000436F6C6C6973696F6E20646574656374AD
:108E8000656420696E206572726F722C2065786946
:108E90007420776974682072657475726E202D3243
:108EA0000D0A00002DE9FF4F8A468E49804691B099
:108EB000D1E90240D1E9007609908B480D69DFF8CD
:108EC0002CB2C06A70B98A48C06A58B98948C06A69
:108ED00040B98948C06A28B98848C06A10B988482A
:108EE000C06A88B1894C87A104F1300002F0C5F84E
:108EF000DBF8240020B186A104F1300002F0BDF8B7
:108F000015B00120BDE8F08F784883F00049007863
:108F1000722833D140460AF0C7FFDFF818B2864BFB
:108F20005A460AF097FD0AF091FA804650460AF038
:108F3000BBFF5A46804B0AF08DFD0AF087FA824645
:108F400013980AF0B1FF5A467B4B0AF083FD0AF0F2
:108F50007DFA139048460AF0A7FF5A46764B0AF06E
:108F600079FD0AF073FA81461E980AF09DFF5A4671
:108F7000714B0AF06FFD0AF069FA1E9039464046BF
:108F80000BF090F9804650460AF08EFF6B4A6C4B0E
:108F90000AF094FE82460F4630460AF085FF52469C
:108FA0003B460AF057FD0AF051FA07460AF07CFFEB
:108FB000CDE9020106468A4613980AF075FFDFF8EC
:108FC00084B1614B5A460AF073FA5A465E4B0AF076
:108FD00075FE8346204605910AF066FF5A46059BBA
:108FE0000AF038FD534632460AF074FE0AF02EFAB3
:108FF000044628461E990BF055F90AF055FF06461F
:109000000D46204601910AF04FFF504A504B0AF09E
:1090100021FD8346484604910AF046FF4D4A4E4BD7
:109020000AF058FE81468A4609980AF03DFF4A46F2
:1090300053460AF00FFD5A46049B0AF039FA2B46B4
:1090400032460AF035FA0AF001FA05460AF02CFF1A
:10905000824689463046012201990BF0D6FA5246E3
:109060004B460AF037FE0AF0F1F906461F48406AFF
:1090700020B330460AF018FFCDE9060128460AF071
:1090800013FF8346204605910AF00EFFCDE90A0141
:10909000DDE902918A4640460AF006FF0B46DDE90B
:1090A0000A1CCDF810B0CDF80CC0CDF80090CDE979
:1090B00001A1024629A1364801F0DFFF0A48C0F8A5
:1090C000188000F5B870876100F5B870846100F50C
:1090D000B870856100F5B870866115B00020BDE8F4
:1090E000F08F0000F0460100AC050010C800001031
:1090F0001C0700108C080010FC0900106C0B0010FD
:10910000DC0C00104E414B0D0A0000001402001050
:109110000D0A53636F72626F74206D7573742062F1
:109120006520486F6D656420666972737421210D36
:109130000A000000E8C35CB0DDA54C4052B81E85B3
:10914000EB115E40E17A14AE47C157404818062C37
:10915000B98ACD3FA4703D0AD73356400D0A71300D
:109160003D25352E32662071313D25352E32662063
:1091700071323D25352E32662071333D25352E3234
:10918000662071343D25352E3266200D0A00000020
:109190004402001010B504461D4801F0FFF91D48B7
:1091A00001F0FCF91C4801F0F9F91C4801F0F6F94E
:1091B0001B4801F0F3F91B4801F0F0F9072C12D21B
:1091C000DFE804F0110406080A0C0E00104808E05D
:1091D000104806E0104804E0104802E0104800E0A3
:1091E000104801F019F80A4801F038F8094801F070
:1091F00035F8094801F032F8084801F02FF808481E
:1092000001F02CF8BDE81040064801F027B8000036
:10921000AC0500101C0700108C080010FC090010A1
:109220006C0B0010DC0C00100021044A016041604E
:10923000D2E90012C0E90212704700004C47010059
:1092400081684FF0E02079B1012915D002291BD0A7
:10925000032918BF70474FF48071C0F88011BFF325
:109260004F8FBFF36F8F70472021C0F88011BFF37D
:109270004F8FBFF36F8F70474021C0F88011BFF34D
:109280004F8FBFF36F8F70478021C0F88011BFF3FD
:109290004F8FBFF36F8F7047806F00280CBF012086
:1092A000002070472DE9F04184B017460E46044671
:1092B000FFF7C6FFE464A0680025002808BF334814
:1092C00053D0012808BF32484FD0022808BF314888
:1092D0004BD0032814BF25652F4846D04FF0FF30F0
:1092E000C4E93B05206D002841D02767002FCABF85
:1092F000206F0020F6F7BCFF2566A065A566A56770
:10930000C4F88050254FDFF898802046D7E9001335
:10931000CDE90013CDE902480022694601F052FB75
:109320000399684600291CBF896888476667002E34
:10933000CABF606F0020F6F79BFF6566E065E566D3
:10934000E567C4F88450D7E90213CDE90013CDE9ED
:10935000024820460122694601F034FB0399684621
:1093600000291CBF8968884704E02065B6E70DA086
:1093700003F0C2FB216D0720087284F8885004B006
:109380002046BDE8F04100F03EBA000000C00040B9
:10939000000001400080094000C009403C47010036
:1093A000C04F01004D4F4453455249414C206D750B
:1093B00073742068617665206120646566696E65F6
:1093C00064205541525420746F2066756E63746931
:1093D0006F6E2E0070B50446006F002819BFA26D95
:1093E000002A226D107D04D041B1A06F0028FCD06E
:1093F0000AE010F0010FFCD0107870BDA06F0028BB
:1094000004BF4FF0FF3070BDA06E165CA06E401C14
:10941000A066A06E216F8842A4BF0020A066A06F46
:10942000216F884209D0206D057925F00101017175
:10943000204600F085F8206D057172B6A06F401EC1
:10944000A06762B6304670BD70B50446D0F85CC007
:10945000006D0B46CDB2017DBCF1000F1CBFD4F8EE
:1094600074C0BCF1000F1ED011F0200F08D0E16FC6
:10947000002902BFD4F8EC10B1F1FF3F05705DD0B8
:10948000BAB1067901210171E06F616F884207D19D
:109490000021204600F01CF9E06F616F8842F7D090
:1094A000206D06712FE011F0200FFCD00570002018
:1094B00070BDE06F616F884225D1C4F88430D4F864
:1094C000BC1004F14C0009B1884711E0D4F8C01079
:1094D00071B1D4F8C42072B1D4F8C8C001EB6C03E8
:1094E0001CF0010F01D019688A58014618469047B0
:1094F0004FF0FF3070BDD4F8C83013F0010F18BF23
:10950000002BE9D1F4E7206D017921F0020101710E
:10951000616EE06D455472B6E06F401CE06762B664
:10952000606E401C6066606E616F8842A4BF002060
:109530006066206D017941F002010171002070BD6B
:1095400070B50446006D00281FBF216F0029A16D72
:10955000002919D0007D10F0010F14BF002570BD47
:10956000206D007884F85500A06F216F88424DD19E
:1095700094F85500C4F88000D4F8AC2004F14C01F4
:1095800042B3084690476BE0D4F88C2004F14C01BC
:109590001AB1BDE8704008461047D4F89000002882
:1095A00008BF70BDD4F8942062B100BFD4F89830E1
:1095B00000EB630013F0010F01D003689A58BDE877
:1095C00070401047D4F8983013F0010F18BF002BEB
:1095D000ECD170BDD4F8B020002A41D0D4F8B4301A
:1095E00063B100BFD4F8B80002EB600210F0010FC5
:1095F00001D01068C3581046984731E0D4F8B8003D
:1096000010F0010F18BF0028ECD129E0A06D70B157
:1096100094F85510226E8154A06F401CA067206EF4
:10962000401C2066206E216F8842A8BF256604F189
:109630004C00D4F88C1009B1884711E0D4F8901090
:1096400071B1D4F89430C3B1D4F898C001EB6C0276
:109650001CF0010F01D01168CB5801461046984705
:1096600094F8880094F85510884221D1D4F8DC1081
:1096700004F14C0049B188471AE0D4F8982012F060
:10968000010F18BF002ADFD1EAE7D4F8E01079B162
:10969000D4F8E4209AB100BFD4F8E8C001EB6C0321
:1096A0001CF0010F01D019688A58014618469047EE
:1096B000206D007D10F0010F7FF452AF70BDD4F823
:1096C000E83013F0010F18BF002BE5D1F0E70000E0
:1096D00070B50446006D0D4600281CBF606F002861
:1096E00027D0E06D002818BF002622D0E06F0028A8
:1096F0005CD0206D017D11F0200F57D0E26EE16D3E
:10970000895C84F854100170E06F401EE067E06EE1
:10971000401CE066E06E616F8142D8BFE666002DB6
:10972000E4D0D4F89C1004F14C0319B318468847D0
:10973000DCE7D4F89C2004F14C01002A42D1D4F893
:10974000A0C0BCF1000F08BF70BDD4F8A4204AB17E
:10975000D4F8A8300CEB630013F0010F45D0036878
:109760009A5842E0D4F8A80010F0010F18BF002862
:10977000EED170BDD4F8A0000028B7D0D4F8A42052
:1097800062B100BFD4F8A81000EB610011F0010F26
:1097900001D001688A5819469047A7E7D4F8A81065
:1097A00011F0010F18BF0029A0D0EBE7E06F0028EF
:1097B00018BF70BD0120216D0871D4F8CC2004F1D0
:1097C0004C011AB1BDE8704008461047D4F8D030BB
:1097D000002B08BF70BDD4F8D4204AB1D4F8D8C04B
:1097E00003EB6C001CF0010FB9D1BDE870401047CD
:1097F000D4F8D80010F0010F18BF0028EED170BDCA
:109800000121FFF765BF81684FF0E020002908BF04
:1098100020210CD0012908BF402108D0022908BF0F
:10982000802104D003290CBF4FF480717047C0F829
:109830000011704738B515464FF4165200922A466B
:1098400001F0AAFB0C4901605C3141630022C26453
:109850003C3901630623102208498C3002F016FCC3
:10986000A0F18C044FF480722B4611462046FFF77E
:1098700019FD204638BD0000C84B010029920000A8
:1098800010B50446284820605C3060633C38206393
:10989000A1684FF0E02031B101290CD0022912D08B
:1098A000032918D01FE02021C0F88011BFF34F8F8B
:1098B000BFF36F8F17E04021C0F88011BFF34F8FC7
:1098C000BFF36F8F0FE08021C0F88011BFF34F8F7F
:1098D000BFF36F8F07E04FF48071C0F88011BFF3C2
:1098E0004F8FBFF36F8FA06D002818BFF6F708FDEC
:1098F000E06D002818BFF6F703FD0C4820605C30CF
:1099000060633C38206304F1300001F0EFFB303835
:109910000446074940F80C1B022310220549F7F7BB
:1099200071F9204610BD0000C84B0100C04C010079
:10993000684C01003B3401002DE9F0470446836187
:10994000C4E90412D0F850801F4615460E4612F0A6
:10995000FF4F08BF002514D040460AF0A5FA824602
:10996000894628460AF0A0FA02460B460020144910
:1099700009F05AFE52464B460AF06CF809F066FDB3
:109980000546607890B115F0FF400ED0294630466C
:109990000AF088FC8146D4E901010AF083FC4946BB
:1099A0000AF022FBA16C0AF07DFCA064C4E9016509
:1099B000414638460AF018FBE060BDE8F087000039
:1099C0000000F03FB1F5000FB8BF70472DE9F0413E
:1099D0000D46066D0446314628460AF005FB07464B
:1099E000A1680AF05FFCA060294630460AF0FCFA44
:1099F000A16C0AF057FCA0643846E1680AF052FCFA
:109A00002565E060BDE8F081C16170472DE9F04750
:109A10000F4604461646114638460AF00FFD98BF19
:109A2000BDE8F087394630460AF044FD8046A16B18
:109A30000AF0DAFA8146616A0AF034FC606205468F
:109A40004846A16C0AF02EFCA064B5F17E5FC4BF4D
:109A50004FF07E50606204DCB5F5000FB8BF002502
:109A60006562C4F83880C4E90C76BDE8F0872DE95A
:109A7000F0410E4604461546114630460AF0DEFC1B
:109A800098BFBDE8F081314628460AF013FD07462D
:109A9000616C0AF0A9FAE16A0AF004FCE062B0F134
:109AA0007E5FC4BF4FF07E50E06204DCB0F5000F73
:109AB000B8BF0020E0626764C4E90F65BDE8F081CB
:109AC0000162704770B504460078656CE16B30B197
:109AD000E06C0AF0EFFC29460AF086FA05E0606DBA
:109AE0000AF0E8FC29460AF07FFAE062216B206A5E
:109AF0000AF0E0FCA16B0AF077FA60620020A06433
:109B000070BD2DE9F047076B0446006A39460AF03C
:109B1000D1FCA66B31460AF067FA0546B0F17E5FCC
:109B2000C8BF4FF07E5503DC15F1FF4F28BF00255D
:109B30003946E0690AF0BEFC31460AF055FAB0F148
:109B40007E5FC8BF4FF07E5003DC10F1FF4F28BF8F
:109B5000002029460AF0AEFC0646E06AB0F17E5FBE
:109B6000A8BFB6F5000F0ADAB0F5000F02DA16F159
:109B7000FF4F04D23146A06C0AF0C2F9A064284617
:109B8000616A0AF097FC216D0AF02EFA824620786D
:109B9000D4F84490D4F83C80002738B14146E06CBA
:109BA0000AF088FC49460AF01FFA07465146E06869
:109BB0000AF078FB8246A16CA0680AF073FB31467C
:109BC0000AF09EF951460AF075FC61680AF06AFBDA
:109BD00039460AF095F9A06210F1FF4F28BF002026
:109BE00005D2B0F17E5FC8BF4FF07E5000DDA062AD
:109BF00065624946E0620AF055FB4146BDE8F04720
:109C00000AF07EB9C16401210170704710B50446A5
:109C1000002908BF00201DD06078D0B92078E16B02
:109C200030B1E06C0AF046FC616C0AF0DDF905E049
:109C3000606D0AF03FFC616C0AF0D6F9E062216BBE
:109C4000206A0AF037FCA16B0AF0CEF960620020AE
:109C5000A0640120607010BD2DE9FF4F81B0002588
:109C600004464D4EDDF838A02570914628466570B3
:109C7000AB46314637460AF0E1FB20D93046A16BAE
:109C80000AF0B2F90090616A0AF00CFB606280464B
:109C90000098A16C0AF006FBA064B8F17E5FC4BF17
:109CA0004FF07E50606206DCB8F5000FB8BF4FF091
:109CB0000008C4F82480C4F830B0C4E90D76002749
:109CC000314638460AF0BAFB18D9B0463046616CC6
:109CD0000AF08AF9E16A0AF0E5FAE062B0F17E5F23
:109CE000C4BF4FF07E50E06204DCB0F5000FB8BF97
:109CF0000020E062C4F84480C4E90F76C4F850A0A4
:109D0000DDF81080029FC4F81880C4E9047919F0C6
:109D1000FF4F08BF002614D050460AF0C5F806468B
:109D20008B4648460AF0C0F802460B4600201B4905
:109D300009F07AFC32465B4609F08CFE09F086FB9E
:109D400006466078A0B116F0FF4F08BFA5640FD09B
:109D5000314638460AF0A6FA8146D4E901010AF0F4
:109D6000A1FA49460AF040F9A16C0AF09BFAA064F6
:109D7000C4E90176514640460AF036F9E5612562AC
:109D80006562A562E562A564E5646565E06005B0AD
:109D90002046BDE8F08F0000333353400000F03F11
:109DA0002DE9F04F0446C06E8FB0002849D0D4F89A
:109DB000680104F5B475816828468847281D02F0BB
:109DC000C1FD06462868C1682846884730460AF023
:109DD0006BF806908B46A06A0AF066F804908A46F3
:109DE000606A0AF061F8CDE90001206A0AF05CF8C7
:109DF0008146029160680AF057F807468846A069D4
:109E00000AF052F805460E4604F5807001F058F845
:109E10000AF04AF8069ACDE90C2B0B46216F049AFA
:109E20000968CDE9082A0A91DDE90012CDE9061298
:109E300002990246CDE904918DE8E0015148F6F718
:109E40008BFAA06E052824BF0FB0BDE8F08FDFE8C5
:109E500000F03E0345648F00A168A06C0AF022FA6E
:109E6000616D0AF04DF86065616CB1F5000F216C11
:109E700030DB0AF0E3FA01D2206C00E0606D60652F
:109E80000146A0690AF03CF8A061A06D0AF00CF848
:109E900000223D4B09F0C8FB05460E4604F58070D4
:109EA00001F00EF80AF000F82A46334609F0D0FE19
:109EB0000BD9216C606D21F0004120F000400AF0C8
:109EC000BDFA24BF0FB0BDE8F08F0220A0660FB02E
:109ED000BDE8F08F0AF0B2FAD0D3CDE7216CA069CB
:109EE0000AF00EF8A061A06D09F0DEFF4FF05532C8
:109EF000264B09F0AFFD05460E4604F5807000F0D4
:109F0000DFFF09F0D1FF2A46334609F0A1FE9CBFCE
:109F10000320A0660FB0BDE8F08FA168A06C0AF026
:109F2000C1F9616D0AF0BBFA01466065A06909F0EC
:109F3000E7FFA061606C0425B0F5000F216AE06BBB
:109F400006DB0AF07BF907D8E06BA566A06103E0A9
:109F50000AF074FA98BFA56604F5807000F0B0FFAF
:109F6000A16D0AF06BFA98BFA5660FB0BDE8F08F3F
:109F700004F1D80001F014F904F5807000F0BEFF80
:109F80000020A3E7F85D0100000008405555E53FBB
:109F900010B50446D0F8140101F02CFB20600AF043
:109FA00021F92062216B0AF085FAA1680AF07AF99A
:109FB0006062616B0AF07EFAA062A169D4F81001B8
:109FC000FFF722FD216AD4F81001FFF779FDD4F8DC
:109FD0001001FFF796FD01466060D4F88C0090B147
:109FE000D4F890000028D4F8180103D0012201F021
:109FF00067FD01E001F078FC206A2063606A60631D
:10A00000A069E06110BD002060600021D4F8180153
:10A01000F0E7000070B5044600F5B475D0F86801AB
:10A02000816828468847281D02F08CFC064628686F
:10A03000C16828468847304609F036FF4FF066323F
:10A040000E4B09F007FD0E4A0E4B09F0EDFA09F030
:10A05000FDF9606720F00040D4F884100AF0EEF9B2
:10A060003CBF606FC4F88400A16F656F28460AF09A
:10A0700021FAA567C4F88000284670BD66660A40CC
:10A08000CDCCCCCCCCCCE03F2DE9F8438265044666
:10A09000C16315460E4600680AF0A4F831460AF07E
:10A0A000FEF90746294609F09FFF80466064A068D4
:10A0B00009F0FAFE06468946404609F0F5FE002200
:10A0C0001B4B09F0C7FC4B46324609F0C3FC09F0B4
:10A0D000BDF929462064C84608460AF0E3F801465F
:10A0E000384609F081FF09F0DFFE0022114B09F02C
:10A0F000B1FC3246434609F0ADFC09F0A7F9A06473
:10A10000002060650120A06604F5807000F00FFF5C
:10A1100004F5807000F019FFA06800900648214601
:10A12000D0E9022304F1D80009F0FAF8BDE8F88379
:10A130000000F83F000012402C4701004361C0E9D5
:10A140000312D0F81001FFF7F7BB70B504460D46B7
:10A15000D0F8140101F07EF928460AF043F80146D0
:10A16000A061D4F81001BDE87040FFF74DBC0000BD
:10A1700070B50446D0F81001FFF7A4FC234A244927
:10A18000D4F81001FFF742FC4FF07E522149D4F879
:10A190001001FFF76CFC0021D4F81001FFF732FD2D
:10A1A0000121D4F81001FFF731FDA168D4F81001A6
:10A1B000FFF708FCD4F8140101F0A6FAD4F8140152
:10A1C00001F0D6F90021D4F8140101F043F900257B
:10A1D000A5612946D4F81001FFF716FCD4F8140144
:10A1E00001F008FA2060D4F81001FFF76BFCA561BC
:10A1F0000021D4F81001FFF707FCD4E903126369CA
:10A20000D4F81001BDE87040FFF796BB00D8564760
:10A2100000D856C7000080BF70B50446D0F81401BE
:10A2200001F072FAD4F8140101F0A2F90021D4F877
:10A23000140101F00FF9D4F8140101F0DBF9002545
:10A2400025622060D4F81001FFF73CFCA561D4F82A
:10A250001001BDE870400021FFF7D6BB38B50025DE
:10A2600004464560D0F81001FFF72CFCE06A28B1E5
:10A27000A5610021D4F81001FFF7C6FBD4E9031251
:10A280006369D4F81001FFF757FB0120C4F88C0074
:10A29000A068009004482146D0E9002304F1B000F2
:10A2A00009F03EF838BD00002C4701002DE9F04FC1
:10A2B0008FB0044654E0B049A06909F021FEA061C6
:10A2C000AE4808F0BFFFE06E002849D0D4F868011E
:10A2D00004F5B475816828468847281D02F032FBD2
:10A2E00006462868C16828468847304609F0DCFDE4
:10A2F00082468B46A06A09F0D7FDCDE90201606A6B
:10A3000009F0D2FDCDE90001206A09F0CDFD8146BA
:10A310000491606809F0C8FD07468846A06909F005
:10A32000C3FD05460E4604F5807000F0C9FD09F036
:10A33000BBFD0246CDE90CAB206F0B4600680A90CE
:10A34000DDE90201CDE90801DDE90001CDE9060101
:10A3500004998B48CDE904918DE8E001F5F7FCFF05
:10A36000206F0068012808D04FF07C5008F06AFF89
:10A37000206F0068002836D08CE0D4F8680104F51E
:10A38000B475816828468847281D02F0DBFA064626
:10A390002868C16828468847304609F085FD4FF097
:10A3A0006632784B09F056FB774A784B09F03CF956
:10A3B00009F04CF8606720F00040D4F884100AF0EF
:10A3C0003DF83CBF616FC4F88410A16F606F0AF064
:10A3D00071F8C4F88000616FA1670846E16F09F069
:10A3E0002DFFC1D267E76A49A0690AF063F8A0614E
:10A3F000684808F027FFE06E002847D0D4F86801CD
:10A4000004F5B475816828468847281D02F09AFA39
:10A4100006462868C16828468847304609F044FD4A
:10A4200001910490A06A09F03FFD00910290606ADA
:10A4300009F03AFD82460391206A09F035FD814614
:10A440008B46606809F030FD07468846A06909F030
:10A450002BFD05460E4604F5807000F031FD09F035
:10A4600023FD0B46019A0499CDE90C12216F09686E
:10A470000A91009A0299CDE9081203990246CDE9A2
:10A4800006A18DE8E00B3E48F5F766FF206F0068F7
:10A490000028A8D0D4F8140101F036F9D4F814013A
:10A4A00001F066F80021D4F8140100F0D3FFD4F8CD
:10A4B000140101F09FF8002525622060D4F81001F6
:10A4C000FFF700FBA5610021D4F81001FFF79CFA0B
:10A4D000E06E002804BF0FB0BDE8F08F04F5B4753E
:10A4E000D4F86801816828468847281D02F02AFAB6
:10A4F00006462868C16828468847304609F0D4FCDB
:10A5000082468B46A06A09F0CFFCCDE90201606A61
:10A5100009F0CAFCCDE90001206A09F0C5FC8146BA
:10A520000491606809F0C0FC07468846A06909F0FC
:10A53000BBFC05460E4604F5807000F0C1FC09F036
:10A54000B3FC8C46CDE90CAB216F09680A91DDE9BB
:10A550000213CDE90813DDE90012CDE906120499D2
:10A560000246CDE904918DE8E00163460A48F5F71B
:10A57000F3FE0FB0BDE8F08F0000C842CDCC4C3DDB
:10A58000F85D010066660A40CDCCCCCCCCCCE03F77
:10A5900000002041CDCCCC3DA85D010000214160F0
:10A5A000C0F88C10B03000F0FBBD00002DE9FF4F6B
:10A5B00081B09846DDE90E790E46B030DDF840A056
:10A5C00000F096FA00258A4C45620460283000F0BD
:10A5D0008FFA45620460283000F0C7FCA0F5807453
:10A5E000844940F81C1F71684160B1688160F1685E
:10A5F000C160316901610399C4F83051C4F8345124
:10A60000C4F83851C4F83C51C4F8405104F598706E
:10A61000C4F8445102F0A4FB04F5A47B02F0FAF95B
:10A620004146584607F08AFF02F03AFAC4F8505102
:10A63000C4F85451C4F85851C4F85C51C4F860517E
:10A6400004F5A8703946C4F8645102F089FBCDF8CE
:10A650000090DFF8A8916848C4F86801D9F80000B4
:10A6600004F5B47B002804BF09F10400C9F8000018
:10A6700009F10409484504D059226149614807F0AD
:10A680004BFD0BF10400009902F010F95B480168E2
:10A69000002904BF011D0160494504D059225849D1
:10A6A000584807F039FD5BF8380DB0F1FF3F04D191
:10A6B0002422554955A007F02FFDDBF80C10DBF8DC
:10A6C0000400086004F5A47B4FF0000902F0A2F931
:10A6D0004946584607F0CEFF02F0E2F9D4F850019F
:10A6E00004F5A879B0F1FF3F04D12422464947A0E0
:10A6F00007F012FDD9F81010D9F8040008604A4894
:10A7000048496560C4E902104848C4E90405A561E8
:10A71000E56125624FF0FF306562C4E90A50E563E8
:10A72000256443486564C4E91250E56541482566DF
:10A73000C4E91405A56525606566A566E5663E481D
:10A7400000912146D0E9002304F1B00008F0E8FDB3
:10A750003A48C4F88C50C4E91F056567A567C4F87A
:10A760008450C4F888507220C4F8905084F8940043
:10A77000582001F041FC30B1A168002300911A4635
:10A780001946FFF769FAC4F81001302001F034FCD3
:10A7900018B13146039A01F075F8C4F814013C2051
:10A7A00001F02AFC18B13A46414601F005FBC4F815
:10A7B00070A0C4F81801D4F8140100F0A5FFD4F873
:10A7C000140100F0D5FE0021D4F8140100F042FE7F
:10A7D000A5612946D4F81001FFF716F9D4F8140141
:10A7E00000F008FF206005B02046BDE8F08F0000B3
:10A7F000784D0100A44C01008C4D01007001001047
:10A80000044E0100F04D0100645D01006F626A2D8D
:10A810003E70696E20213D202850696E4E616D6545
:10A82000294E43000AD7233C0000E1430000D242F6
:10A830000000D841000040412C4701003333B33EB3
:10A8400070B5114D00F1D804C0F8D850204600F082
:10A85000A7FC616A04F1180000291CBF89688847B9
:10A86000204600F059F928380446056000F098FCAD
:10A87000616A04F1180000291CBF896888472046D6
:10A8800000F04AF9B03870BD784D010070B504464B
:10A890000068416A20468847206801220021036938
:10A8A000204698470546B0F1FF3F206811D00222AC
:10A8B0000369002120469847064620680022294661
:10A8C0000369204698472068816A204688473046B9
:10A8D00070BD816A204688474FF0FF3070BD7047D9
:10A8E0007047000070B50546174C16482860206870
:10A8F000002804BF201D2060261DB04204D059222C
:10A900001249134807F008FC00211248D4F800301F
:10A9100010228C4650F82140AC4208BF40F821C0BC
:10A92000491C521EF6D10849002B12BF0868081DA9
:10A930000860B04204D059220449054807F0ECFBF6
:10A94000284670BD344C010050010010044E010037
:10A95000F04D0100A80F0010001D07F0A3BF10B5B7
:10A960000C46001D08F000F9204610BD10B500EBA4
:10A97000011000F10C04806928B940F2E712054982
:10A98000054807F0C9FBE06801682046BDE81040B3
:10A99000084700008B5101008651010070B5044644
:10A9A00000680D460168204688472946201D07F0AB
:10A9B00097FEE562206841682046BDE87040084780
:10A9C000704700002DE9F041054600680F46164625
:10A9D00001682846884702F01DF805EB0610F96863
:10A9E00000F10C0499B1E168204600291CBF896878
:10A9F0008847F86818B14268394620469047F86899
:10AA0000E06001223146281D08F036F80EE0E168CA
:10AA10000A4F204600291CBF8968884708482760DC
:10AA2000E06000223146281D08F026F802F038F8D0
:10AA3000286841682846BDE8F041084753B4000043
:10AA4000CC4F0100704700002DE9F0478A461B49B2
:10AA500040F8041B002140F8041B1C46914640F8B6
:10AA6000041B02231022164901F010FBDFF854806A
:10AA7000A0F10C050026046205EB061000F10C04A1
:10AA8000114FE168204600291CBF89688847761C61
:10AA9000C4F80C802760022EEED34A465146281D8A
:10AAA00007F01CFF281DE96A07F01AFE2A4607492D
:10AAB000281D07F0D3FF2846BDE8F087684C010049
:10AAC000D13F0000CC4F010053B400006DA900003D
:10AAD0000168896808470A46D0F810C00346011D7E
:10AAE000604608F058BA0269011D104608F0A1BA84
:10AAF00010B504460648206000206060A060E06059
:10AB000002F0CEF80349206108F0B5FA204610BDE6
:10AB1000804C0100D1AA000010B504460348206013
:10AB2000211D206908F085FA204610BD804C0100E7
:10AB300010B5002908BF10BD01290CD0022918BF8B
:10AB400010BD00F13804406C50B1E0680168204647
:10AB5000BDE81040084700F12804406B0028F4D1FC
:10AB600040F2E7120249034807F0D6FAEDE7000089
:10AB70008B5101008651010070B50D46064601F06B
:10AB800049FFE86806F13804A8B1E16820460029C9
:10AB90001CBF896888473CB1E86818B142682946FB
:10ABA00020469047E868E0600122022106F11C007F
:10ABB00002F086F910E0E168094D204600291CBF2B
:10ABC0008968884714B107482560E06000220221A7
:10ABD00006F11C0002F074F9BDE8704001F060BF9E
:10ABE00051B40000CC4F010070B50D46064601F08F
:10ABF00011FFE86806F12804A8B1E16820460029A1
:10AC00001CBF896888473CB1E86818B1426829468A
:10AC100020469047E868E0600122114606F11C00DA
:10AC200002F04EF910E0E168094D204600291CBFF2
:10AC30008968884714B107482560E0600022012137
:10AC400006F11C0002F03CF9BDE8704001F028BF9D
:10AC500051B40000CC4F010070B504461448206088
:10AC600000206060A060E06020616061A061E06140
:10AC7000206260620D46606360640E4A0E4914F102
:10AC800028001CBF0260C16014F13800094A1CBFD3
:10AC90000260C1602346094A294604F11C0002F003
:10ACA000BFF82946201D02F046F8204670BD00007E
:10ACB000944C010051B40000CC4F010031AB0000B6
:10ACC00010B504460A48206004F11C0002F0A0F808
:10ACD000606C383410B181682046884754F8040C01
:10ACE000103C10B1816820468847A4F1280010BDAF
:10ACF000944C01000021F5F70FBE000007480168E1
:10AD0000002904BF011D0160001D814208BF70477A
:10AD100059220349034807F0FFB900007C010010E5
:10AD2000044E0100F04D010070B5044600680E4667
:10AD300041682046884720684168204688470F4D73
:10AD40002868A0420AD0D4E902120023201D07F08F
:10AD5000C5FF201D216908F021F82C60206881685A
:10AD6000204688473146201D08F008F9054620682E
:10AD7000816820468847284670BD00007801001091
:10AD800070B5044600680D4616464168204688475F
:10AD9000C4E902560F4D0020286020684168204613
:10ADA00088472868A0420AD0D4E902120023201D57
:10ADB00007F094FF201D216907F0F0FF2C60206848
:10ADC000816820468847206881682046BDE8704039
:10ADD000084700007801001007480168002904BFF7
:10ADE000011D0160001D814208BF704759220349BF
:10ADF000034807F091B900007C010010044E0100E7
:10AE0000F04D010070B5044600680D4641682046CB
:10AE1000884725610F4D0020286020684168204642
:10AE200088472868A0420AD0D4E902120023201DD6
:10AE300007F054FF201D216907F0B0FF2C60206847
:10AE4000816820468847206881682046BDE87040B8
:10AE5000084700007801001038B504461448DDF8B2
:10AE600010C0206000200825C4E90105E0601148F9
:10AE70002061201DCDF800C008F00CF82068416862
:10AE8000204688470C4D2868A0420AD0D4E9021217
:10AE90000023201D07F022FF201D216907F07EFFFF
:10AEA0002C602068816820468847204638BD000015
:10AEB000A44C010040420F007801001070470000D0
:10AEC00070B5044601F0A6FD01F0A4FD2068002540
:10AED00020B1E06808F0AAF86168451A01F0E0FDC9
:10AEE000A0682C1801F0DCFD204609F07BF9BDE8D4
:10AEF0007040014909F078B80024744970B50446DF
:10AF000001F088FD01F086FD2068002520B1E06891
:10AF100008F08CF86168451A01F0C2FDA068284469
:10AF2000A06000202060BDE8704001F0B9BD10B500
:10AF3000044601F06FFDE06808F078F860600020DA
:10AF4000A060BDE8104001F0ABBD10B5044601F0B3
:10AF500061FD206828B9E06808F068F860600120A9
:10AF60002060BDE8104001F09BBD70B50025056074
:10AF700045600446856001F093FEE06001F04AFD03
:10AF8000E06808F053F8C4E9010501F089FD2046A6
:10AF900070BD70477047000010B51C46029BFFF75C
:10AFA00053FD2146303000F081F8044940F8301D4F
:10AFB0005C3141633C39016310BD0000C04C0100AD
:10AFC000002070472DE9F041054600680F460C4609
:10AFD0008E18416A28468847B4420AD02868026B16
:10AFE00028469047B0F1FF3F03D004F8010BB4426C
:10AFF000F4D12868816A28468847E01BBDE8F081C3
:10B0000000207047002070470FB470B504460068F8
:10B01000416A2046884706AD6069F5F7F0FB2A468D
:10B0200060690599F5F704FB05462068816A2046AA
:10B030008847284670BC5DF814FB2DE9F0410546B1
:10B0400000680F460C468E18416A28468847B4426D
:10B050000AD0286814F8011BC26A28469047B0F14C
:10B06000FF3F18BFB442F4D12868816A2846884758
:10B07000E01BBDE8F081002070470FB470B50446B6
:10B080000068416A2046884706AD6069F5F7B7FB5E
:10B090002A4660690599F5F75AF905462068816ADC
:10B0A00020468847284670BC5DF814FB10B584B074
:10B0B00000F066F904460A4820603C3060600020D9
:10B0C0006061224607A16846F5F752F906A1684675
:10B0D000F5F7FBFB6061FFF70DFE04B0204610BDE5
:10B0E0002C4D01003A257000772B000010B5044666
:10B0F000054820603C3060606069F5F717FC204629
:10B10000BDE8104000F04EB92C4D010070B50D4661
:10B11000044601F07FFC2046FFF7E5FC65612069ED
:10B1200007F084FF616901442046FFF7D4FCBDE8C5
:10B13000704001F0B5BC0000F0B5064685B0C868A7
:10B1400017466D460C4610B1426828469047E068A5
:10B1500003901249384609F0A5F809F023F8716AFE
:10B16000074606F11804204600291CBF8968884755
:10B170003CB12946039810B1426820469047039895
:10B18000E06039463046FFF7C1FF03996846002961
:10B190001CBF8968884705B0F0BD000000247449D1
:10B1A00010B5044601F036FC2046FFF79CFC18342D
:10B1B0002046E16800291CBF89688847002C1CBF15
:10B1C0000020E060BDE8104001F06ABC10B5044604
:10B1D0004068616901442046FFF77DFC606A1834CD
:10B1E00028B940F2E7120549054806F095FFE068E6
:10B1F00001682046BDE81040084700008B5101005F
:10B200008651010010B50446084820602046FFF72B
:10B21000C7FF606A183410B1816820468847A4F1DE
:10B220001800BDE81040FFF777BC0000784D010022
:10B2300007480168002904BF011D0160001D81420B
:10B2400008BF704759220349034806F065BF000054
:10B2500070010010044E0100F04D01000748016824
:10B26000002904BF011D0160001D814208BF704715
:10B2700059220349034806F04FBF00007001001037
:10B28000044E0100F04D0100007B704770B506468A
:10B290000D46154808F02EF814480468F4B1A0686B
:10B2A000C8B12A463146F5F7AAFBA0B9A068F5F760
:10B2B00087FBA8420FD10C480168002904BF011D7B
:10B2C0000160001D814204D059220949094806F055
:10B2D00023FF204670BD6468002CE0D1024808F0CE
:10B2E00009F8002070BD00009801001094010010C2
:10B2F000044E0100F04D010070B504460B480026D5
:10B30000A160C4E900060D462273094807F0F2FF68
:10B31000002D08BF666003D00648016861600460C4
:10B32000034807F0E7FF204670BD0000A44D010070
:10B33000980100109401001010B504460D482060DB
:10B340000D4807F0D7FFA06878B10C490868A04203
:10B3500004BF6068086008D04168A14203D0084675
:10B360004968A142FBD161684160034807F0C2FF10
:10B37000204610BDA44D010098010010940100105A
:10B3800010B5064A40F8042B0022FFF7B5FF044928
:10B3900040F8041D3431416010BD0000344C010000
:10B3A000B44D010010B5001DFFF7C6FFBDE8104009
:10B3B000001FFFF797BA10B50446406828B1FFF7A1
:10B3C00063FF012804BF606810BD002010BD10B5E8
:10B3D0000446406810B1FFF757FF08B1002010BDC8
:10B3E0006068002818BF001F10BD4068002818BF03
:10B3F0000120704710B54068002808BF10BDFFF756
:10B4000043FF00280CBF0120002010BD00687047DA
:10B4100010B5044600202060606008782F280DD108
:10B42000487858B14B1C00212360226810782F28DF
:10B4300006D038B1501C491C2060F6E7204610BDEC
:10B44000501C20601846FFF721FF6060204610BDA9
:10B45000704770472DE9F0410D460446002208214F
:10B46000001DFFF78DFC3A4F201D3946FFF7CAFC3F
:10B47000A06904F11806B0F1FF3F04D12422354938
:10B4800035A006F049FE316970680860012007F0B8
:10B49000F9FE00220821201DFFF772FC3E463946C6
:10B4A000201DFFF7AFFC9821201DFFF73DFC290E62
:10B4B000201DFFF739FCC5F30741201DFFF734FCC1
:10B4C000C5F30721201DFFF72FFCE9B2201DFFF770
:10B4D0002BFCA06904F11805B0F1FF3F04D1242230
:10B4E0001C491DA006F018FEE96868680860012084
:10B4F00007F0C8FEA06904F11805B0F1FF3F04D1C0
:10B500002422144914A006F007FE2969686808601F
:10B51000012007F0B7FE00220821201DFFF730FCB4
:10B520003146201DFFF76EFCE021201DFFF7FCFBDC
:10B5300054F8180FB0F1FF3F04D12422054906A0AA
:10B5400006F0EAFDE16860680860BDE8F08100008F
:10B5500080841E00645D01006F626A2D3E70696E1A
:10B5600020213D202850696E4E616D65294E4300B3
:10B5700070B5044600220821001DFFF701FC1A4E99
:10B58000201D3146FFF73EFCA06904F11805B0F11B
:10B59000FF3F04D124221549154806F0BDFD296955
:10B5A00068680860012007F06DFE00220821201D58
:10B5B000FFF7E6FB3146201DFFF724FC8821201D04
:10B5C000FFF7B2FB0321201DFFF7AEFB54F8180F65
:10B5D000B0F1FF3F04D124220449054806F09CFD48
:10B5E000E1686068086070BD80841E00645D0100D1
:10B5F00058B500002DE9F041044600220821001D45
:10B60000FFF7BEFB3D4F201D3946FFF7FBFBA0694E
:10B6100004F11806B0F1FF3F04D12422384939481B
:10B6200006F07AFD316970680860012007F02AFE93
:10B6300000220821201DFFF7A3FB3946201DFFF73C
:10B64000E1FBE821201DFFF76FFBA06904F118065C
:10B65000B0F1FF3F04D1242229492A4806F05CFDBD
:10B66000F16870680860012007F00CFEA06904F121
:10B670001806B0F1FF3F04D124222149214806F0E9
:10B680004BFD316970680860012007F0FBFD002266
:10B690000821201DFFF774FB3946201DFFF7B2FB80
:10B6A0006021201DFFF740FB0021201DFFF73CFB20
:10B6B00060F31F650021201DFFF736FB60F317457F
:10B6C0000021201DFFF730FB60F30F250021201D16
:10B6D000FFF72AFB60F30705A06904F11806B0F133
:10B6E000FF3F04D124220649064806F015FDF16803
:10B6F0007068086028462560BDE8F08180841E00DF
:10B70000645D010058B5000070B5044600220821B0
:10B71000001DFFF735FB304E201D3146FFF772FB51
:10B72000A06904F11805B0F1FF3F04D124222B4990
:10B730002B4806F0F1FC296968680860012007F0D1
:10B74000A1FD00220821201DFFF71AFB3146201D14
:10B75000FFF758FB2021201DFFF7E6FAA06904F14E
:10B760001805B0F1FF3F04D124221C491C4806F003
:10B77000D3FCE96868680860012007F083FDA069D0
:10B7800004F11805B0F1FF3F04D1242213491448F5
:10B7900006F0C2FC296968680860012007F072FDA4
:10B7A00000220821201DFFF7EBFA3146201DFFF78C
:10B7B00029FBE021201DFFF7B7FA54F8180FB0F16C
:10B7C000FF3F04D124220549054806F0A5FCE168A5
:10B7D0006068086070BD000080841E00645D010028
:10B7E00058B5000070B5244E04463146001DFFF7E1
:10B7F00009FB2046FFF788FF00220821201DFFF7E4
:10B80000BFFA3146201DFFF7FDFAA06904F11805C3
:10B81000B0F1FF3F04D124221849194806F07CFCFE
:10B82000296968680860012007F02CFD2546002280
:10B830000821201DFFF7A4FA3146281DFFF7E2FA80
:10B840008821281DFFF770FA0321201DFFF76CFAED
:10B85000A0691835B0F1FF3F04D1242207490848F8
:10B8600006F05AFCE968686808602046BDE8704048
:10B870000021FFF7EFBD000080841E00645D010021
:10B8800058B5000070B50446144B40F8043F4B68AF
:10B8900043608B688360CB68C360096901611146AE
:10B8A0000022A261E26122626262A26204F11800D7
:10B8B000E26201F055FAA06904F11805B0F1FF3F0A
:10B8C00004D124220649074806F026FCE968686886
:10B8D00008602046FFF786FF204670BDA44C01009B
:10B8E000645D010058B5000070B50D460446B1F125
:10B8F0007E5FC8BF4FF07E5503DC15F1814F88BFD6
:10B900006A4D62786A486B49002A00F086808D4251
:10B9100026DBE06804F10C06B0F1FF3F04D12422DD
:10B920006549664806F0F8FB316970680860606A2E
:10B9300004F12406B0F1FF3F04D124225E495F48A0
:10B9400006F0EAFBF16870680860241D01F062F8F7
:10B950002946204606F08EFEBDE8704001F0A0B8F2
:10B96000854219D9606A04F12406B0F1FF3F04D181
:10B9700024225149514806F0CFFB316970680860B4
:10B98000E06804F10C06B0F1FF3F69D124224A4976
:10B990004A4806F0C1FB63E0207804F10C0500285A
:10B9A000E06800F1010023D020B924224249434835
:10B9B00006F0B2FB296968680860606A04F1240532
:10B9C000B0F1FF3F04D124223B493C4806F0A4FBE0
:10B9D000296968680860251D4FF07E5401F01AF847
:10B9E0002146284606F046FEBDE8704001F058B8F2
:10B9F00020B924223049314806F08EFB2969686855
:10BA00000860606A04F12405B0F1FF3F3ED12422B2
:10BA100029492A4806F080FB38E08D4218DBE068AF
:10BA200004F10C06B0F1FF3F04D12422224923483F
:10BA300006F072FB316970680860241D00F0EAFFAF
:10BA40002946204606F016FEBDE8704001F028B8F1
:10BA5000854215D9E06804F10C06B0F1FF3F95D09E
:10BA6000F1687068086025F00045241D00F0D2FFE1
:10BA70002946204606F0FEFDBDE8704001F010B8F2
:10BA8000E06804F10C05B0F1FF3FC0D02969686897
:10BA90000860251D002400F0BDFF2146284606F061
:10BAA000E9FDBDE8704000F0FBBF0000000080BF72
:10BAB0006F1283BA6F12833A645D010050BE0000BA
:10BAC00070B50D460446B1F17E5FC8BF4FF07E559C
:10BAD00003DC15F1814F88BFB24D6378B248B3499A
:10BAE000002B00F0D98052B18D42C0F28780606A8D
:10BAF00004F12406B0F1FF3F40F076806FE08D4204
:10BB00001BDBE06804F10C06B0F1FF3F04D12422F6
:10BB1000A749A84806F000FB316970680860606AB0
:10BB200004F12406B0F1FF3F40F0C0802422A04978
:10BB3000A04806F0F1FA00F0B9B885421BD9606A56
:10BB400004F12406B0F1FF3F04D12422984999481A
:10BB500006F0E2FA316970680860E06804F10C06EA
:10BB6000B0F1FF3F40F0D48024229149914806F083
:10BB7000D3FA00F0CDB8207804F10C050028E06875
:10BB800000F1010014D020B924228949894806F027
:10BB9000C3FA296968680860606A04F12405B0F195
:10BBA000FF3F59D124228249824806F0B5FA53E07A
:10BBB00020B924227E497F4806F0AEFA29696868D8
:10BBC0000860606A04F12405B0F1FF3F40F0DB80BB
:10BBD00024227749774806F09FFA00F0D4B824224F
:10BBE0007349744806F098FA316970680860E06833
:10BBF00004F10C06B0F1FF3F58D197E7854214D904
:10BC0000E06804F10C06B0F1FF3F04D1242268493A
:10BC1000684806F081FA316970680860606A04F16A
:10BC20002406B0F1FF3F73D19EE7207804F10C05A4
:10BC30000028E06800F101001ED020B924225C49F0
:10BC40005C4806F069FA296968680860606A04F16E
:10BC50002405B0F1FF3FA5D0296968680860251D5B
:10BC60004FF07E5400F0D6FE2146284606F002FD35
:10BC7000BDE8704000F014BF20B924224C494D4863
:10BC800006F04AFA296968680860606A04F12405C8
:10BC9000B0F1FF3F77D19BE7B2B18D424FDBE06857
:10BCA00004F10C06B0F1FF3F3FF440AFF16870685B
:10BCB0000860241D00F0AEFE2946204606F0DAFC9E
:10BCC000BDE8704000F0ECBE8D4218DBE06804F186
:10BCD0000C06B0F1FF3F04D124223549354806F067
:10BCE0001BFA316970680860241D00F093FE294634
:10BCF000204606F0BFFCBDE8704000F0D1BE854292
:10BD000016D9E06804F10C06B0F1FF3F3FF42CAF08
:10BD1000F1687068086025F00045241D00F07AFE87
:10BD20002946204606F0A6FCBDE8704000F0B8BEEB
:10BD3000E06804F10C05B0F1FF3F24D148E78542EB
:10BD40001AD9E06804F10C06B0F1FF3F04D12422B7
:10BD50001749184806F0E0F931697068086025F065
:10BD60000045241D00F056FE2946204606F082FCC0
:10BD7000BDE8704000F094BEE06804F10C05B0F13D
:10BD8000FF3F3FF425AF296968680860251D00243E
:10BD900000F040FE2146284606F06CFCBDE87040ED
:10BDA00000F07EBE000080BF6F1283BA6F12833A2C
:10BDB000645D010050BE00002DE9F04116460446C6
:10BDC000071D0D4600F026FE2946384606F0B6FB54
:10BDD00000F066FE0025E56025616561A561E5610D
:10BDE00004F10C003146256200F0BAFF6562A562DD
:10BDF000E5622563656304F12400691EA56300F014
:10BE0000AFFF6570271D322600F004FE314638462C
:10BE100006F014FC00F044FE261D00F0FBFD294650
:10BE2000304606F027FC00F03BFEE06804F10C050C
:10BE3000B0F1FF3F04D12422044905A006F06CF9BB
:10BE40002969686808602046BDE8F081645D0100EA
:10BE50006F626A2D3E70696E20213D202850696E08
:10BE60004E616D65294E43002DE9F0410F48006A8F
:10BE700008F07CF907F09BFD0D4604460C4A0D4B7B
:10BE800007F0E8FD06460F46204629460A4A0B4BB6
:10BE900007F0E0FD22462B4607F0DCFD32463B462C
:10BEA00007F006FBBDE8F04107F0D0BADC0C00104B
:10BEB0003BDF4F8D976E923F8DEDB5A0F7C6A0BECC
:10BEC00010B50446806A134908F01AF8A062E06AC7
:10BED0000A30E062B0F57A7F18BF10BD0020E06242
:10BEE000216B491C21633C2918BF10BD2063616B85
:10BEF000491C61633C2918BF10BD6063A16B491CDC
:10BF0000A163182918BF10BDA063E06B401CE0635B
:10BF100010BD000000002041F0B589B0FEF7E8FD3B
:10BF200004461F48206000206062E0622063606376
:10BF3000A063E0631B4804AED0E90010CDE9001017
:10BF400019486946CDE90240426830469047039857
:10BF50000790616A04F1180542F21077284600291B
:10BF60001CBF896888473DB13146079810B14268C7
:10BF7000284690470798E86039462046FFF7C6F8FC
:10BF8000079904A800291CBF896888476846039957
:10BF900000291CBF89688847204609B0F0BD000011
:10BFA000784D010054470100B44F010010B504461C
:10BFB000084820602046FFF7F3F8616A04F1180092
:10BFC00000291CBF896888472046BDE81040FEF75D
:10BFD000A3BD0000784D010001213038FDF7FAB90A
:10BFE00001223038FDF730BA70473038FEF7B4BC64
:10BFF0003038FEF7B4BC704710B5F4F739F90400D7
:10C0000004BF02A000F078FD204610BD4F7065729D
:10C0100061746F72206E6577206F7574206F662073
:10C020006D656D6F72790D0A00000000490050EADD
:10C03000C12018BF04204A0D18BF40F0010040F293
:10C04000FF72B2EB515F08BF40F00200012808BF49
:10C05000052070472DE9F0410A4D0E4607462C6831
:10C060002868B0F1805F07D221466C06C4222046C2
:10C07000F4F71CFD2046286004EB87000664BDE849
:10C08000F081000008ED00E0012070472DE9F0414B
:10C090001C4617460E00804607D0054602E028469B
:10C0A000B0473D442046641EF9D24046BDE8F081C9
:10C0B0000020F6F7CBBA40F2013200204FF0E04109
:10C0C00008F0A3BA024A0020110708F09EBA000047
:10C0D00001FDFFFF10B50446D1E9000100F002F8B0
:10C0E000206010BDF8B504460D466A4600F0ACFD70
:10C0F00000987E30009000281FDC00221346204666
:10C10000294607F0E9FB18D0002140F608004FF05F
:10C11000000006462046294607F098F9044640F6F6
:10C12000080006EA00014FF0000034F0004004BFB0
:10C130000220F7F76CF82046F8BD0098FF280DDBC9
:10C140000220F7F764F8002213462046294607F03C
:10C150007FFD8CBF04484FF0FF40F8BD20462946C4
:10C16000BDE8F84007F072B9000080FF2DE9F04704
:10C17000A94884B00024046044608460C460046101
:10C18000A6490122446100F00FFEA548A5490122FD
:10C19000046044608460C4600461446100F004FE93
:10C1A000A148A2490122046044608460C460046123
:10C1B000446100F0F9FD9E489E490460446084603B
:10C1C000C4600461446100F0CBFD9B4A0023511E12
:10C1D0009A48FDF72FFB9A4A9A49FFF755FF9A4B69
:10C1E000601E5A1C0090511C9848FEF735FE944A78
:10C1F0009749FFF749FF9748974D04604460846072
:10C20000C46004612946446100F095FD93486E1EA8
:10C210003146046044608460C4600461446100F09D
:10C220008AFD8F48AF1E3946046044608460C46054
:10C230000461446100F07FFD8A48A5F1030841468E
:10C24000046044608460C4600461446100F073FD74
:10C250008548A5F104094946046044608460C460CF
:10C260000461446100F067FD8048A5F1050A51466C
:10C27000046044608460C4600461446100F05BFD5C
:10C2800029467B48FEF7E8FC6D4A7A49FFF7FCFE39
:10C2900031467948FEF7E0FC694A7649FFF7F4FE3B
:10C2A00039467648FEF7D8FC654A7249FFF7ECFE3E
:10C2B00041467348FEF7D0FC614A6E49FFF7E4FE41
:10C2C00049467048FEF7C8FC5D4A6A49FFF7DCFE44
:10C2D00051466D48FEF7C0FC594A6649FFF7D4FE47
:10C2E0006A48FEF742FE6A48FFF716FE544A69495B
:10C2F000FFF7CAFE684A6948691C0090CDE901123F
:10C300005249674B674A01F52970FEF74FF94C4ACD
:10C310006549FFF7B9FE654A6548A91C0090CDE95B
:10C3200001124A49634B644A01F21440FEF73EF998
:10C33000434A5D49FFF7A8FE604A6148E91C009046
:10C34000CDE9011241495F4B5F4A01F28450FEF78B
:10C350002DF93B4A5449FFF797FE5C4A5C48291D7A
:10C360000090CDE901125B4B3849DA1F01F2F4600D
:10C37000FEF71CF9324A4C49FFF786FE564A5749E8
:10C3800057480090CDE90112CB1C8A1E2F4901F6B7
:10C390006400FEF70BF92A4A4349FFF775FE514A3C
:10C3A000514952480090CDE901124B1C8A1E274981
:10C3B00001F6D410FEF7FAF8214A3B49FFF764FE74
:10C3C0004B484C4981600C304B4981600C30816096
:10C3D0004A484B490160001D01604A48FEF788FB4E
:10C3E000494D0560164A49494462FFF74DFE4848E9
:10C3F000FEF77EFB0560124A44494462FFF744FEA3
:10C400004448FEF775FB0560446204B00C4ABDE881
:10C41000F0473E49FFF738BEB401001032C0092092
:10C42000CC01001033C00920E401001034C0092001
:10C43000FC0100109CC0092003C009201402001058
:10C44000000000008198000007C0092008030010C8
:10C45000BDAE00001C03001016C0092034030010FC
:10C460004C030010640300107C03001094030010C0
:10C47000AC030010C1AC0000F40300103C04001039
:10C4800084040010CC040010140500105C0500109A
:10C490006C050010ADBF0000F400001020C00920A2
:10C4A00045C0092038C0092041A80000F80000104C
:10C4B00021C0092044C0092039C00920FC00001017
:10C4C00024C0092043C009203AC0092000010010FF
:10C4D00028C0092042C00920040100103EC00920E4
:10C4E00029C00920080100103FC009202AC00920E6
:10C4F0004C0E0010D5380D43BCF4E142240100106D
:10C500004F2FDF41700E0010784D010005B2000082
:10C51000980E0010C00E001010B504460A46D4E96B
:10C520000003194600F0ACFDC4E9000110BD000095
:10C5300002486A4620F0070070470000CB12001046
:10C5400030380A2801D2012070470020704710B50A
:10C5500005F0F3FE10BD00000328BCBF00207047AB
:10C560000749002201EB800151F80C0C41F80C2C1A
:10C57000002804BF4FF0FF30704701684968084742
:10C58000A80F00100328BCBF00207047064901EB2C
:10C59000800050F80C0C002804BF4FF0FF307047AB
:10C5A0000168896908470000A80F00100328BCBF74
:10C5B00001207047064901EB800050F80C0C002860
:10C5C00004BF4FF0FF3070470168C968084700009A
:10C5D000A80F00102DE9F0430E4683B081466B4949
:10C5E000F4F7BEFA6B4D6A4C6F1E20B36A49484699
:10C5F000F4F7B6FA00282ED068494846F4F7B0FAA6
:10C60000002838D0664C2068002804BF201D206018
:10C61000251DA84204D059226249634805F07CFDDB
:10C620002168624F002400BF57F8240098B3641CAF
:10C63000102CF9D332E0206848B92A4639465C48C4
:10C6400006F04CF94FF41651594806F049F803B07A
:10C650000020BDE8F083206848B92A46394654488E
:10C6600006F03CF94FF41651514806F039F803B082
:10C670000120BDE8F083206848B92A4639464C4875
:10C6800006F02CF94FF41651494806F029F803B08A
:10C690000220BDE8F083FFE7102C11D340480029A9
:10C6A00004BF011D01600068A84204D059223D4921
:10C6B0003D4805F031FD03B04FF0FF30BDE8F08399
:10C6C0004FF0FF3047F824003548002904BF011D12
:10C6D00001600068A84204D059223249324805F06E
:10C6E0001BFD99F800004FF000083A2810D0494689
:10C6F0006846FEF78DFE6846FEF777FEA0B36846F3
:10C70000FEF778FE0028684609D0FEF760FE23E0B9
:10C710006A4628A14846F3F793FF00981CE0FEF70D
:10C720004AFE08B316F0020F18BF022523D000BF3F
:10C7300016F00C0F18BF45F4007516F0040F18BF63
:10C7400045F4806506466846FEF760FE014630689F
:10C750002A4683683046984700281FBF47F82400C0
:10C76000E01C03B0BDE8F08347F8248003B04FF02D
:10C77000FF30BDE8F08316F0040F18BF0125D7D1B4
:10C7800016F0080F14BF09250025D1E77C480100E9
:10C790005801001003C00920834801008B480100A4
:10C7A00050010010044E0100F04D0100A80F0010D0
:10C7B000600100103A25700070B514460D4603283C
:10C7C00012DA1148006848B9104A1148511E06F0A3
:10C7D00085F84FF416510E4805F082FF0C4806F01C
:10C7E00061F8287001200DE00A4901EB800050F843
:10C7F0000C0C002804BF4FF0FF3070BD01688B683F
:10C8000029469847201A70BD5801001003C009201E
:10C8100060010010A80F00100328BCBF0020704763
:10C82000064A02EB800050F80C0C002804BF4FF0C1
:10C83000FF3070470268136900221847A80F0010E4
:10C8400070B514460E46032818DA1448006848B933
:10C85000134A1448511E06F041F84FF4165111487E
:10C8600005F03EFF0025002C06D9715D0D4806F04D
:10C870007BF96D1CAC42F8D820460DE00A4901EB6B
:10C88000800050F80C0C002804BF4FF0FF3070BD42
:10C8900001680B6831469847201A70BD5801001096
:10C8A00003C0092060010010A80F001070B50D46EC
:10C8B00004461849284605F0E7FDC0B22070FF285D
:10C8C00004D12F22144915A005F026FC194850F870
:10C8D000C41F41F4805140F8681BC16F21F04071C2
:10C8E000C167C16F41F08071C16713481349006887
:10C8F0000844401E90FBF1F04FF40011401E41EA45
:10C9000000200F4908602846BDE87040014905F045
:10C91000E9BD00005C470100405E01006F626A2DC6
:10C920003E61646320213D20284144434E616D6592
:10C93000294E430000C00F4068010010405DC60052
:10C9400000400340314910B58446086820F0FF00DC
:10C95000086008689CF80020012404FA02F21043E1
:10C960000860086840F080700860486810F0004F68
:10C97000FBD00A6822F080720A60C0F30B120868CC
:10C9800020F0FF00086008689CF8003004FA03F308
:10C9900018430860086840F080700860486810F02C
:10C9A000004FFBD00B6823F080730B600B68C0F363
:10C9B0000B1023F0FF030B600B689CF800C004FA17
:10C9C0000CFC43EA0C030B600B6843F080730B60B4
:10C9D0004B6813F0004FFBD0D1F800C02CF0807CE6
:10C9E000C1F800C0C3F30B11824202D913460246BC
:10C9F0001846884288BF0846824288BF104607F022
:10CA000009FCBDE81040024907F04CBC004003405F
:10CA10000108803970B5EFF31080012121EA000090
:10CA200080F0010572B60D4C6068002808BF2570C3
:10CA30006068B0F1FF3F04D13522094909A005F033
:10CA40006BFB606828B125B9392205490FA005F0B4
:10CA500063FB6068401C606070BD00008C010010CA
:10CA6000C8600100696E746572727570745F656E7E
:10CA700061626C655F636F756E746572203C2055F2
:10CA8000494E5433325F4D4158000000696E746561
:10CA90007272757074735F64697361626C6564004F
:10CAA00010B50E4C6068002808BF10BDEFF3108071
:10CAB000012121EA000090F0010F04D14A22084927
:10CAC00008A005F029FB6068401E606060680028CF
:10CAD00006BF2078002810BD62B610BD8C01001082
:10CAE000C8600100696E74657272757074735F64FA
:10CAF000697361626C6564000FB410B503A9029894
:10CB000005F0F0FB012000F001F8000004460848A1
:10CB1000F3F775FE0748F3F772FE05F00BFC0028EB
:10CB200018BF05F0D7FD002C18BF05F01FFBFEE76E
:10CB30001C110010701100100168002901DCF5F7CC
:10CB4000F8B9491E016041684A1C42600878704784
:10CB50002DE9F041C1F30A52A2F2FF362F4A304BC1
:10CB60000D460446142E2FDA002E12DA06F0A0FC31
:10CB70000022134607F06CF84CD2002DA4BF00240D
:10CB8000254647DA25F00040204318BF254D41D007
:10CB900018E0DFF894C02CFA06F705EA070C5CEA07
:10CBA000040C08BFBDE8F08106F082FC00221346A9
:10CBB00007F04EF82ED2002D03DA4FF48010F0402B
:10CBC0000544BD43002425E0332EC8BFBDE8F081F5
:10CBD000A6F1140C4FF0FF3727FA0CF73C4208BFC0
:10CBE000BDE8F08107F06AF80022134607F030F83C
:10CBF00010D2002D0DDA142E08BF6D1C09D0C6F11D
:10CC00003400012101FA00F02044A04238BF6D1C1D
:10CC10000446BC4329462046BDE8F0819C75008847
:10CC20003CE4377E0000F0BFFFFF0F008A68002A57
:10CC300001DCF5F76CBA521E8A604A68C0B2531C18
:10CC40004B6010707047000010B51446002222603F
:10CC5000114A21F000439342A8BF10BD53EA0002DD
:10CC600008BF10BDB3F5801FA8BF226807DA3622BF
:10CC700007F0CBFC6FF0350221F000432260DFF8B3
:10CC80001CC06FF31E510CEB23531A4441F0FF51AB
:10CC900041F00051226010BD0000F07F02FCFFFF58
:10CCA00000487047B84A010070B5044600680D4658
:10CCB000B0F1FF3F04D12C2209490AA005F02CFA5B
:10CCC00045B1012D18BF70BDA068016862681143AD
:10CCD000016070BDA068016862689143F8E70000D8
:10CCE0009C5E01006F626A2D3E70696E20213D20BE
:10CCF0002850696E4E616D65294E430070B50C4633
:10CD000005460160B1F1FF3F08BF70BD002120461C
:10CD100005F014FB04F01F00012101FA00F0686027
:10CD200024F01F0000F11801E960091D296108398C
:10CD30006961A86070BD70B5032605460C46FFF713
:10CD4000DDFFB4F1FF3F08BF70BD00212846FFF7AB
:10CD5000ABFF31462846BDE8704000F015B9000031
:10CD600070B50D4604460226FFF7C8FFB5F1FF3F38
:10CD700008BF70BD2068B0F1FF3F04D124220849EC
:10CD8000084805F0C9F9216960680860012120465A
:10CD9000FFF78AFF31462046BDE8704000F0F4B846
:10CDA000F45E0100F8CD00002DE9F04104460E4686
:10CDB00002271546FFF7A2FFB6F1FF3F08BFBDE807
:10CDC000F0812068B0F1FF3F04D1242209490AA074
:10CDD00005F0A2F96068002D14BFE16821690860C0
:10CDE00001212046FFF760FF39462046BDE8F041AB
:10CDF00000F0CAB8F45E01006F626A2D3E70696E81
:10CE000020213D202850696E4E616D65294E4300FA
:10CE10008068024A002142F820107047E80E001096
:10CE200070B51D460446B1F1FF3F04BF4FF0FF301F
:10CE300070BD1248124E026021F01F0001F01F0168
:10CE4000B042C4E900011FBF0E4988420EA0FFF79F
:10CE500053FE2068B042606818BF2030164941F880
:10CE60002050A06015491520FFF7F4F84FF0E0219D
:10CE70004FF40010C1F80001002070BD2C0100101B
:10CE800000C0092040C0092070696E73206F6E20B9
:10CE90007468697320706F72742063616E6E6F7452
:10CEA0002067656E657261746520696E7465727263
:10CEB0007570747300000000E80E001091CF000040
:10CEC00010B403684FF0010CA3F100542D4BB4F5DE
:10CED0001C2402D0402C06D00AE004790CFA04F499
:10CEE000C3F88C4004E004790CFA04F4C3F8AC40B5
:10CEF00001290168A1F10051A1F51C2112D091B3C3
:10CF000040291CBF10BC7047002AD3F8B410007928
:10CF10000CFA00F014BF084321EA0000C3F8B40083
:10CF200010BC704789B140291CBF10BC7047002A53
:10CF3000D3F8B01000790CFA00F014BF084321EACE
:10CF40000000C3F8B00010BC7047D3F89010002A5E
:10CF500000790CFA00F014BF084321EA0000C3F87E
:10CF6000900010BC7047FFE7D3F89410002A0079B6
:10CF70000CFA00F014BF084321EA0000C3F8940043
:10CF800010BC704700800240006805F005BA000040
:10CF90002DE9F05FDFF8DC90D9F88470D9F888606B
:10CFA000D9F8A450D9F8A840DFF8CCA04FF0010B75
:10CFB0009FB100BFB7FA87F0C0F11F0000F0FF0873
:10CFC0005AF8280018B12D4A0121126890470BFA2F
:10CFD00008F0C9F88C003F1AECD1002E18BFDFF81A
:10CFE0009C8011D0B6FA86F0C0F11F00C7B25AF883
:10CFF000270018B1D8F80020022190470BFA07F05B
:10D00000C9F88C00361AEDD1002D18BF1B4F14D073
:10D01000B5FA85F0C0F11F00C6B2102E07D20AEB98
:10D020008600D0F8800010B13A68012190470BFAD1
:10D0300006F0C9F8AC002D1AEAD1002C14BF0F4E2F
:10D04000BDE8F09FB4FA84F0C0F11F00C5B2102D06
:10D0500007D20AEB8500D0F8800010B132680221B7
:10D0600090470BFA05F0C9F8AC00241AEAD1BDE8E4
:10D07000F09F000000800240E80E00102C0100101C
:10D080002DE9F04106460C4640F2FF75174635EA99
:10D0900014502BD000221346304606F01DFC25D03C
:10D0A0003A463046214607F0B0FA06460C4635EAC5
:10D0B000145010D000221346304606F00DFC15D156
:10D0C0000220F6F7A4F8FEF7FDFF0A46214662F3B8
:10D0D0001E01BDE8F0810220F6F799F8FEF7EBFF9C
:10D0E0000A46214662F31E01BDE8F0813046214622
:10D0F000BDE8F081DCB0E84806F0A4F8E748E84C69
:10D100000C900CA94FF080420F94E648FEF714F8FB
:10D110000F990CA800291CBF89688847F820E249AC
:10D1200081F800044FF4E131E048FDF737FCE0A25C
:10D13000EAA1EC48FDF7A1FFEBA2EEA1E948FDF75B
:10D140009CFFFAF7E1FEFAF7C9FDF348FDF710F886
:10D15000F248FDF70DF8F248FDF70AF8F148FDF73F
:10D1600007F8F148FDF704F8F048FDF701F8DFF89B
:10D17000A893EF484946C9F80C00EE4808610246FA
:10D180000023EB494846FCF7D9FF09F5B87AEA488D
:10D19000CAF80C00E94809F5B87102460861002395
:10D1A000E54909F5B870FCF7C9FF09F53875E2489B
:10D1B000E860E248286102460023DF492846FCF780
:10D1C000BDFFDFF880B3DFF8788305F5B87600237C
:10D1D000C6E9038B5A46414605F5B870FCF7AEFF29
:10D1E00005F538770023C7E9038B5A46414605F514
:10D1F0003870FCF7A3FF05F58A68D44AD249C8E91C
:10D200000312002305F58A60FCF798FFD0480C90C4
:10D210000CA9D04A0F9405F23460FDF78DFF0F99E9
:10D220000CA800291CBF89688847CB4C2068B0F146
:10D23000FF3F04D12422C949C94804F06DFF216988
:10D24000606808600124C9F89040CAF89040C5F8A9
:10D250009040C6F89040C7F89040C248C8F8904047
:10D26000FDF773FE9148FCF717F8002844F0A186FB
:10D270004D9001218D48FCF7ADF8C0B28DF8A400A7
:10D2800020385E2884F09586DFE810F0912685240A
:10D29000A2256503F7122E1BA225A225A225A225F1
:10D2A000771DA225A225A225A225A2256D03A225D0
:10D2B000A225A225A225A225A225A225A225A22536
:10D2C000A225A225B812A225DE125E005603920303
:10D2D000EB0317065410A2254B126907BF0AB80FBB
:10D2E0000F13A225AB06D41A890405128C0DA225B2
:10D2F000A225FB0C2A0AA2254C0DD206970769032A
:10D30000EA10990CA225A2259512A225A225920326
:10D31000EB0317065410A2254B126907BF0AB80F7A
:10D320000F13A225AB06D41A890405128C0DA22571
:10D33000A225FB0C2A0AA2254C0DD20697076903E9
:10D34000EA10C422AD0C2A23584C87A104F1300006
:10D35000FDF793FE8BA104F13000FDF78EFE91499D
:10D3600004F13000FDF789FE8FA104F13000FDF7D4
:10D3700084FE984904F13000FDF77FFE96A104F188
:10D380003000FDF77AFE734D284605F05BFF9EA145
:10D3900004F13000FDF771FEA2A104F13000FDF7A9
:10D3A0006CFEAAA104F13000FDF767FEAAA104F10A
:10D3B0003000FDF762FEB1A104F13000FDF75DFE23
:10D3C000B5A104F13000FDF758FE284605F03AFFFC
:10D3D000B9A104F13000FDF750FEBEA104F1300008
:10D3E000FDF74BFEC1A104F13000FDF746FE3CA164
:10D3F00004F13000FDF741FEC5A104F13000FDF756
:10D400003CFE284605F01EFFCBA104F13000FDF7DD
:10D4100034FED2A104F13000FDF72FFE30A104F15B
:10D420003000FDF72AFED7A104F13000FDF725FEFC
:10D43000D9A104F13000FDF720FEDDA104F1300098
:10D44000FDF71BFEE3A104F13000FDF716FE2846B0
:10D4500005F0F8FEE3A104F13000FDF70EFEE5A1B2
:10D4600004F13000FDF709FEE9A104F13000FDF7F9
:10D4700004FEF4A104F13000FDF7FFFDF74904F1CB
:10D480003000FDF7FAFDF6A104F13000FDF7F5FDDF
:10D49000284605F0D7FEF9E1CDCC4C3E658500006D
:10D4A000CC4F0100700E001004E000E014020010E8
:10D4B0002F7372632F617869735F53636F72626F4A
:10D4C00074436F6E74726F6C6C65725F323031389A
:10D4D000303730362E637070000000000D0A25735F
:10D4E0000D0A0000440200104A756C2020362032DC
:10D4F0003031380056657273696F6E20312E3020DE
:10D500002D20726576202573204A2E204272616498
:10D51000736861770D0A0000AC0500101C0700104D
:10D520008C080010FC0900106C0B0010DC0C0010C3
:10D530000000524300000243000066430000FA432B
:10D540000000CD4300C0784400007A4300001B4334
:10D5500081610000CDCC4C3DFC010010645D0100F8
:10D56000204900005C0500103F202D20546869739D
:10D57000206D656E75206F6620636F6D6D616E64E2
:10D58000730D0A0030202D205A65726F20616C6C7B
:10D5900020656E636F646572206368616E6E656C92
:10D5A000730D0A006059010043202D2043757272EB
:10D5B000656E743A2053747265616D2074686520DD
:10D5C0004D6F746F722043757272656E74730D0ABD
:10D5D000000000006C5801004A202D20457863654A
:10D5E0007263697365204A6F696E7420646567723F
:10D5F0006565732F72616469616E732066756E6311
:10D6000074696F6E0D0A000057202D2057726974DF
:10D61000652076616C756520746F20617869730D83
:10D620000A00000054202D2054726170657A6F69E1
:10D6300064616C2050726F66696C65204D6F766511
:10D6400020636F6D6D616E640D0A000048202D200F
:10D65000486F6D650D0A000053202D20536574201E
:10D66000706F696E7420696E20656E636F64657299
:10D6700020636F756E74730D0A0000005A202D2010
:10D680005A65726F20456E636F64657220636861CE
:10D690006E6E656C0D0A000056202D20496E766571
:10D6A0007274206D6F746F7220646972656374693F
:10D6B0006F6E0D0A0000000058202D20457863652C
:10D6C000726369736520526F626F7469632041727F
:10D6D0006D0D0A004F202D204178697320746F2052
:10D6E0007475726E204F6E200D0A000046202D20AA
:10D6F0004178697320746F207475726E204F66666E
:10D70000202844656661756C74290D0A00000000CC
:10D7100050202D205365742050726F706F727469A1
:10D720006F6E616C204761696E206F6E20616E20A4
:10D73000417869730D0A000049202D20536574203B
:10D74000496E74656772616C204761696E206F6E07
:10D7500020616E20417869730D0A000044202D205D
:10D7600053657420446572697661746976652047F3
:10D7700061696E206F6E20616E20417869730D0AB9
:10D780000000000042202D20506974636820477219
:10D7900069707065720D0A004E202D20526F746101
:10D7A000746520477269707065720D0A0000000090
:10D7B00047202D20476F20486F6D652028616674D3
:10D7C00065722070726576696F757320686F6D651C
:10D7D000290D0A004C202D204E6F7420757365644E
:10D7E0000D0A00004B202D206E6F74207573656448
:10D7F0000D0A000059202D204D6173746572204878
:10D800006F6D652066756E6374696F6E0D0A00003A
:10D810004D202D204368616E6765206F75747075AB
:10D8200074206D6F64652028636F756E74732C208F
:10D83000646567726565732C2072616469616E73DB
:10D840000D0A000040202D20546F67676C6520642E
:10D850006562756720666C61670D0A00A459010056
:10D8600024202D20536574206275666665722072CF
:10D870006561642074696D656F7574202845782E24
:10D8800020242E30325C72290D0A0000EDA104F133
:10D890003000FDF7F2FBFAA104F13000FDF7EDFBDB
:10D8A000F94904F13000FDF7E8FBF84904F13000D4
:10D8B000FDF7E3FB284605F0C5FCF54904F130000F
:10D8C000FDF7DBFBF3A104F13000FDF7D6FBF3A17C
:10D8D00004F13000FDF7D1FBFBA104F13000FDF7AE
:10D8E000CCFBEDA104F13000FDF7C7FB284605F0A5
:10D8F000A9FCFE4904F13000FDF7BFFBFC4904F12F
:10D900003000FDF7BAFBFB4904F13000FDF7B5FB31
:10D91000E1A104F13000FDF7B0FBF7A104F1300004
:10D92000FDF7ABFB284605F08DFCFB48FBF7B4FC8C
:10D930000028FAD104F03DBBF848416A00290CBF29
:10D94000012100214162002914BFF5A1F8A1F2488C
:10D95000303003F0A1BFF8F793FD04F02ABBF7F7CE
:10D960009DF904F026BB0120FBF714FCF44D28467A
:10D9700005F068FC0220FBF70DFC284605F062FC70
:10D980000320FBF707FC284605F05CFC0420FBF7AE
:10D9900001FC284605F056FC05242046FBF7FAFB5F
:10D9A000284605F04FFC641C062CF6DD04F001BB94
:10D9B000D94CE4A104F13000FDF75FFB29AAECA1EA
:10D9C00004F13000FDF720FB9DF8A4004F2818BF9C
:10D9D0006F281ED1E748FCF741FCE748FCF73EFC06
:10D9E000E648FCF73BFCE648FCF738FCE548FCF76A
:10D9F00035FCE548FCF732FCE44C2068B0F1FF3F11
:10DA000004D12422E249E34804F086FB21696068DE
:10DA100008609DF8A400462818BF662844F0C98213
:10DA2000D448FCF7BBFDD448FCF7B8FDD348FCF75D
:10DA3000B5FDD348FCF7B2FDD248FCF7AFFDD248A4
:10DA4000FCF7ACFDD14C2068B0F1FF3F04D124229B
:10DA5000CF49D04804F060FBE1686068086004F0DA
:10DA6000A8BAC74CE06A18B904F5B870C06A28B102
:10DA7000C348FCF7F3FBC348FCF7F0FBA64DC6A177
:10DA800005F13000FDF7F9FA2EAACBA105F130001F
:10DA9000FDF7BAFA2E99A0690F4606F031FA05F69D
:10DAA0005816A0613946B06906F004FDB0613846E9
:10DAB00006F0FAF902460B46C0A105F13000FDF769
:10DAC000DCFAC0A105F13000FDF7D7FA05F5527078
:10DAD000FDF72DFA2DE0206A06F0E6F906460F461E
:10DAE000A06906F0E1F905460C46D8F8200006F0DA
:10DAF000DBF982468B46D8F8180006F0D5F9804647
:10DB00008946B548FDF7DCF906F0CEF9CDE90454B5
:10DB1000CDE906678DE8000F0B460246AFA1BB4872
:10DB2000FDF7ABFABA4805F08DFB7B48FBF7B4FB79
:10DB300050B3DFF84C82B74D2946D8F8180006F0EC
:10DB4000DFF9D8F8201006F079FB0AD32946D8F877
:10DB5000180006F0AFFCD8F8201006F06FFC84F037
:10DB60002882884C2946A06906F0CAF9216A06F085
:10DB700065FBB0D32946A06906F09CFC216A06F03B
:10DB80005DFCA8D304F015BA01216348FBF722FC21
:10DB9000C0B2712818BF5128CBD104F00ABA784C12
:10DBA000E06A18B904F5B870C06A28B17448FCF787
:10DBB00055FB7448FCF752FBDFF85CB196A10BF102
:10DBC0003000FDF75AFA2EAA7BA10BF13000FDF7C9
:10DBD0001BFA2E99A0690E4606F092F90BF658151D
:10DBE000A0613146A86906F08BF9A861304606F0BD
:10DBF0005BF902460B4671A10BF13000FDF73DFACF
:10DC000070A10BF13000FDF738FAA5F5C260FDF701
:10DC10008EF9DFF800A220E1A86906F045F98046F8
:10DC20008946A06906F040F906460F466A48FDF7A6
:10DC300047F906F039F902462868CDF81080CDE999
:10DC40000590F9E023202D2053656C662054657300
:10DC5000742077697468206D6F746F7220637572B9
:10DC600072656E747320616E6420656E636F6465A7
:10DC70007220646972656374696F6E0D0A0000003A
:10DC80002525202D200D0A00B4580100005901005F
:10DC90009453010026202D200D0A00002A202D205B
:10DCA0004D616E75616C6C7920696E6372656D652E
:10DCB0006E742F64656372656D656E7420616E208D
:10DCC000617869730D0A00007C202D204661737411
:10DCD000204D6F746F72204D6178204375727265AC
:10DCE0006E742066696E640D0A000000705A0100AF
:10DCF000E05A0100FC590100507265737320616E97
:10DD000079206B657920746F20636F6E74696E750E
:10DD1000652E0D0A0000000014020010C80000105B
:10DD20000D0A4465627567204F6E0D0A0000000001
:10DD30000D0A4465627567204F66660D0A00000093
:10DD40000AD7A33B0D0A416C6C3A20276F27206647
:10DD50006F7220616C6C204F6E2C20276627206626
:10DD60006F7220616C6C206F66660D0A0000000007
:10DD700025630000AC0500101C0700108C08001083
:10DD8000FC0900106C0B0010DC0C0010FC010010F2
:10DD9000645D0100204900000D0A456E7465722023
:10DDA000777269737420706974636820636F756E2D
:10DDB00074730D0A000000002566000025660D0A38
:10DDC000000000005072657373207120746F207121
:10DDD000756974200D0A00005C050010543D252E65
:10DDE0003266205350343D252E336620706F7334D5
:10DDF0003D252E3366205350353D252E3366207049
:10DE00006F73353D252E3366200D0A004402001045
:10DE1000BC74133C000070410D0A456E746572209D
:10DE2000777269737420726F7461746520636F75A3
:10DE30006E74730D0A00000020680096CDE9017031
:10DE40000B46EAA10BF13000FDF717F9F64805F093
:10DE5000F9F9F648FBF720FA20B35146A06906F01D
:10DE60004FF8216A06F0EAF908D35146A06906F096
:10DE700021FB216A06F0E2FA84F09B805146A869F2
:10DE800006F03EF8296A06F0D9F9FFF4C5AE51460E
:10DE9000A86906F00FFB296A06F0D0FAFFF4BCAEC1
:10DEA00004F087B80121E148FBF794FAC0B2712869
:10DEB00018BF5128D1D104F07CB8DC4CDCA104F1AE
:10DEC0003000FDF7DAF829AAAFF25C1104F1300056
:10DED000FDF79AF89DF8A40073280CD06D2862D045
:10DEE000632864D0E0A104F13000FDF7C6F84FF0DC
:10DEF0007E5003F05BBDE2A104F13000FDF7BDF8F8
:10DF0000E548FCF787F8E548FCF784F8E448FCF7B7
:10DF100081F8E448FCF77EF8E348FCF77BF8E34837
:10DF2000FCF778F8E148406F05F0BEFF8246DE4816
:10DF30008B46406F05F0B8FF8046DA488946406F4F
:10DF400005F0B2FF0646D6480F46406F05F0ACFF1D
:10DF50000546D2480391406F05F0A6FF0090CE48D9
:10DF60000C46406F05F0A0FF0DF1100CCDE9014506
:10DF70008CE8C00F0B460246CDA1D648FDF77DF8D0
:10DF8000D54805F05FF9A948FBF786F90028B7D115
:10DF90000121A648FBF71EFAC0B2712818BF51280C
:10DFA000AED104F006B8F8F781F804F002B8BA4927
:10DFB0000020C1F8840001F5B871C1F8840001F5B2
:10DFC000B871C1F8840001F5B871C1F8840001F599
:10DFD000B871C1F8840001F5B871C1F8840003F08C
:10DFE000E8BFBD4F914EBD4D012400BF05F1340087
:10DFF0000FC88DE80F00D5E90B23B9A106F1300059
:10E00000FDF73BF8384605F01DF98848FBF744F961
:10E0100018B1002CEAD103F0CCBF01218348FBF7F3
:10E02000D9F9C0B2712818BF5128F2D103F0C1BF8D
:10E0300000207E4C2F90B2A104F13000FDF71DF8B6
:10E0400029AAAFF2D42104F13000FCF7DDFFB6A11C
:10E0500004F13000FDF711F82FAAAFF2A42104F16A
:10E060003000FCF7D1FF2F9805F01EFF02460B464B
:10E07000AFF2B82104F13000FCF7FFFF9DF8A400D7
:10E080003138062883F09587DFE810F00600160087
:10E0900029003900490059002F9805F005FF024674
:10E0A0000B46A9A104F13000FCF7E7FF2F9806F01A
:10E0B0005DF8014678480EE02F9805F0F5FE02461F
:10E0C0000B46ABA104F13000FCF7D7FF2F9806F008
:10E0D0004DF801467148FCF738F803F06ABF2F98F5
:10E0E00005F0E2FE02460B46ABA104F13000FCF75E
:10E0F000C4FF2F9806F03AF801466948EBE72F98DD
:10E1000005F0D2FE02460B46ADA104F13000FCF74B
:10E11000B4FF2F9806F02AF801466248DBE72F98F3
:10E1200005F0C2FE02460B46AFA104F13000FCF739
:10E13000A4FF2F9806F01AF801465B48CBE72F980A
:10E1400005F0B2FE02460B46B1A104F13000FCF727
:10E1500094FF2F9806F00AF801465448BBE75F4D3C
:10E1600064202E782870B44805F06CF8DFF8CCC233
:10E170000020B349CDF830C1CDE90010014602902E
:10E18000B04BB14A6046F7F7A3FB4C9805F08CFE04
:10E190000F460446AD4AAE4B05F05CFC22463B46BA
:10E1A00005F086F905F052F9F8F7A0F8A9A1494859
:10E1B000FCF763FF2E7003F0FCBE1C4CA7A104F11A
:10E1C0003000FCF75AFFADA104F13000FCF755FF19
:10E1D0004FF00009DFF8C4B2DFF8C4A2A4F1480789
:10E1E00067E10A2E00D25DE10BE20000543D252ECE
:10E1F00032662053503D252E336620636F3D252E19
:10E20000336620706F733D252E33662076656C3D36
:10E21000252E3366206163633D252E336620202042
:10E22000202020200D0A0000BC74133C14020010B2
:10E230000D0A50726573732027732720746F207343
:10E24000747265616D2C20276D2720666F72206DBA
:10E2500061782C2027632720746F20636C656172BE
:10E26000206D61780D0A000057726F6E6720636F32
:10E270006D6D616E6420676976656E210000000037
:10E280000D0A5072657373207120746F2071756967
:10E2900074200D0A00000000AC0500101C070010DF
:10E2A0008C080010FC0900106C0B0010DC0C001036
:10E2B000252E336620252E336620252E3366202515
:10E2C0002E336620252E336620252E3366200D0A38
:10E2D00000000000440200100AD7A33CC800001050
:10E2E0000D0A253164202531642025316420253133
:10E2F000642025316420253164202531640D0A0015
:10E300000D0A456E746572206178697320746F2000
:10E310006368616E676520656E636F646572207601
:10E32000616C75650D0A00000D0A0D0A456E746575
:10E3300072206E657720656E636F6465722076610A
:10E340006C75653A000000007570646174696E67F1
:10E3500020526F626F7469632041786973203120A5
:10E3600076616C756520746F20252E31660D0A006C
:10E370007570646174696E6720526F626F7469634F
:10E38000204178697320322076616C756520746F46
:10E3900020252E31660D0A007570646174696E6700
:10E3A00020526F626F746963204178697320332053
:10E3B00076616C756520746F20252E31660D0A001C
:10E3C0007570646174696E6720526F626F746963FF
:10E3D000204178697320342076616C756520746FF4
:10E3E00020252E31660D0A007570646174696E67B0
:10E3F00020526F626F746963204178697320352001
:10E4000076616C756520746F20252E31660D0A00CB
:10E410007570646174696E6720526F626F746963AE
:10E42000204178697320362076616C756520746FA1
:10E4300020252E31660D0A00CDCCCC3D0000A04039
:10E44000B89EB1C23D0ABEC25C8FF0429A999999BA
:10E450009999C93F4F4B0D0A000000000D0A5072F8
:10E46000657373207120746F20717569742045780D
:10E470006572636973650D0A00000000526563658B
:10E4800069766564206D6F766520746573742063AA
:10E490006F6D6D616E640D0A00000000C3F5C8BFAA
:10E4A000C3F5C83FDFE806F005182D445A6E809783
:10E4B000AEC5FB48CDF80090CDF804905B465246BF
:10E4C0000021CDF80890F7F703FA0546F548F7F76D
:10E4D0000DFF04460126C2E0F449CDF80090CDE9D5
:10E4E0000191F1485B4652460021F7F7F1F90546E4
:10E4F000EF48F04904F0AAFFF7F7F8FE04460226B9
:10E50000ADE0EE48CDF80090CDE901B0DFF8A8C34A
:10E510005B46524600216046F7F7DAF90546E848BF
:10E52000E84904F093FFF7F7E1FE0446032696E07E
:10E53000E548CDF80090CDF804905B4652460021A6
:10E54000CDF80890F7F7C4F90546E048E04904F033
:10E550007DFFF7F7CBFE0446042680E0CDE900B945
:10E560000023D94852461946CDF80890F7F7B0F97C
:10E570000546D648D64904F069FFF7F7B7FE0446CA
:10E5800005266CE0D449CDE9001AD2480023D34ACD
:10E59000CDF80890D249F7F79BF90546D148F7F72F
:10E5A000A5FE044606265AE0CB49CDE9001ADFF85D
:10E5B00038C3CE4802900023C84AC9496046F7F7DD
:10E5C00087F90546BA48CA4904F040FFF7F78EFEBE
:10E5D0000446072643E0C048CDE9000ADFF808C337
:10E5E0000023BE4ABE49CDF808906046F7F770F99F
:10E5F0000546AF48BE4904F029FFF7F777FE044609
:10E6000008262CE0B449CDE9001ADFF8DCC2B7488F
:10E6100002900023B14AB2496046F7F759F905461E
:10E62000A348B34904F012FFF7F760FE0446092639
:10E6300015E0A948CDE9000ADFF8ACC20023A74ADB
:10E64000A749CDF808906046F7F742F90546984883
:10E65000A74904F0FBFEF7F749FE04460026A5484B
:10E66000FAF71AFE38B90121A248FAF7B3FEC0B290
:10E67000712808BF0125F9F7E1FC3868DFF87882D6
:10E68000B0F1FF3F04D12C229C499D4803F044FD8A
:10E690007869006879680842D8F8000000F1010044
:10E6A00001D010B106E080B90AE0242293499448D1
:10E6B00003F032FDD8F81010D8F80400086009E023
:10E6C00024228E498E4803F027FDD8F80C00D8F894
:10E6D0000410016055EA04003FF483AD03F069BC07
:10E6E000844C88A104F13000FCF7C7FC29AAAFF6DE
:10E6F000801104F13000FCF787FC8BA104F130009D
:10E70000FCF7BBFC2FAAAFF6501104F13000FCF768
:10E710007BFC2F9805F0C8FB02460B46AFF6641150
:10E7200004F13000FCF7A9FC84A104F13000FCF7EF
:10E73000A4FC4DAAAFF6801104F13000FCF764FC94
:10E740004D9805F0B1FB02460B46AFF6901104F16F
:10E750003000FCF792FC9DF8A400342831D007DC8F
:10E7600031280DD0322817D033281ED003F021BC19
:10E7700035282FD0362836D062283DD003F019BC7A
:10E7800071A104F13000FCF778FC75484D9A2F997F
:10E79000FBF77AFC03F00DBC72A104F13000FCF72A
:10E7A0006CFC76484D9A2F9907E075A104F1300072
:10E7B000FCF763FC78484D9A2F99FBF765FC03F052
:10E7C000F8BB76A104F13000FCF757FC79484D9A6C
:10E7D0002F99F2E778A104F13000FCF74EFC7C4859
:10E7E0004D9A2F99E9E77BA104F13000FCF745FC35
:10E7F0007E484D9A2F99E0E77DA104F13000FCF7A7
:10E800003CFC57484D9A2F99D7E73A4C7F4904F181
:10E810003000FCF732FC5BAAAFF6AC2104F130000B
:10E82000FCF7F2FB9DF86C0162282BD010DC342839
:10E8300029D006DC312827D0322826D0332825D00D
:10E8400014E0352823D0362822D0612821D00DE0CD
:10E8500070281FD006DC64281DD065281CD06728CE
:10E860001BD003E0722819D0732818D068A104F1D6
:10E870003000FCF702FC1F48FAF70EFD002843F0B9
:10E88000988397E112E1F1E0D2E0DBE0E4E0F7E029
:10E8900000E147E136E173E11CE13BE12AE121E1DE
:10E8A0003333A3400AD7C340CDCC8C3F0000A041F6
:10E8B0009A999959B81EF53F33338340000020429E
:10E8C0003333337314AE134000006040CDCCCCCC56
:10E8D000CCCC10400000A04014AE47BF14AE473F60
:10E8E0000AD7A33E0000C040CDCC0C4000004842F7
:10E8F000B81E054014020010CC010010645D010038
:10E90000204900000D0A456E7465722061786973B4
:10E9100020746F206D6F76652074726170617A6FFC
:10E9200069640D0A000000000D0A0D0A456E746549
:10E930007220706F736974696F6E3A00456E74650A
:10E94000722074696D653A004D6F76696E6720526A
:10E950006F626F746963204178697320310D0A001A
:10E96000AC0500104D6F76696E6720526F626F7450
:10E970006963204178697320320D0A001C0700107A
:10E980004D6F76696E6720526F626F7469632041C4
:10E9900078697320330D0A008C0800104D6F76697A
:10E9A0006E6720526F626F746963204178697320CB
:10E9B000340D0A00FC0900104D6F76696E67205215
:10E9C0006F626F746963204178697320350D0A00A6
:10E9D0006C0B00104D6F76696E6720526F626F741A
:10E9E0006963204178697320360D0A00DC0C001041
:10E9F0004D6F76696E672042617365206F662053A4
:10EA0000636F72626F740D0A00000000C05B01004A
:10EA10000D0A496E76616C696420706172616D6582
:10EA200074657220656E74657265640D0A0000007D
:10EA3000E6A104F13000FCF720FBEA48FBF70EFCEE
:10EA4000E84830E0E8A104F13000FCF716FBEC48A0
:10EA5000FBF704FCEA4826E0EAA104F13000FCF7E9
:10EA60000CFBEE48FBF7FAFBEC481CE0ECA104F1D0
:10EA70003000FCF702FBF048FBF7F0FBEE4812E039
:10EA8000EEA104F13000FCF7F8FAF248FBF7E6FBE0
:10EA9000F04808E0F0A104F13000FCF7EEFAF44889
:10EAA000FBF7DCFBF248FBF701FCE4E6F1A104F123
:10EAB0003000FCF7E2FAF9F781FF28B1F1A104F187
:10EAC0003000FCF7DAFAD6E6F3A104F13000FCF7E7
:10EAD000D4FAD0E6F5A104F13000FCF7CEFAF5F750
:10EAE000CBFAC8E6F5A104F13000FCF7C6FAF7F757
:10EAF00033F9C0E6F6A104F13000FCF7BEFAF8F7EE
:10EB0000F3FDB8E6F8A104F13000FCF7B6FAF8F727
:10EB1000F7F9B0E6FAA104F13000FCF7AEFAF6F727
:10EB2000B1FCA8E6F6F7BAF8050022D0AD48FBF72D
:10EB300035FDB348FBF732FDB848FBF72FFDBE4863
:10EB4000FBF72CFDC348FBF729FDC948FBF726FD61
:10EB5000F0A104F13000FCF790FAF548406A002873
:10EB60003FF489AE2A46F3A104F13000FCF785FAA0
:10EB700081E6AFF2207104F13000FCF77EFA7AE60C
:10EB8000F3A104F13000FCF778FA01AAAFF6D851EE
:10EB900004F13000FCF738FA019805F085F90246D7
:10EBA0000B46F8A104F13000FCF767FAE048019940
:10EBB000816260E60121FC48FAF70CFC5BE6FA484A
:10EBC000FAF76AFB50B1F949F948FCF756FAF648EA
:10EBD000FAF762FB0028FAD103F0EBB90121F24801
:10EBE000FAF7F8FBEBE7F04CF2A104F13000FCF788
:10EBF00044FA04F56670F7F717F8F04D284604F06C
:10EC000021FBEFA104F13000FCF737FA04F5A16015
:10EC1000F7F70AF8284604F015FBEBA104F13000E1
:10EC2000FCF72BFA04F5CF60F6F7FEFF284604F058
:10EC300009FBE7A104F13000FCF71FFA04F5FD60C1
:10EC4000F6F7F2FF284604F0FDFAE3A104F13000E4
:10EC5000FCF713FA04F65810F6F7E6FF284604F01E
:10EC6000F1FADFA104F13000FCF707FA04F6C8203E
:10EC7000F6F7DAFF284604F0E5FAF7F717FA03F09B
:10EC800098B9C94CD8A104F13000FCF7F6F929AACB
:10EC9000AFF6247104F13000FCF7B6F99DF8A4201A
:10ECA000D9A104F13000FCF7E8F99DF8A420DBA11C
:10ECB00004F13000FCF7E1F954AAAFF6047104F155
:10ECC0003000FCF7A1F9549805F0EEF8CDE9000109
:10ECD0009DF8A420DAA104F13000FCF7CEF99DF8EC
:10ECE000A4003138062883F06481DFE810F00600C4
:10ECF00009000F001200150018003A48549901E06D
:10ED00003F485499F6F7AEFA03F053B94348549983
:10ED1000F8E749485499F5E74E485499F2E75448C2
:10ED20005499EFE7A04CCCA104F13000FCF7A5F911
:10ED300029AAAFF6C47104F13000FCF765F99DF81B
:10ED4000A420D0A104F13000FCF797F955AAD4A172
:10ED500004F13000FCF758F99DF8A420A2F131002D
:10ED6000062817D2DFE800F00306090C0F121D4831
:10ED700055990DE0224855990AE02848559907E031
:10ED80002D48559904E03348559901E03848559984
:10ED9000C0F890101348C3A1D0F8903004F13000AF
:10EDA00002F094BD804CCBA104F13000FCF765F972
:10EDB0004AAACFA104F13000FCF726F99DF82811EA
:10EDC0003139062900D295E19DE10000486F6D6957
:10EDD0006E6720526F626F74696320417869732097
:10EDE000310D0A00AC050010486F6D696E67205246
:10EDF0006F626F746963204178697320320D0A0075
:10EE00001C070010486F6D696E6720526F626F7447
:10EE10006963204178697320330D0A008C08001063
:10EE2000486F6D696E6720526F626F74696320412D
:10EE300078697320340D0A00FC090010486F6D6971
:10EE40006E6720526F626F74696320417869732026
:10EE5000350D0A006C0B0010486F6D696E6720520B
:10EE60006F626F746963204178697320360D0A0000
:10EE7000DC0C0010486F6D696E6720626173650D70
:10EE80000A000000486F6D6520626173652066614D
:10EE9000696C6564210D0A00486F6D6520626173BD
:10EEA0006520737563636573730D0A00486F6D6940
:10EEB0006E6720456C626F770D0A0000486F6D69C0
:10EEC0006E672053686F756C6465720D0A000000F0
:10EED000486F6D696E6720577269737420526F7442
:10EEE0006174650D0A000000486F6D696E672057F8
:10EEF000726973742050697463680D0A0000000021
:10EF0000486F6D696E6720477269707065720D0A8F
:10EF1000000000000D0A0D0A4E414B0D0A484F4DEE
:10EF200045204641494C45442121210D0A0000005D
:10EF3000C80000104D617374657220486F6D6520C4
:10EF400072657475726E65642025640D0A00000098
:10EF50000D0A456E746572206E657720676C6F626E
:10EF6000616C2064656C61792074696D6520666FE1
:10EF70007220686F6D652066756E6374696F6E735D
:10EF80000D0A0000686F6D6544656C6179476C6FB0
:10EF900062616C2064656C6179206973206E6F77A3
:10EFA00020252E33660D0A00140200102C53010098
:10EFB0004402001041786973310D0A00CDCCCC3D7C
:10EFC00041786973320D0A0041786973330D0A0084
:10EFD00041786973340D0A0041786973350D0A0070
:10EFE00041786973360D0A000D0A456E746572200A
:10EFF0006178697320746F20676976652073657422
:10F0000020706F696E743A0041786973202563201F
:10F01000656E74657265642E0D0A0000456E746538
:10F02000722076616C756520666F7220736574203E
:10F03000706F696E7420617869732025630D0A0012
:10F040004178697325632073657420706F696E74ED
:10F0500020252E31660D0A000D0A456E746572205A
:10F060006178697320746F20496E76657274206DC3
:10F070006F746F7220646972656374696F6E0D0AD4
:10F0800000000000456E7465722076616C75652025
:10F09000666F7220696E76657273696F6E0D0A0015
:10F0A00025640000417869732563206D6F746F7269
:10F0B00020646972656374696F6E20696E7665722B
:10F0C00073696F6E2073657420746F2025640D0A58
:10F0D000000000000D0A456E746572206178697346
:10F0E00020746F2073657420506B0D0A00000000BF
:10F0F00025630000DFE801F0030527292B2DF248E6
:10F1000000E0F248C06804F0CFFE02460B46F0A1D2
:10F1100004F13000FBF7B1FF9DF82821F3A104F1C1
:10F120003000FBF7AAFF56AAF7A104F13000FBF765
:10F130006BFF9DF828013138062832D2DFE800F055
:10F140000B11171D2329F148DCE7F148DAE7F148F4
:10F15000D8E7F148D6E7DC485699C160D0E90423E6
:10F160001CE0DA485699C160D0E9042316E0E7486C
:10F170005699C160D0E9042310E0E5485699C16072
:10F18000D0E904230AE0E3485699C160D0E904239A
:10F1900004E0E1485699C160D0E90423FAF7CEFFB4
:10F1A00004E0DEA104F13000FBF767FF9DF8285171
:10F1B000A5F13101062908D2DFE801F00305181A8C
:10F1C0001C1EC14800E0C148C06804F06DFECDE9D6
:10F1D00000012A46D8A104F13000FBF74EFFE248B7
:10F1E000FAF75AF80028FAD102F0E3BEC748EBE775
:10F1F000C748E9E7C748E7E7C748E5E7DA4CDBA1D6
:10F2000004F13000FBF739FF4AAAAFF21C1104F1F8
:10F210003000FBF7F9FE9DF828113139062908D294
:10F22000DFE801F0030527292B2DA74800E0A748B8
:10F23000006904F039FE02460B46A5A104F1300036
:10F24000FBF71BFF9DF82821CFA104F13000FBF74D
:10F2500014FF57AAACA104F13000FBF7D5FE9DF8CE
:10F26000A4003138062838D2DFE800F00B1117214E
:10F27000272FA648DCE7A648DAE7A648D8E7A6483D
:10F28000D6E79148579A02614369C1681AE08F48EE
:10F29000579A02614369C16814E09C48579A026119
:10F2A0004369C168D0F81001FAF746FB1AE09848A4
:10F2B000579A02614369C16804E09648579A02610F
:10F2C0004369C168FAF73AFF0CE09348579A026124
:10F2D0004369C168FAF732FF04E090A104F13000FD
:10F2E000FBF7CBFE9DF82851A5F13101062908D284
:10F2F000DFE801F00305181A1C1E734800E073488C
:10F30000006904F0D1FDCDE900012A46A5A104F170
:10F310003000FBF7B2FE9448F9F7BEFF0028FAD19F
:10F3200002F047BE7948EBE77948E9E77948E7E733
:10F330007948E5E78C4CA7A104F13000FBF79DFE6E
:10F340004AAAAFF2542104F13000FBF75DFE9DF8AC
:10F3500028113139062908D2DFE801F003052729F1
:10F360002B2D594800E05948406904F09DFD0246A4
:10F370000B4657A104F13000FBF77FFE9DF82821D2
:10F380009BA104F13000FBF778FE58AA5EA104F1BE
:10F390003000FBF739FE9DF828013138062832D2BB
:10F3A000DFE800F00B11171D23295848DCE7584807
:10F3B000DAE75848D8E75848D6E74348589B4361AE
:10F3C000D0E903121CE04148589B4361D0E9031285
:10F3D00016E04E48589B4361D0E9031210E04C48B8
:10F3E000589B4361D0E903120AE04A48589B4361A5
:10F3F000D0E9031204E04848589B4361D0E9031266
:10F40000FAF79CFE04E045A104F13000FBF735FE5D
:10F410009DF82851A5F13101062908D2DFE801F055
:10F420000305181A1C1E284800E02848406904F00B
:10F430003BFDCDE900012A4674A104F13000FBF741
:10F440001CFE4948F9F728FF0028FAD102F0B1BDA7
:10F450002E48EBE72E48E9E72E48E7E72E48E5E798
:10F46000414C76A104F13000FBF707FE29AAAFF268
:10F47000803104F13000FBF7C7FD9DF8A40034286B
:10F4800008BF23481DD00BDC312815D0322808BF17
:10F490000E4816D0332808BF1C4812D002F089BD90
:10F4A000352808BF1B480CD0362808BF1A4808D09A
:10F4B000612807D002F07DBD0348FAF7ADFE02F0E7
:10F4C00078BDD3E0D6E00000AC0500101C070010AA
:10F4D00043757272656E742076616C756520697310
:10F4E0002025372E32660D0A00000000456E746537
:10F4F000722076616C756520666F72204178697341
:10F50000256320506B0D0A00256600008C08001052
:10F51000FC0900106C0B0010DC0C00100D0A496E89
:10F5200076616C696420617869732073656C6563CA
:10F530007465640D0A0000004178697325632050EA
:10F540006B2073657420746F2025660D0A507265F8
:10F55000737320616E79206B657920746F206578F4
:10F5600069740D0A00000000140200100D0A456EB7
:10F57000746572206178697320746F2073657420DC
:10F58000496B0D0A00000000456E746572207661BB
:10F590006C756520666F7220417869732563204918
:10F5A0006B0D0A0041786973256420496B207365EF
:10F5B0007420746F2025660D0A5072657373206184
:10F5C0006E79206B657920746F20657869740D0AF7
:10F5D000000000000D0A456E746572206178697341
:10F5E00020746F2073657420446B0D0A00000000C6
:10F5F000456E7465722076616C756520666F722049
:10F6000041786973256320446B0D0A004178697362
:10F61000256320446B2073657420746F2025660D6C
:10F620000A507265737320616E79206B657920745E
:10F630006F20657869740D0A000000000D0A456EA0
:10F64000746572206178697320746F205A65726FD7
:10F650002028312D362C206F722027612720666FDD
:10F660007220616C6C290D0A00000000FAF7D4FDCD
:10F6700002F09FBCF548FAF7CFFDF548FAF7CCFD4C
:10F68000F448FAF7C9FDF448FAF7C6FDF348FAF76B
:10F69000C3FDF348EAE7FF4CF2A104F13000FBF7A9
:10F6A000ECFC29AAAFF2B85104F13000FBF7ACFC36
:10F6B0009DF8A400342808BFE7481DD00BDC312892
:10F6C00015D0322808BFE24816D0332808BFE148D9
:10F6D00012D002F06EBC352808BFE0480CD03628A6
:10F6E00008BFDF4808D061280AD002F062BCD748C2
:10F6F000FAF7B4FD02F05DBCFAF7B0FD02F059BCB8
:10F70000D248FAF7ABFDD248FAF7A8FDD148FAF78C
:10F71000A5FDD148FAF7A2FDD048FAF79FFDD048E1
:10F72000EAE7DC4CDCA104F13000FBF7A6FC29AAD7
:10F73000AFF2446104F13000FBF766FC9DF8A400D1
:10F74000342808BFC44818D00CDC312808BFBF4893
:10F7500013D0322808BFBE480FD0332808BFBD4899
:10F760000BD01FE0352808BFBC4806D0362808BF9C
:10F77000BB4802D0612803D014E0FAF70FFF11E074
:10F78000B248FAF70BFFB248FAF708FFB148FAF7A8
:10F7900005FFB148FAF702FFB048FAF7FFFEB0489C
:10F7A000FAF7FCFE9DF8A420C8A104F13000FBF795
:10F7B00064FC02F0FEBBB74CC8A104F13000FBF7BB
:10F7C0005CFC29AAAFF2D86104F13000FBF71CFC05
:10F7D0009DF8A400312807D1CC4901204860CCA174
:10F7E00004F13000FBF749FC9DF8A400302842F0FA
:10F7F000E083C64900204860C8A121E0A54CCBA108
:10F8000004F13000FBF739FC29AAAFF21C7104F1B6
:10F810003000FBF7F9FB9DF8A400312807D1BB4964
:10F8200001208860D0A104F13000FBF726FC9DF890
:10F83000A400302842F0BD83B44900208860D1A1E3
:10F8400004F1300002F028B8924CD54904F13000A0
:10F85000FBF713FCD34AAFF2503104F13000FBF751
:10F86000D3FBAA48D04AC168914203DCCF4A9142F7
:10F8700082F29F83C26002F09CBBA44C606A18B104
:10F88000CBA1D348FBF7F9FBD24AAFF28431D04881
:10F89000FBF7BAFBD0496069884203DCC349884260
:10F8A00082F28783616102F084BB7A4DCB4905F116
:10F8B0003000FBF7E2FB5AAAAFF2CC7105F1300041
:10F8C000FBF7A2FB9DF86801702800F0CC8304DCF4
:10F8D00062280CD065287DD004E0722800F0CB852A
:10F8E000732878D0BEA105F1300001F0D5BFC3A1C7
:10F8F00005F13000FBF7C1FBC4A105F13000FBF7B7
:10F90000BCFB06AAAFF6180105F13000FBF77CFB43
:10F910009DF81820C5A105F13000FBF7AEFB9DF85E
:10F920001800642821D1C3A105F13000FBF7A5FB25
:10F930000AAAAFF22C4105F13000FBF765FB0A98EB
:10F9400004F0B2FA02460B46C2A105F13000FBF703
:10F9500094FBCA480A99A0F50A660160F26A4AB1A6
:10F96000C74905F13000FBF788FB9DF818007228A5
:10F9700005D037E0806804F095FCB061F5E7C1A1DF
:10F9800005F13000FBF779FB05AAAFF2844105F1E0
:10F990003000FBF739FB059804F086FA02460B4667
:10F9A000C0A105F13000FBF768FBB44E059870600C
:10F9B00004F07AFA0022C54B04F04CF8C44AC54B57
:10F9C00003F032FE03F042FDA6F50A6701463060FF
:10F9D000F86A01E079E29FE170B1A94905F13000D0
:10F9E000FBF74BFB002C02F0E4829DF81800642822
:10F9F00007D0722816D084E1B06804F053FCB861D7
:10FA0000F0E79E488168A0F50A60006A04F0ECFA0D
:10FA100004F04AFA02460B46AFA105F13000FBF7AD
:10FA20002CFB6EE195488168A0F50A60006A04F03D
:10FA3000DBFA04F039FAAE4AAE4B04F00BF803F0EF
:10FA400005FD04F031FA02460B4655E1AC05001005
:10FA50001C0700108C080010FC0900106C0B001033
:10FA6000DC0C00100D0A456E7465722061786973B4
:10FA700020746F207475726E204F6E2028312D36E1
:10FA80002C206F722027612720666F7220616C6CBA
:10FA9000290D0A00140200100D0A456E74657220CB
:10FAA0006178697320746F207475726E204F66667A
:10FAB0002028312D362C206F722027612720666F79
:10FAC0007220616C6C290D0A000000004178697396
:10FAD0002563204F66660D0A000000000D0A456E82
:10FAE000746572203120746F207475726E20737487
:10FAF0007265616D204F6E2C203020746F207475FC
:10FB0000726E204F66663A0D0A000000C8000010B1
:10FB100053747265616D204F6E0D0A0053747265E7
:10FB2000616D204F66660D0A000000000D0A456EEB
:10FB3000746572203120746F207475726E20737436
:10FB40007265616D204F75747075742041637469BE
:10FB50007665204F6E2C203020746F207475726E85
:10FB6000204F66663A0D0A0053747265616D204F2E
:10FB7000757470757420416374697665204F6E0DDD
:10FB80000A00000053747265616D204F75747075C2
:10FB90007420416374697665204F66660D0A000023
:10FBA00034540100D4000010000070426F12833AF8
:10FBB0000D0A456E7465722073657269616C2072FE
:10FBC0006561642074696D656F75740D0A000000CD
:10FBD00044020010DC00001000002041605B0100C6
:10FBE000496E636F7272656374206A6F696E742008
:10FBF000656E74657265642E0D0A0000426173655E
:10FC00002073656C65637465640D0A0064656772D2
:10FC1000656573206F722072616469616E7320285C
:10FC200064206F722072293F0D0A000025630D0ABF
:10FC300000000000456E746572206465677265653A
:10FC40007320746F207475726E20626173653A0D53
:10FC50000A0000004465677265657320656E74650F
:10FC60007265643A252E32660D0A507265737320F0
:10FC70007120746F20657869740D0A004C0E0010B5
:10FC8000294E0100456E7465722072616469616E6F
:10FC90007320746F207475726E20626173653A0D03
:10FCA0000A00000052616469616E7320656E7465BC
:10FCB0007265643A252E32660D0A507265737320A0
:10FCC0007120746F20657869740D0A0000806640A9
:10FCD0006E861BF0F921094062617365203D202585
:10FCE000342E326620646567202020200D0A000033
:10FCF00070E20DA545DF913FEBA105F13000FBF768
:10FD0000BCF9EF4803F09EFAEE48F9F7C5FA00286F
:10FD100042F04F8100F088BDEBA105F13000FBF708
:10FD2000ACF9AFF2181105F13000FBF7A6F906AAFD
:10FD3000AFF6444105F13000FBF766F99DF8182055
:10FD4000AFF2181105F13000FBF797F99DF8180094
:10FD500064282CD1E1A105F13000FBF78EF90AAA45
:10FD6000AFF65C0105F13000FBF74EF90A9804F09C
:10FD70009BF802460B46E6A105F13000FBF77DF942
:10FD8000E5490A98C96A69B9DFF89093D9F82C1047
:10FD900041B909F5B878D8F82C1019B908F5B87731
:10FDA000F96A49B1DE4905F13000FBF766F99DF8C3
:10FDB000180072285ED147E0DA4E306004F074F823
:10FDC000D94ADA4B03F086FF83468A46B06804F0CE
:10FDD0006BF85A46534603F03DFE03F037FBDFF85D
:10FDE00038B306463146DBF8200004F063FB824658
:10FDF000CBF818605146D9F8180004F081F8C9F81A
:10FE000018008AF0004004F04FF8C94AC94B03F0CB
:10FE100021FE06468946D8F8180004F045F84B46FE
:10FE2000324603F057FF03F011FBC8F81800B04644
:10FE30004E46B86904F038F84246334603F038FBC2
:10FE400003F004FBB861B2E7BBA105F13000FBF79A
:10FE500014F905AAAFF6501105F13000FBF7D4F8FC
:10FE6000059804F021F802460B46A9A105F13000DF
:10FE7000FBF703F9002C02F09C80AA48806804F08C
:10FE800013F80646A4480C46006A04F00DF8002258
:10FE9000B24B03F00DFB3246234603F0C5FB03F0E3
:10FEA000D5FA04F001F802460B46ADA105F1300089
:10FEB000FBF7E3F8824803F0C5F98248F9F7ECF95B
:10FEC000002800F0B18402F074B8AAA105F1300056
:10FED000FBF7D3F8AFF2CC2105F13000FBF7CDF8FA
:10FEE00006AAAFF6F45105F13000FBF78DF89DF846
:10FEF0001820AFF2C82105F13000FBF7BEF89DF8DD
:10FF00001800642828D1A0A105F13000FBF7B5F84E
:10FF10000AAAAFF60C2105F13000FBF775F80A9834
:10FF200003F0C2FF02460B4679A105F13000FBF752
:10FF3000A4F87A4E0A98F16A49B906F5B878D8F863
:10FF40002C1021B906F53879D9F82C1049B19A4905
:10FF500005F13000FBF791F89DF81800722853D195
:10FF60003CE0964F386003F09FFF954A954B03F0B5
:10FF7000B1FE82468B46B86803F096FF52465B4658
:10FF800003F068FD03F062FA07463946306A04F070
:10FF900091FAB76103F088FF654A664B03F05AFD9A
:10FFA00007460E46D8F8180003F07EFF3A4633465F
:10FFB00003F090FE03F04AFA31463E46C8F81800B6
:10FFC0000F46D9F8180003F06FFF32463B4603F0A6
:10FFD0006FFA03F03BFAC9F81800BDE77AA105F102
:10FFE0003000FBF74AF805AAAFF6E42105F130002E
:10FFF000FBF70AF8059803F057FF02460B4644A1A9
:020000040001F9
:1000000005F13000FBF739F8002C01F0D2876B487E
:10001000806803F049FF064640480C46006A03F03A
:1000200043FF0022704B03F049FE3246234603F0A3
:10003000FBFA634A634B03F041FE03F007FA03F057
:1000400033FF02460B4669A105F13000FBF715F8B6
:100050001B4803F0F7F81B48F9F71EF9002800F0D9
:10006000E38301F0A6BF65A105F13000FBF705F8B9
:10007000AFF2684105F13000FAF7FFFF06AAAFF6CC
:10008000907105F13000FAF7BFFF9DF81820AFF22C
:10009000644105F13000FAF7F0FF9DF8180064287C
:1000A00000D1B5E0D8E0000062617365203D2025F5
:1000B000312E346620726164202020200D0A000059
:1000C0000AD7A33C1402001053686F756C64657204
:1000D0002073656C65637465640D0A00456E746514
:1000E00072206465677265657320746F2074757221
:1000F0006E2073686F756C6465722028686F6D651B
:100100003D3132302E323820646567293A0D0A00BD
:1001100025660D0A000000001C0700108C08001066
:1001200044510100580E001052B81E85EB115E407C
:10013000909E2287889BCF3F456E746572207261C6
:100140006469616E7320746F207475726E207368B9
:100150006F756C6465723A0D0A00000000A9CA4010
:1001600053686F756C646572203D20252E326620C1
:100170000D000000456C626F772073656C656374D9
:1001800065640D0A00000000456E746572206465A8
:10019000677265657320746F207475726E20456C8C
:1001A000626F772028686F6D653D39352E303220BB
:1001B000646567293A0D0A00D84F0100640E0010EB
:1001C000E17A14AE47C15740456E74657220726182
:1001D0006469616E7320746F207475726E20456C53
:1001E000626F773A0D0A000080F6C440456C626F7A
:1001F00077203D20252E3266200D00005069746363
:10020000682073656C65637465640D0A0000000006
:10021000FBA105F13000FAF730FF0AAAAFF618513A
:1002200005F13000FAF7F0FE0A9803F03DFE0246B1
:100230000B46FEA105F13000FAF71FFFFD49DDF87E
:100240002890C86A18B901F5B870C26A4AB1FA496B
:1002500005F13000FAF711FF9DF8180072287CD1E3
:10026000CFE0F648016AA0F5B870006A03F048FED6
:100270004FF0FF3104F0F7F903F016FE8A46064608
:10028000EF4AF04B03F0D0F903F0E0F803F00CFE76
:10029000CDE9006A02460B46EB4905F13000FAF75A
:1002A000ECFEE448016A00F5B870006A04F002F957
:1002B00003F0FAFD4FF0FF3204F0A7F9E34AE44BF4
:1002C00003F0F6F803F0C2F803F0EEFD0F468046A7
:1002D000DB4ADC4B03F0A8F903F0B8F8394647468F
:1002E000884603F0E1FDCDE9007802460B46D94986
:1002F00005F13000FAF7C1FED7484946006803F01F
:10030000D1FF03F0D1FD07468846484603F0CCFDF7
:10031000CDE9007802460B46D04905F13000FAF7E6
:10032000ACFE38464146012204F06FF98B46074681
:100330004FF0FF3204F069F9804689463046514655
:10034000012204F062F942464B4603F0B1F803F093
:100350007DF882463E46D84600E05EE003F0A4FD0C
:10036000074632464346079103F0B4FC03F06EF8AB
:1003700006460146504604F09DF803F095FD4FF007
:10038000FF3204F042F9AE4AAE4B03F04DF903F0F0
:100390005DF883465146304603F0B2FD03F084FD1C
:1003A0004FF0FF3204F031F9A54AA64B03F03CF9B7
:1003B00003F04CF803F078FD80468946584603F078
:1003C00073FD02460B46A64905F13000CDE90089D0
:1003D000FAF753FE974930468E6103F065FD0246F9
:1003E0000B46A04905F13000FAF747FE93483A461C
:1003F0009D49C0F818A005F13000079BFAF73DFEB3
:100400002AE79AA105F13000FAF737FE05AAAFF600
:10041000087105F13000FAF7F7FD002C01F0C985ED
:100420009948C06D03F040FD064682480C46016ABB
:1004300000F5B870006A04F03DF803F035FD4FF0A8
:10044000FF3204F0E2F83246234603F0EDF802F002
:10045000FDFF03F029FD02460B468CA105F130009B
:10046000FAF70BFE8D4802F0EDFE8D48F8F714FF09
:10047000F0B301F09EBD8BA105F13000FAF7FDFD50
:10048000AFF6780105F13000FAF7F7FD06AA89A169
:1004900005F13000FAF7B8FD9DF81820AFF67401A9
:1004A00005F13000FAF7E9FD9DF81800642825D120
:1004B00081A105F13000FAF7E0FD0AAAAFF6B871A4
:1004C00005F13000FAF7A0FD0A9803F0EDFC0246B2
:1004D0000B4656A105F13000FAF7CFFD5548DDF87F
:1004E0002890C16A19B900F5B871CA6A5AB100E01A
:1004F0009AE17B4905F13000FAF7BFFD9DF818003D
:1005000072287BD157E14D494A48096A006A03F0D5
:10051000F7FC4FF0FF3104F0A6F803F0C5FC0F46DE
:100520000646474A474B03F07FF802F08FFF3946F3
:1005300037460E4603F0B8FCCDE9007602460B467E
:10054000684905F13000FAF798FD3A48016A00F56C
:10055000B870006A03F0AEFF03F0A6FC4FF0FF3264
:1005600004F053F8394A3A4B02F0A2FF02F06EFF52
:1005700003F09AFC8A460646314A324B03F054F89F
:1005800002F064FF03F090FCCDE9006A02460B46DE
:10059000554905F13000FAF770FD544849460068A6
:1005A00003F080FE03F080FC07468846484603F0CF
:1005B0007BFCCDE9007802460B464D4905F1300041
:1005C000FAF75BFD38464146012204F01EF88B46DF
:1005D00080464FF0FF3204F018F80746894630464F
:1005E0005146012204F011F84B463A4602F060FFF2
:1005F00002F02CFF824603F057FC7BE0E6E00000AF
:10060000456E746572206465677265657320746FEA
:100610002070697463682028686F6D653D2D3838D7
:100620002E383120646567293A00000025372E33C3
:10063000660D0A00FC090010025101006C0B00104D
:10064000A089B0E1E9E53B401A500100E3DD91B13A
:10065000425BA3C03D500100240100106150010025
:100660008E500100CE500100E8500100456E7465C7
:10067000722072616469616E7320746F20506974B6
:1006800063683A0D0A000000C800001050697463E6
:1006900068203D20252E3266200D00000AD7A33C9D
:1006A00014020010526F6C6C2073656C6563746586
:1006B000640D0A0025630000456E74657220646550
:1006C000677265657320746F20726F6C6C20286888
:1006D0006F6D653D302E3020646567293A0D0A0044
:1006E000644F0100674E01008A4E0100280100108E
:1006F000AC4E010042465B460491079003F0DEFADF
:1007000002F0A4FE81460146504603F0D3FE03F0FA
:10071000CBFB4FF0FF3203F078FFF84AF84B02F0C2
:1007200083FF02F093FE32905146484603F0E8FB07
:1007300003F0BAFB4FF0FF3203F067FFEF4AF04BD4
:1007400002F072FF02F082FE33904846049F079E3B
:1007500003F0AAFB80468B4642465B46E94905F119
:100760003000CDE90067FAF788FC339803F09CFB72
:1007700006460F46329803F097FB02460B46E249C5
:1007800005F13000CDE90067FAF777FCDF48424613
:100790005B46C0F81890DE4905F13000FAF76DFCB1
:1007A000DC48DD49C0F818A005F13000049B079A29
:1007B000FAF763FCA2E6D9A105F13000FAF75DFC77
:1007C00005AADDA105F13000FAF71EFC002C01F0AE
:1007D000F083DA48006E03F067FB0646CD480C460E
:1007E000016AA0F5B870006A03F08AFB03F05CFBB5
:1007F0004FF0FF3203F009FF3246234602F014FFA8
:1008000002F024FE03F050FB02460B46CCA105F19A
:100810003000FAF732FCCE4802F014FDCD48F8F76C
:100820003BFD002841F0C5830121CA48F8F7D2FDFD
:1008300001F0BFBBC74CC8A104F13000FAF71DFCA2
:1008400059AAAFF2901104F13000FAF7DDFB9DF8E0
:100850006421AFF6284104F13000FAF70EFC9DF850
:100860006401632803D0642806D0722820D0B348DE
:100870006321017001F09DBBC548C16A00F5B870E5
:10088000C06A0143C348C26A00F5B870C06A104329
:100890000143A048C06A0143BF48C06A084311BF72
:1008A000BEA16421A54801707EF4CAAF01F081BBEE
:1008B000B748C16A00F5B870C06A0143B548C26A5A
:1008C00000F5B870C06A104301439248C06A014302
:1008D000B148C06A084311BFB8A17221974801709E
:1008E0007EF4AEAF01F065BBBCA1C148FAF7C5FB11
:1008F000002C41F05E8300BFEFF78EFCDFF8F4823E
:10090000002501462A46C8FB01208211A2EBE070B7
:10091000A0EBC00000EB800001EB400003F062FCA4
:1009200003F0C2FA0022B44B02F07EFE00224FF028
:10093000804302F0BDFD02F089FD3490EFF76CFCBE
:1009400001460246AD4E2846C6FB01025011A0EBFF
:10095000E270A0EB001000EB4000084403F027F821
:100960000022A74B03F0B6F902F070FD3190EFF7CB
:1009700053FCA44F87FB00214A11A2EBE1716FF0F9
:100980001802514300EB810003F011F800229E4B46
:1009900002F08EFD02F05AFD3290EFF73DFC9B49CC
:1009A00081FB00125111A1EBE2726FF0540102FBC6
:1009B000010002F0FCFF0022954B03F08BF902F0DE
:1009C00045FD3390EFF728FC014687FB01204211DB
:1009D000A2EBE0706FF01802504301EB800002F0D0
:1009E000E6FF00228B4B03F075F902F02FFD07465E
:1009F000EFF712FC02462946C6FB0210C111A1EB1B
:100A0000E070A0EB001000EB400002EB800002F071
:100A1000CEFF0022804B03F05DF902F017FD064681
:100A2000EFF7FAFB0146C8FB00518A11A2EBE17116
:100A3000A1EBC10101EB810100EB410003F0D2FB0E
:100A400037903E480078722834D1319803F02CFA60
:100A5000724DDFF8CC812A46434602F0FBFF02F0DC
:100A6000F5FC3190329803F01FFA2A46434602F013
:100A7000F1FF02F0EBFC3290339803F015FA2A46AE
:100A8000434602F0E7FF02F0E1FC3390384603F002
:100A90000BFA2A46434602F0DDFF02F0D7FC074678
:100AA000304603F001FA2A46434602F0D3FF02F033
:100AB000CDFC0646379803F0F7F9834630460B9194
:100AC00003F0F2F9CDE90801384603F0EDF982466A
:100AD0000791339803F0E8F905460591329803F041
:100AE000E3F981460391319803F0DEF900908846DE
:100AF000349803F0D9F90B46024693E0A089B0E19F
:100B0000E9E53B40D94E0100F04E0100FC09001020
:100B1000304F01006C0B00104A4F0100456E7465A8
:100B2000722072616469616E7320746F20526F6C01
:100B30006C3A0D0A0000000025660000C800001095
:100B4000526F6C6C203D20252E3266200D00000077
:100B50000AD7A33C140200100D0A456E746572207A
:100B6000446576696365204D6F64652028633D6345
:100B70006F756E74732C20643D6465677265657370
:100B80002C20723D72616469616E73293F0D0A0009
:100B9000AC0500108C080010DC0C00100D0A45722A
:100BA000726F72206368616E67696E6720746F2070
:100BB000646567206D6F6465210D0A000D0A45723A
:100BC000726F72206368616E67696E6720746F2050
:100BD000726164206D6F6465210D0A000D0A507208
:100BE000657373207120746F20717569740D0A002C
:100BF00044020010EBA00EEA00002440B7600BB6E0
:100C0000004036401F85EB51000034406160606059
:100C100000204040000049400080564070E20DA591
:100C200045DF913FCDF828B0CDF818A00495EDA18F
:100C3000FB48CDE90189FAF720FA37980097CDE90A
:100C40000160DDE93330DDE93112F4F741FEF54DA5
:100C5000DFF8D4B305F5B87605F5387705F58A6879
:100C600005F5B86905F5E66A55E031A8009037AB9F
:100C700036AA35A933A8F7F7C3FDEC48FBF7F4F81B
:100C800003F012F9CDE90601319803F00DF9CDE931
:100C90000401379803F008F934900391369803F073
:100CA00003F900900291359803F0FEF8019132901B
:100CB000339803F0F9F802460B46DDE90601CDE969
:100CC0000801DDE90401CDE9060103993498CDE975
:100CD000040102990098CDE9020132980090D4A154
:100CE000CF48FAF7CAF9DF4802F0ACFADE48F8F765
:100CF000D3FA58B90121DC48F8F76CFBC0B271286F
:100D000014BF5128012401D020281DD0DBF8100089
:100D1000002818BF0124A86E00281CBFB06E002850
:100D200026D0B86E00281CBFD8F8680000281FD055
:100D3000D9F8680000281CBFDAF86800002817D02E
:100D4000002C92D001F035B9B6490420886601F52F
:100D5000B871886601F5B871886601F5B871886662
:100D600001F5B871886601F5B871886601F021B99E
:100D7000002C3FF4C1AD01F01CB90020BA4C2E90FC
:100D8000BAA104F13000FAF778F929AAAFF2DC61D0
:100D900004F13000FAF738F99DF8A420BEA104F15F
:100DA0003000FAF76AF9BEA104F13000FAF765F9EC
:100DB0009DF8A40070286FD00ADC62280ED0652848
:100DC0006BD0672808BFC24D00F03E8301F0F1B838
:100DD000722874D0732874D001F0EBB8DFF8F49265
:100DE000BD4F904DDFF840A20DF59C7801219E4843
:100DF000F8F7F0FAC6B28DF8A4602B2E04D138466D
:100E0000A96903F07DF8A8612D2E02D0632E05D0CC
:100E10001FE04846A96903F073F819E0AFA104F197
:100E20003000FAF72AF92EAAB3A104F13000FAF73C
:100E3000EBF82E9803F038F80B460246AFA104F108
:100E40003000FAF71AF92E9803F090F903F0CAF976
:100E5000A8614FAB53AA52A951A8CDF80080F7F76B
:100E6000CFFC9AF800007228519817D003F01CF8B4
:100E700006468B46A86903F017F8CDE9006B0246D9
:100E80000B46A0A104F13000FAF7F7F89DF8A40092
:100E90007128ABD101F08DB8F9E18FE103F004F8CE
:100EA00006468B46A86902F0FFFFCDE9006B0B46B2
:100EB00002469CA104F13000FAF7DFF8E6E755E2BC
:100EC000FFE7A14DDFF87CA205F5B87705F5387886
:100ED00005F58A6901216448F8F77CFAC6B28DF8F5
:100EE000A4602B2E25D1DFF864B2A969584603F01F
:100EF00007F8A8615846B96903F0D1FAB861D8F883
:100F0000180002F0D1FFDFF848B253465A4602F00B
:100F1000E1FE02F09BFAC8F81800D9F8180002F0B8
:100F2000C3FF5A46534602F0C3FA02F08FFAC9F8DB
:100F300018002D2E02D0632E25D03FE0834EA969E4
:100F4000304603F0ACFAA8613046B96902F0D8FF28
:100F5000B861D8F8180002F0A7FF7D4E534632461C
:100F600002F0A6FA02F072FAC8F81800D9F81800D0
:100F700002F09AFF3246534602F0ACFE02F066FAE7
:100F8000C9F818001AE073A104F13000FAF775F8F7
:100F90002EAA59A104F13000FAF736F82E9802F083
:100FA00083FF02460B4655A104F13000FAF765F8BD
:100FB0002E9803F0DBF803F015F9A8614EA8009015
:100FC0004FAB53AA52A951A8F7F71AFC164800785C
:100FD0007228529804D002F067FF06468B46C9E09B
:100FE000DBE00000743D25372E336620623D253757
:100FF0002E336620733D25372E336620653D253719
:101000002E336620703D25372E336620723D2537FE
:101010002E336620673D25372E33660D0A0000000B
:1010200044020010AC050010C8000010C9000010F8
:10103000423D25372E336620533D25372E3366201B
:10104000453D25372E336620503D25372E3366200B
:10105000523D25372E336620473D25372E33666DAA
:101060006D0D00000AD7A33C140200100D0A456E56
:1010700074657220726F626F74206A6F696E74207B
:10108000746F206368616E67652028627365707293
:1010900067290D0A0000000025630D0A000000000A
:1010A000456E746572202B2F2D2F632F71202869B8
:1010B0006E6372656D656E742C2064656372656D18
:1010C000656E742C2071756974290D0A000000008A
:1010D000DC0C001000008CC200008C42456E746570
:1010E0007220636F756E747320746F206D6F7665F8
:1010F00020626173653A00002564000025640D0AD2
:1011000000000000426173653A20636F756E74736E
:101110003D252E3166206465673D252E32660D0A19
:1011200000000000426173653A20636F756E74734E
:101130003D252E3166207261643D252E33660D0AF1
:10114000000000003BAB2A401C0700100000584282
:10115000CA350532456E74657220636F756E74739F
:1011600020746F206D6F76652073686F756C646591
:10117000723A0000A86902F097FECDE9006B0B46B9
:101180000246FBA104F13000F9F777FF9DF8A400B7
:1011900071287FF49FAE00F00CBF02F085FE06467A
:1011A0008B46A86902F080FECDE9006B02460B4633
:1011B000F8A104F13000F9F760FFE7E7FE4DFF4EBC
:1011C0004EAF0121FE48F8F705F9C0B28DF8A40032
:1011D0002B2804BF3620F7F78FF99DF8A4002D289F
:1011E00004BF3620F7F72EFA9DF8A40063281CD11F
:1011F000F4A104F13000F9F740FF2EAAAFF2081174
:1012000004F13000F9F700FF2E9802F04DFE02467F
:101210000B46AFF2181104F13000F9F72EFF2E98AB
:1012200002F0A4FF02F0DEFFA8614FAB53AA52A95F
:1012300051A80097F7F7E4FA30787228539815D040
:1012400002F032FE80468946A86902F02DFE0B4668
:101250000246E3A104F13000CDE90089F9F70DFF62
:101260009DF8A4007128ACD100F0A3BE02F01CFED2
:1012700080468946A86902F017FE02460B46E0A1A7
:1012800004F13000CDE90089F9F7F7FEE8E7E44D15
:10129000DFF828A305F5B8760121C948F8F79AF8D0
:1012A000C7B28DF8A4702B2F0BD1DFF87883A96912
:1012B000404603F0F4F8A8614046B16902F020FE10
:1012C000B0612D2F02D0632F0CD010E0D64FA9694A
:1012D000384603F0E4F8A8613846B16902F010FE20
:1012E000B06104E0D1A104F13000F9F7C6FE4EA8C8
:1012F00000904FAB53AA52A951A8F7F781FA9AF878
:10130000000072284F981BD002F0CEFD81468B461C
:10131000B06902F0C9FD07468846A86902F0C4FD1D
:101320008DE8800B02460B46CAA104F13000F9F7A4
:10133000A4FE00BF9DF8A4007128ADD100F039BE15
:1013400002F0B2FD81468B46B06902F0ADFD074662
:101350008846A86902F0A8FD8DE8800B02460B467E
:10136000C8A104F13000F9F788FEE3E7AC4DDFF8DF
:101370004CA205F5B87601219148F8F72BF8C7B2D1
:101380008DF8A4702B2F0BD1DFF89882A969404605
:1013900002F0B6FDA8614046B16902F0B1FDB0614E
:1013A0002D2F02D0632F0CD010E09F4FA969384633
:1013B00002F0A6FDA8613846B16902F0A1FDB06156
:1013C00004E09AA104F13000F9F757FE4EA800900E
:1013D0004FAB53AA52A951A8F7F712FA9AF8000096
:1013E00072284E981AD002F05FFD81468B46B06994
:1013F00002F05AFD07468846A86902F055FD8DE8BF
:10140000800B0B460246ABA104F13000F9F735FE24
:101410009DF8A4007128AED100F0CBBD02F044FDD0
:1014200081468B46B06902F03FFD07468846A869B1
:1014300002F03AFD8DE8800B02460B46A9A104F1AB
:101440003000F9F71AFEE3E701215D48F7F7C2FF24
:10145000C0B28DF8A4002B280ED1AE48296A814273
:1014600005DAAD48A96902F04BFDA86104E0ABA123
:1014700004F13000F9F701FE9DF8A4002D280ED1EB
:10148000286AB0F5000F05DBA348A96903F007F847
:10149000A8613BE0A8A104F13000F9F7EEFD9DF84A
:1014A000A400632832D1AAA104F13000F9F7E5FDC8
:1014B0002EAAAFF2BC3104F13000F9F7A5FD2E9849
:1014C00002F0F2FC02460B46A8A104F13000F9F745
:1014D000D4FDE96D2E9802F0B1FE06D2296E2E9849
:1014E00002F0ACFF38BF2E98D2D3286E02F0DCFC9D
:1014F00006460F46E86D02F0D7FC0B4602469EA159
:1015000004F13000CDE90067F9F7B7FD286A02F071
:101510002DFE02F04CFA07468846A24AA24B02F082
:1015200099FA0646894638464146A04AA04B02F041
:1015300091FA3A46434602F08DFA32464B4601F0A4
:10154000B7FF01F083FF064638464146994A9A4B59
:1015500002F080FA81468A4638464146974A984BBF
:1015600002F078FA3A46434602F074FA4A4629E114
:1015700053686F756C6465723A20636F756E74732F
:101580003D252E3166206465673D252E32660D0AA5
:101590000000000053686F756C6465723A20636FD9
:1015A000756E74733D252E3166207261643D252E63
:1015B00033660D0A000000008C080010C8000010FF
:1015C00014020010456E74657220636F756E74733B
:1015D00020746F206D6F766520656C626F773A00BE
:1015E000456C626F773A20636F756E74733D252E7C
:1015F0003166206465673D252E32660D0A000000C5
:10160000456C626F773A20636F756E74733D252E5B
:101610003166207261643D252E33660D0A0000009C
:10162000FC0900100000E0410000E0C1636F756E2E
:101630007473206E6F7420616E206F7074696F6EAA
:1016400020666F72207069746368207965740D0A72
:101650000000000050697463683A20636F756E740F
:10166000734178343D252E316620636F756E747337
:101670004178353D252E3166206465673D252E3243
:10168000660D0A0050697463683A20636F756E7462
:10169000734178343D252E316620636F756E747307
:1016A0004178353D252E3166207261643D252E330B
:1016B000660D0A00526F6C6C3A20636F756E74731E
:1016C0004178343D252E316620636F756E74734109
:1016D00078353D252E3166206465673D252E3266BE
:1016E0000D0A0000526F6C6C3A20636F756E747354
:1016F0004178343D252E316620636F756E747341D9
:1017000078353D252E3166207261643D252E336685
:101710000D0A000000609F45000020413531303047
:10172000206D6178206F70656E20726561636865F9
:101730006421210D0A00000030206D617820636C67
:101740006F7365207265616368656421210D0A000D
:10175000456E74657220636F756E747320666F7268
:1017600020677269707065720D0A0000636F756E94
:1017700074733D25640D0A00436F756E7473206F9A
:101780007574206F662072616E676520286D6178C0
:101790003D252E31662C206D696E3D252E31660D5E
:1017A0000A0000003BDF4F8D976E923F8DEDB5A094
:1017B000F7C6A0BEC7BAB88D06F0463F3A8C30E2F5
:1017C0008E7955BE534601F073FE01F03FFE074689
:1017D000686F02F069FB82468B46384602F064FB74
:1017E00080468946304602F05FFB06460F46A869F0
:1017F00002F05AFB8DE8C00F02460B46F9A104F136
:101800003000F9F73AFC9DF8A40071287FF41CAE73
:1018100000F0CFBB642110A8EFF77AF9FE4F322118
:1018200010A87A69F6F744FF8146AFF29C2110A810
:10183000EFF730F9786AD0B1DFF8E083F84E002492
:1018400010ADF8A12A5D06F13000F9F716FC40460C
:10185000641C01F0F7FC285D0028F2D1786A30B1F1
:1018600010AB4A46F0A106F13000F9F706FCAFF6DE
:10187000245110A8EFF79EF82DA9009149AB2AAA90
:10188000CDE901232CAB2BAAF0A1EEF7D9FE052858
:1018900006D0F848F1A100BFF9F7EFFB00F089BBD3
:1018A00049980090DDE92B012A9B2D9AF7F7FAFA67
:1018B000F148F4F71BFD02F095FC796A51B102F092
:1018C000F3FA02460B46EB48ECA100BFF9F7D5FB53
:1018D00000F06FBBEDA1E748F9F7CFFB00F069BB63
:1018E000EC48C06A70B9EC48C06A58B9EB48C06AA5
:1018F00040B9EB48C06A28B9EA48C06A10B9EA485A
:10190000C06A40B1E9A1DB48F9F7B7FBED4801F047
:1019100099FC00F04EBBC04F786A18B1EAA1D548D7
:10192000F9F7ABFB642130A8EFF7F2F8322130A8C9
:101930007A69F6F7BDFE8146D5A130A8EFF7AAF87F
:10194000786AD0B1DFF8D482B54E002430ADB5A1AD
:101950002A5D06F13000F9F790FB4046641C01F067
:1019600071FC285D0028F2D1786A30B130AB4A466C
:10197000ADA106F13000F9F780FBAFF6306130A879
:10198000EFF718F80DF5967C49AB2AAA2DA98DE83A
:101990000E102CAB2BAAD6A1EEF752FE062808D0CB
:1019A000AEA1B448F9F769FBC64800BF01F04AFC94
:1019B000FFE23C78722C33D12B9802F075FAD14DAE
:1019C000D14E2A46334602F045F801F03FFD2B90F8
:1019D0002C9802F069FA2A46334602F03BF801F0EF
:1019E00035FD2C902D9802F05FFA2A46334602F01E
:1019F00031F801F02BFD2D902A9802F055FA2A4675
:101A0000334602F027F801F021FD2A90499802F0B0
:101A10004BFA2A46334602F01DF801F017FD4990B3
:101A2000BA492B98884202DCB949884200D92B91E7
:101A3000B8492C988842C8BF2C9104DC10F1FF4FA4
:101A400024BF00202C90B4482D99814202DCB34879
:101A5000814200D92D90B2482A99814202DCAF48D8
:101A6000814200D92A90AF484B998142C8BF4B9020
:101A700004DC11F1FF4F24BF00204B90722C33D1B6
:101A80002B9802F011FAA84CA84D22462B4601F0E3
:101A9000E1FF01F0DBFC2B902C9802F005FA2246C6
:101AA0002B4601F0D7FF01F0D1FC2C902D9802F0CD
:101AB000FBF922462B4601F0CDFF01F0C7FC2D902B
:101AC0002A9802F0F1F922462B4601F0C3FF01F0FB
:101AD000BDFC2A90499802F0E7F922462B4601F016
:101AE000B9FF01F0B3FC49904B48406A30B34B98C2
:101AF00002F0DAF982468B46499802F0D5F9804621
:101B000089462A9802F0D0F906460F462D9802F031
:101B1000CBF904460D462C9802F0C6F9509001917D
:101B20002B9802F0C1F90B4602A981E8F00F509AF8
:101B3000009202467EA14F48F9F79FFA499800901B
:101B4000DDE92B012A9B2D9AF7F7ACF956484B9902
:101B500081614C9802F0A8F904460D46824A834BF5
:101B600001F078FF22462B4601F0A2FC01F06EFC4A
:101B7000F4F7BCFB02F036FB2749496A00293FF421
:101B8000A9AE00BF02F090F902460B463BA13948CE
:101B9000F9F773FA0DE2204F642110A87A69F6F77D
:101BA00087FD81463AA110A8EEF774FF786AB8B1B4
:101BB000DFF868801A4E002410AD1AA12A5D06F1E4
:101BC0003000F9F75AFA4046641C01F03BFB285DEF
:101BD0000028F2D1786A18B110AB4A4612A1C7E0CA
:101BE000CAE00000477269707065723A20636F75D1
:101BF0006E74733D252E3166206D6D3D252E336646
